:020000040800F2
:10000000B8F20120B50200082D900008D17D00084B
:10001000CD8E0008A92A000889AB00080000000066
:100020000000000000000000000000001197000820
:10003000094000080000000091920008419B000860
:10004000CF020008CF020008CF020008CF0200084C
:10005000CF020008CF02000841430008CF02000889
:10006000CF0200084D43000859430008CF020008A2
:10007000A13E0008CF020008CF020008CF0200080E
:10008000CF020008CF020008CF020008CF0200080C
:10009000AD2A0008BD2A0008CF0200086543000809
:1000A0000D9C0008CF020008CF020008CF02000814
:1000B000CF020008CF020008CF020008CF020008DC
:1000C000CF020008CF020008CF020008CF020008CC
:1000D000CF02000841AB0008CF02000859AB00086E
:1000E000CF020008CF020008CF020008CF020008AC
:1000F000CF020008CF020008CF020008CF0200089C
:10010000CF020008CF020008CF020008CF0200088B
:10011000CF020008CF020008CF020008CF0200087B
:10012000CF020008B13E0008C13E0008D13E0008E1
:10013000CF020008CF020008CF020008CF0200085B
:10014000CD2A0008DD2A0008CF020008CF020008EF
:10015000CF020008E13E0008CF02000871AB0008A2
:10016000CF020008CF020008CF020008CF0200082B
:10017000CF020008CF020008CF02000800000000F4
:10018000CF020008CF02000800F002F800F082F869
:100190000AA090E8000C82448344AAF10107DA45E2
:1001A00001D100F077F8AFF2090EBAE80F0013F0B2
:1001B000010F18BFFB1A43F001031847540B01004D
:1001C000940B01000A444FF0000C10F8013B13F0AF
:1001D000070408BF10F8014B1D1108BF10F8015BA0
:1001E000641E05D010F8016B641E01F8016BF9D193
:1001F00013F0080F1EBF10F8014BAD1C0C1B09D1EA
:100200006D1E58BF01F801CBFAD505E014F8016B5B
:1002100001F8016B6D1EF9D59142D6D370470000ED
:10022000103A24BF78C878C1FAD8520724BF30C822
:1002300030C144BF04680C607047000000230024F4
:1002400000250026103A28BF78C1FBD8520728BFE6
:1002500030C148BF0B607047662910F006837529CE
:1002600000F01C81632900F06485732900F0698522
:10027000002070471FB510F0E6FA00F0E8F900F032
:1002800065FD0400002000210FF050FBE0601FBD61
:1002900010B510BD00F05EFE1146FFF7EBFF0AF04F
:1002A0005DFF00F07CFE03B4FFF7F2FF03BC00F03B
:1002B000BDFE00000948804709480047FEE7FEE709
:1002C000FEE7FEE7FEE7FEE7FEE7FEE7FEE7FEE706
:1002D00004480549054A064B70470000F99B000891
:1002E00089010008B8DD0120B8F20120B8E2012040
:1002F000B8E2012053EA020C00F069802DE9F04BCE
:100300004FF00006002B1FBFB3FA83F503FA05F484
:1003100024FA05F65E4012BF1643B2FA82F502FADD
:1003200005F4C5F120051EBF22FA05FC44EA0C04C1
:10033000203556EA044C4FEA144418BF641C4FF0B1
:1003400000084FF00009904271EB030C39D30029EB
:1003500019BFB1FA81F701FA07F6B0FA80F700FA8F
:1003600007F6C7F120071EBF20FA07FC46EA0C0675
:100370002037B6FBF4FCA7EB0507103F07F01F0B77
:10038000CBF120062CFA06F60CFA0BFB44BFB34661
:100390000026202FA4BF5E464FF0000B5BEA060C40
:1003A00008BF4FF0010B19EB0B0948EB0608ABFB3C
:1003B000027C06FB02CC0BFB03CCC01B71EB0C01D7
:1003C000C1E70B46024641464846BDE8F08B13B5EF
:1003D000084318BF4FF0FF300146AFF30080BDE87F
:1003E0001C4070470FB41CB5084B06AA7B446946F5
:1003F0000090059800F073FC04460020694600F068
:1004000081FC20461CBC5DF814FB000015090000AF
:100410000FB47CB50C0009AA009001D02044401E06
:10042000084B7B4469460190089800F058FC05464B
:100430001CB10020694600F065FC28467CBC5DF8D4
:1004400014FB0000E908000070B50C460546012ABF
:1004500005D02878800600D5EA69002302E0012350
:1004600005E05B1C934202D2E05C0028F9D1A86948
:10047000E618C01AA861286A184428622846AFF313
:10048000008004E0D5E9012114F8010B9047B44243
:10049000F8D32846AFF3008070BD00002DE9F0418D
:1004A0000646002410687529314616A510D0AFF312
:1004B0000080002802DA404213A507E031688A076D
:1004C00001D512A502E0490704D511A5012401E0D8
:1004D000AFF3008000210A2206F1240709E0B0FBF7
:1004E000F2FCB0FBF2F302FB1C00303078541846EB
:1004F000491C0028F3D123462A463046BDE8F04186
:1005000000F081B9000000002D0000002B00000069
:10051000200000002DE9F0474FF0000A894604460C
:10052000C0F820A02046E1688847002876D025281A
:1005300006D0D4E901219047206A401C2062F1E7EF
:10054000E168204600258847C4F81CA0064600271D
:10055000C4F818A02A2E09D030460FF0ADF938B3F0
:1005600004EB8708303EC8F8186019E059F8041BFE
:10057000204604EB87029161E1688847012F064617
:1005800018D1E069002820DA25F020051DE0D8F810
:10059000180000EB800006EB40003038C8F8180067
:1005A0002046E168884706460FF086F90028EED11C
:1005B000012F0AD02E2E08D12046E16888477F1CE3
:1005C0000646022F45F02005C4DBA069002803DAA7
:1005D000404245F00105A061E80701D025F0100573
:1005E000B6B1A6F14100192802D8203645F40065BD
:1005F0004A463146204625604D46FFF72DFE58B14C
:10060000012806D0ED1D25F0070000F1080989E753
:1006100004E005F1040985E730468AE7206ABDE871
:10062000F08700000B4910B5A1F17C020A4CC2E929
:100630003712372106E000EB104342F82130074B18
:1006400000FB03400B1EA1F10101F4DC10BD0120F1
:10065000E8E700002C050020E119D666CD0D010069
:1006600010B5431C02E010F8011B71B18107FAD1EB
:100670004FF0013202C88C1A8C4314EAC211F9D02F
:10068000C01A0A0603D0C01E10BDC01A10BD0A044D
:1006900001D0801E10BD0902FCD0401E10BD032AEF
:1006A00040F2308010F0030C00F0158011F8013B8F
:1006B000BCF1020F624498BF11F801CB00F8013B76
:1006C00038BF11F8013BA2F1040298BF00F801CB3A
:1006D00038BF00F8013B11F0030300F02580083A11
:1006E000C0F0088051F8043B083A51F804CBA0E868
:1006F0000810F5E7121D5CBF51F8043B40F8043BBD
:10070000AFF30080D20724BF11F8013B11F801CBF1
:1007100048BF11F8012B24BF00F8013B00F801CBC2
:1007200048BF00F8012B704710B5203AC0F00B808D
:10073000B1E81850A0E81850B1E81850A0E81850D7
:10074000203ABFF4F5AF5FEA027C24BFB1E818504D
:10075000A0E8185044BF18C918C0BDE810405FEAAF
:10076000827C24BF51F8043B40F8043B08BF70472B
:10077000D20728BF31F8023B48BF11F8012B28BF30
:1007800020F8023B48BF00F8012B704702F0FF033E
:1007900043EA032242EA024200F002B84FF00002AC
:1007A00000B5134694469646203922BFA0E80C5067
:1007B000A0E80C50B1F12001BFF4F7AF090728BF42
:1007C000A0E80C5048BF0CC05DF804EB890028BFBE
:1007D00040F8042B08BF704748BF20F8022B11F0E7
:1007E000804F18BF00F8012B704770477047704763
:1007F00010B500F0AFFA006810BD10B5044600F067
:10080000A9FA046010BD2DE9F0470D4699469246BD
:10081000044600F124080168880604D5E06921F047
:100820001001216000E00120A84201DD471B00E02B
:100830000027A1697A1902EB0900081AA061207843
:10084000C00602D42046AFF30080002608E0D4E9B9
:1008500001211AF806009047206A401C761C20628D
:100860004E45F4DB2078C0060AD52046AFF3008061
:1008700006E0D4E9012130209047206A401C206224
:10088000381EA7F10107F4DC07E0D4E9012118F8CC
:1008900005009047206A401C2062281EA5F1010532
:1008A000F3DC2046AFF300802078000602D502205A
:1008B000BDE8F0870120FBE72DE9FF4F0C461E46FF
:1008C0004FF0FF378BB0D2E90001DDF860800A906D
:1008D0008A46C1F30A5505B93D46002108464FF046
:1008E0000000BAF1000F00F4400005DA00EB8000D0
:1008F0004FF4400101EA50004FEA9059B9F1010F5D
:1009000000DDB9460A9850EA4A000ED044F610506D
:10091000A5F2FF3545432F14B8F1000F1ED07542E4
:10092000291E1EDDC9F100021CE0B8F1010F4FF0D5
:10093000000001D0302103E0F24305E02154401CC7
:10094000B042FBDB30460022002121540B99C1F854
:100950000880C1E900200FB0BDE8F08FBD1B6D1C01
:10096000DEE74A4600DA694206A800F07DFA06ABE7
:1009700093E8070003AB83E8070050460A990DF09F
:10098000F1FA8DE80700A0F500501F380090039899
:10099000002D0ADD42F21F014A460844002303A944
:1009A000039068460DF05AFD09E0A0F500504A4654
:1009B0001F38002303A9039068460DF064FD8DE8FD
:1009C00007000004000C03D04FF0FF30410800E0A6
:1009D0001046B8F1000F03D00022009215461EE029
:1009E000751E05D400F0BAF9303262556D1EF9D586
:1009F000B3460122084302D000227F1C04E0207885
:100A0000302801D100227F1E002A099784D01DE0E2
:100A1000112D07DA00F0A2F9303262556D1C50EA50
:100A20000102F5D1084302D00098C8B10EE00021C0
:100A3000681E05E0235C625C63542254401E491C1E
:100A40008142F7DBAB46A81B401E0990002004F84A
:100A50000B000B98099AC0F80880C0E9002B7AE7D0
:100A600011264FF0000857E72DE9F04F884604465D
:100A7000D21D22F0070191B0D1E90001CDE90A01B0
:100A80000DF038FE02460B98C00F01D02D2007E074
:100A90002068810701D52B2002E0202101EAC00057
:100AA000032A099001D0072A05DB03464146204668
:100AB00000F09AF90BE12078800601D5E06900E0AA
:100AC0000620B8F1650F814606D0B8F1660F18D040
:100AD000B8F1670F70D131E00020B9F1110F00902B
:100AE00001DB112301E009F101030AAA01A90CA805
:100AF000FFF7E2FEDDE90C70002609F101058346EF
:100B000047E001204B4600904FF000470AAA01A998
:100B10000CA8FFF7D1FEDDE90DB00C995D4600266B
:100B200010B909F101000D18B9EB050003D4C0F1AB
:100B3000FF3609F10105A5EB09002BE0B9F1010F22
:100B400001DA4FF001090020B9F1110F0090484679
:100B500001DD112300E003460AAA01A90CA8FFF752
:100B6000ABFEDDE90C704D46002683462078000779
:100B70000AD4AB4500DA5D4601A8012D04DD411918
:100B800011F8011C302907D04F4502DA17F1040F84
:100B900004DA012082460FE06D1EEEE7002F02DC32
:100BA000ED1B3E4403E0781CA84200DD7D1CB81B11
:100BB00000F1010A4FF000472078000703D4AA454E
:100BC00001DB4FF0FF3A0021B7F1004F0DF1430870
:100BD0008DF8431024D002202B23002F01DA7F420E
:100BE0002D230A21021EA0F1010000DC5FB197FB5A
:100BF000F1FC97FBF1F201FB1C7C17460CF1300C69
:100C000008F801CDEEE7A8F101000370218809057D
:100C100001D5452100E06521A0F1010800F8011C83
:100C200009980FA9A1EB0807FF1D00B10120411988
:100C300001EBEA70A1693844081A401EA0612078CF
:100C4000C00602D42046AFF30080099828B1D4E949
:100C500001219047206A401C20622078C00622D5DE
:100C60002046AFF300801EE0002E04DBB34502DD1A
:100C700001A8805D00E03020D4E901219047206A7E
:100C8000401C2062761CAAF101005FEA000A0AD12A
:100C900000F05CF8C0680168405CD4E9012190472D
:100CA000206A401C2062281EA5F10105DCDC07E05B
:100CB000D4E9012118F8010B9047206A401C2062FA
:100CC000381EA7F10107F3DC2046AFF300800320B4
:100CD00011B041E601694A1C02610878704700B50D
:100CE0008FB0CDE901310021059105497944CDE965
:100CF000031011466846FFF70DFC0FB000BD000061
:100D0000E5FFFFFF0A6802F8010B0A607047D1E9AE
:100D100000239A4202D2531C0B601070704710B52A
:100D2000436913B1AFF3008001E0FFF78DFB0120B1
:100D300010BD127800F124010A7000224A700122CD
:100D4000EDE711684FF0FF32E9E700000048704717
:100D5000B4050020004870479405002030B5B0F17C
:100D60000A0271F100034FEA900E4EEA817EB0EB69
:100D70000E0061EB91014FEA101E4EEA017E10EB6E
:100D80000E0041EB11114FEA102E4EEA016E10EBEE
:100D90000E0041EB11214FEA104E4EEA014E10EBCE
:100DA0000E0041EB1141401841F100014FEAD00023
:100DB00040EA41704FEAD1014FEA810444EA90745D
:100DC00010EB800544EB01046D1944EB0404521B45
:100DD000A3414FF0000348BF0A3200D530BD401C8C
:100DE00041F1000130BD00002DE9F0411F460446ED
:100DF00003260168072A01F4006004DB08B116A588
:100E000005E016A503E008B115A500E015A521F041
:100E100010002060A069C01EA0610FB1401EA0613B
:100E20002046AFF300804FB1D4E901213846904706
:100E3000206A401C2062C01C206206E0206AFAE79B
:100E4000D4E9012115F8010B9047761EF8D220460F
:100E5000AFF30080BDE8F0814E414E006E616E0040
:100E6000494E4600696E66002DE9F04781461646F8
:100E70008AB0354878440DC88DE80D003248784472
:100E8000801C03AC0DC884E80D0041F69B3008447B
:100E9000372190FBF1F290FBF1F5A5F1800501FB04
:100EA00012041B3C02D56442012000E00020DFF860
:100EB00098A080460027FA44AAF1BE0A0EE0E00797
:100EC0000AD03246684607EB470101230AEB81014D
:100ED0000DF0D9FA8DE8070064107F1C002CEED1CC
:100EE000194F7F44AE3F19E0E80715D007EB041017
:100EF0000DF1180A90E80E008AE80E00C068F04272
:100F000001D1981908903246012306A903A80DF0D3
:100F1000BAFA03AB83E807006D10641C002DE3D11F
:100F20004FF0010332466946B8F1000F03A802D022
:100F30000DF094FA01E00DF0A6FAC9E90001C9F834
:100F400008200AB0BDE8F08734FB00000048704775
:100F5000940500207546FFF7F9FFAE460500694687
:100F6000534620F00700854618B020B5FFF7B0F9CA
:100F7000BDE820404FF000064FF000074FF000089A
:100F80004FF0000BAC46ACE8C009ACE8C009ACE8D7
:100F9000C009ACE8C00921F007018D46704710B5C3
:100FA0000446AFF300802046BDE81040FFF77BB950
:100FB00030B44FF0013C50F8042B51F8043BCCFA0C
:100FC00052F4D51A20D1FCB950F8042B51F8043B47
:100FD000CCFA52F4D51A17D1B4B950F8042B51F801
:100FE000043BCCFA52F4D51A0ED16CB950F8042B4C
:100FF00051F8043BCCFA52F4D51A05D1002CDAD0C2
:1010000030BC4FF00000704729BAB1FA81F111F0FD
:101010001801D1F120008440F2D1CA40CB4012F037
:10102000FF0213F0FF0330BCD01A704701491820AB
:10103000ABBEFEE72600020070470000B0B52DED04
:10104000028B044600284FF0FF0061D00D460029B6
:101050005ED095ED000A95ED011A95ED022A95ED09
:10106000033A20EE010A22EE033A21EE011A22EEA3
:10107000022A31EE021A30EE030A31EE011AB7EEFF
:10108000008A30EE000A78EE410A0DF061FEB0EE03
:10109000401A95ED000A95ED012A95ED023A95ED7D
:1010A000034A20EE030A24EE022A30EE420A30EE12
:1010B000000AB0EEC02AB4EE482AF1EE10FA84ED30
:1010C000011A02DA0DF042FB01E009F0D5FF84EDD0
:1010D000020A95ED000A95ED011A95ED032A95EDAA
:1010E000023A20EE020A21EE031A30EE010A23EE44
:1010F000031A22EE022A32EE011A31EE011A30EE04
:10110000000A78EE410A0DF023FE002084ED000A6B
:1011100040B2BDEC028BB0BD70B52DED028B002846
:101120004FD0B7EE001A81EE000A0D4604464FF08C
:101130007E51002D80ED040A4FF00000C4E900103C
:10114000A060E06000F09F80D5E900600FF0B0FA89
:1011500041EC180B30460FF0ABFA41EC110BB0EE3E
:10116000480AF0EE680A0DF0F3FC51EC100B0EF09B
:10117000FFFB95ED000AB5EE400AF1EE10FA22D120
:1011800095ED010AB5EE400AF1EE10FA1BD195ED8E
:10119000020AB5EE400AF1EE10FA14D140F2C56031
:1011A000C3F64D7044F62D214AF2564244F2AD7317
:1011B000C3F60D41CBF63932C3F619730FC40020C4
:1011C00061E0FF205FE09FED321A00EE100AB4EEFE
:1011D000410AF1EE10FA1EDCB5EE400AF1EE10FA0B
:1011E00019DB9FED2C2AB4EE420AF1EE10FA25DC51
:1011F000B4EE410AF1EE10FA20DB9FED271AB4EEAF
:10120000410AF1EE10FA2CDCB4EE420AF1EE10FACB
:1012100027DB002037E045F66E10C3F67F7045F2FD
:101220000C3148F6AB0249F28553C3F6B011CBF648
:10123000BB32C3F697530FC4002024E040F2C560D0
:10124000C3F64D7044F62D214AF2564244F2AD7376
:10125000C3F60D41CBF63932C3F619730FC4002023
:1012600011E040F2C560C3F64D7044F62D214AF2FC
:10127000564244F2AD73C3F60D41CBF63932C3F694
:1012800019730FC4002040B2BDEC028B70BD00BFCB
:10129000DB0FC9BFDB0F49C00000B4C20021C0E9A9
:1012A0000011816070470000B0B52DED108B8EB03D
:1012B000044600284FF0FF0018BF002904D140B2B7
:1012C0000EB0BDEC108BB0BD002AF8D04CF200057A
:1012D0004EF69E70C2F20105C3F627502860C3B1D6
:1012E00093ED00EA93ED01FAD3ED028AB5EE40EA00
:1012F000F1EE10FA11D1B5EE40FAF1EE10FA0CD180
:10130000F5EE408AF1EE10FA07D1204600F094FA8B
:10131000D5E7204600F090FAD1E792ED000A92ED71
:10132000011A94ED014A94ED025A92ED022A94EDCD
:10133000036A94ED003A24EE407A61EE050A37EE36
:10134000607A62EE060A37EE607A60EE030A62EEB9
:10135000051A71EEA00A61EE061A70EEE10A61EE5E
:10136000031A62EE042A22EE032A21EE041A91EDFA
:1013700000DA71EEE21A20EE066A31EE021A20EE71
:10138000050A36EE216AD1ED019AD1ED02AA31EEBD
:10139000400AB6EE001AB5EE40DA27EE015A60EECA
:1013A000810A26EE017AF1EE10FA20EE016A0AD1E6
:1013B000F5EE409AF1EE10FA05D1F5EE40AAF1EE05
:1013C00010FA00F0EC812DEE0D0A29EEA91A30EE8C
:1013D000010A2AEEAA1A30EE010A8DED0D6A8DED92
:1013E0000C7ACDED0B0A8DED0A5A06F0F3FC2DEECA
:1013F000001A8DED071A29EE801A2AEE800A8DED6B
:10140000081A8DED090A2EEE0E0A2FEE0F1A30EE95
:10141000010A28EEA81A30EE010A06F0DBFC94ED72
:10142000001A6EEE00DA6FEE00AA94ED034A31EE78
:1014300001EA68EE808A94ED012A94ED023A2AEEE0
:101440008E6A61EE01EA8DED026A28EE8E0A2DEEBB
:10145000AE5A26EE046A62EE02BA35EE465A20EE25
:10146000036A36EE055A2DEEAB6A32EE02FA36EE1C
:10147000055A2AEE8F6A23EE066A36EE055A28EEE2
:101480008F6A26EE046A63EE03FA36EE055A2DEEF5
:10149000AF6A24EE048A35EE465A2DEE886A2DEEA8
:1014A0008E9A35EE465A29EE046A2AEEAE7A37EE67
:1014B000066A22EE000A2DEE8FAA36EE400A23EECF
:1014C0000A6A36EE000A2AEEAB6A30EE460A2AEEC7
:1014D000AF6A73EE039A36EE000A28EEA96A24EE8C
:1014E000066A36EE000A2AEE886A30EE460A25EED3
:1014F000055A20EE000A35EE000A21EE02BA21EE6E
:10150000035A21EE041A8DED051A22EE031A8DED11
:10151000031A23EE041A8DED041A34EE041A8DED2D
:10152000015A22EE04CA6EEE03CA8DED061A29EEA8
:1015300084DA06F04FFC94ED013A94ED022A9DED19
:10154000021A29EE024A21EE031A31EE444A94EDC2
:10155000031A28EEAE5A35EE044A2AEE015A35EE49
:10156000044A28EEAB5AF7EE001A34EE454A2AEE4A
:10157000A95A81EE800A25EE015A35EE044A28EE7A
:10158000AF5A34EE454A28EE885A75EE042A3CEEEE
:101590000C4A9DED075A34EE6C4A34EE454A3BEE58
:1015A0000B5A9DED086A35EE0D5A35EE465A2FEE70
:1015B000056A29EE847AF6EE007A76EE470A37EE6F
:1015C000EF6A36EE486A9DED018A20EE066A3CEE2F
:1015D000487A27EE227A36EE076A36EE6D7A22EEE8
:1015E000226A66EE073A70EEE33ADDED050ADDEDBC
:1015F000034A60EE015A74EEE00ADDED044A60EE43
:10160000200A7BEE244A64EEA24A70EEA40A63EE3E
:10161000224A70EEEA0A74EEE56A66EEA06A77EE98
:10162000EB7A76EEA33A78EE0C6A77EEEF7A60EE1C
:10163000266A67EEA27A76EEA76A76EEE86A60EE30
:10164000027ADDED068A27EEA68A38EE23CA68EE16
:10165000843A2EEE058A78EE233A3BEEAB8A71EEA1
:10166000C81A3FEEAF8A71EEC81A9DED098A21EEC5
:1016700022AA71EEC81AB1EE008A23EE089A21EE72
:10168000899A73EEC93A94ED009A2AEE07BA73EE7E
:101690008B3A29EE22BA77EE8B7A67EEA07A72EE59
:1016A000A22A77EEA33A63EE227A75EEE75A65EE48
:1016B000A65A35EEA3DA68EE853A6EEE045A73EE5A
:1016C000E53A62EE085A65EEA11A73EEE11AF8EEF9
:1016D000003A60EE233A62EE235A75EECB5A65EE7D
:1016E000875A20EE033A71EEA51A73EE0A5A20EEDD
:1016F000090A22EE222A65EEA05A30EE422A75EE41
:10170000A11A22EE262A23EE811A32EE218A2FEE2A
:10171000042A29EE854A31EE241A34EE022A21EEFB
:10172000071A36EE400A32EE011A20EE200A30EE99
:10173000010A23EE261A31EE009A2CEE0C0A2DEE49
:101740000D1A30EE010A28EE081A31EE000A29EED1
:10175000091A31EE000A06F03DFB95ED004A9DEDB9
:101760000A5A20EE0C1ADDED0B0A20EE0D2A24EEAB
:10177000011A9DED0C7A9DED0D6A20EE083A20EEDF
:10178000090A35EE415A24EE021A70EEC10A24EE1F
:10179000031A24EE000A37EE417A36EE406A94EDE1
:1017A000043A94ED000A94ED011A25EE035A94EDE3
:1017B000022A30EE050A20EE835A94ED034A35EEF4
:1017C000011A27EE035A35EE022A26EE033A84ED7B
:1017D000000A84ED011A20EE000A21EE011A33EE10
:1017E000043A30EE010A22EE021A30EE010A23EE2C
:1017F000031A30EE010A84ED022A84ED033A06F062
:10180000E9FA94ED001A94ED012A94ED023A94ED70
:10181000034A20EE011A20EE022A20EE033A20EEBF
:10182000040A002084ED001A84ED012A84ED023AB6
:1018300084ED030A43E50000B0B52DED108B04469E
:1018400000284FF0FF0018BF002900F06981002A2E
:1018500000F066814CF2000542F60230C2F201054A
:10186000C3F60750286092ED000A92ED011A94ED3C
:10187000014A94ED025A92ED022A94ED036A94ED26
:10188000003A24EE407A61EE050A37EE607A62EEA5
:10189000060A37EE607A60EE030A62EE051A71EE10
:1018A000A00A61EE061A70EEE10A61EE031A62EE1A
:1018B000042A22EE032A21EE041A91ED00CA71EEE9
:1018C000E21A20EE066A31EE021A20EE050A36EE22
:1018D000216A91ED01DA91ED02EA31EE400AB6EEAD
:1018E000001AB5EE40CA27EE01BA20EE81AA26EE14
:1018F000019AF1EE10FA20EE018A0AD1B5EE40DA33
:10190000F1EE10FA05D1B5EE40EAF1EE10FA00F072
:10191000BC802CEE0C0A2DEE0D1A30EE010A2EEED4
:101920000E1A30EE010A06F055FA94ED003A94EDE5
:10193000025AF1EE001A2CEE001A94ED014A75EEEF
:10194000050A63EE212A65EE053A62EEA34A61EECE
:10195000205A74EEA54A64EE045A2DEE002A94ED46
:10196000036A34EE047A62EEA52A72EEA42A62EECD
:10197000074A32EEE4CA76EE062A64EE214A66EEA3
:10198000066A64EEA67A21EE22DA77EECD7A23EEAD
:1019900003DA2DEE21DA2EEE000A24EE0DEA33EE04
:1019A000033A7EEE277A22EE03EA77EECE7AB2EEA3
:1019B00000EA24EE0E4A77EEE47A24EE25FA7FEE72
:1019C000277A24EE234A34EE274A60EE244A34EE86
:1019D00084FA2DEE054A21EE033A33EE043A25EE61
:1019E0000E4A25EE215A65EE264A33EE243A62EE7F
:1019F000222A33EE623A33EE453A65EE842A32EE1D
:101A0000833A24EE234A34EE033A20EE050A30EE00
:101A100003DA21EE070A25EEA11A21EE061A31EEAD
:101A2000400A23EEA11A26EE011A30EE010A22EE38
:101A3000201A30EE41EA2CEE0C0A2FEE0F1A30EE8F
:101A4000010A2DEE0D1A31EE000A2EEE0E1A31EEBD
:101A5000000A06F0BFF995ED004A20EE0C1A20EEC0
:101A60000F2A24EE011A20EE0D3A20EE0E0A3BEE6C
:101A700041BA24EE021A3AEE41AA24EE031A24EEE9
:101A8000000A39EE419A38EE408A94ED043A94ED1A
:101A9000000A94ED011A2BEE035A94ED022A30EE5F
:101AA000050A2AEE035A94ED034A35EE011A29EE8F
:101AB000035A35EE022A28EE033A84ED000A84ED3B
:101AC000011A20EE000A21EE011A33EE043A30EE3C
:101AD000010A22EE021A30EE010A23EE031A30EE5A
:101AE000010A84ED022A84ED033A06F073F994EDBD
:101AF000001A94ED012A94ED023A94ED034A20EE87
:101B0000011A20EE022A20EE033A20EE040A0020F9
:101B100084ED001A84ED012A84ED023A84ED030A73
:101B200040B2BDEC108BB0BDB1EE601AB4EE600AED
:101B3000F1EE10FAB4EE401AC8BFB0EE600AF1EE52
:101B400010FAC8BFB0EE410A7047000080B541F2FC
:101B50002C60C2F200000068082109F0D5FD80BDAC
:101B600080B54CF21812C2F2010200201221132398
:101B700000F086F9002080BD80B5022001214FF0E1
:101B8000FF3209F001FE80BD9FED010A704700BFE2
:101B90000000C84380B541F22C60C2F2000000682A
:101BA000102109F0B1FD80BD80B54CF21810C2F2D1
:101BB0000100C21D01200221062300F061F900206E
:101BC00080BD000080B5042001214FF0FF3209F0F4
:101BD000DBFD80BDF0B581B000284FF0FE0700F0BE
:101BE00097800C46002900F0938040F65426C2F2FC
:101BF00000060546307808B1FD2789E009F022FE8D
:101C000041F22C61C2F20001002808607BD0002064
:101C10007E21B622EC6200F08FF901201421B62259
:101C200000F08AF91E2000F083FE00201E2100F043
:101C30004DF90020002100F049F91E2865D101204E
:101C40000021012400F042F90F2860D1032000F0A8
:101C50004FFD042000F04CFD41F63162C0F6000259
:101C600000200121002700F039FE41F64D31C0F679
:101C70000001032000F086FD41F69531C0F6000119
:101C8000042000F07FFD00204021AA2200F054F93A
:101C900000204121012200F04FF9002053210822A9
:101CA00000F04AF900205821042200F045F90020F4
:101CB0007D21042200F040F9322000F039FE01209D
:101CC0000F21012200F038F901201021032200F039
:101CD00033F901201621002200F02EF901201821ED
:101CE000012200F029F901201521802200F024F9B9
:101CF0000A2000F01DFE0320347000F013FD0420C4
:101D000000F010FD04E0FE2702E0FC2700E0FC27C5
:101D100078B201B0F0BD0000002841D04CF218119B
:101D2000C2F20101B1F901209FED1F3A00EE102A25
:101D3000B8EEC00A80EE030AB1F90330B1F905C06C
:101D400001EE103A02EE10CAB8EEC11AB8EEC22A7D
:101D500081EE031A82EE032A4FF60003CFF6FF73DB
:101D600080ED040A4A7C897CD20042EA51120021AB
:101D7000B1EB922F80ED051A80ED062A18BF1A43A9
:101D800000EE102AB8EEC00AB4EE001A20EE010AE6
:101D9000B3EE071A30EE010A80ED0A0A48B2704726
:101DA000FE2148B2704700BF00A0AA45C0B34CF264
:101DB0001811C2F20101B1F90720B1F90930B1F9E6
:101DC0000B1000EE102A01EE103A9FED172A03EED9
:101DD000101AB8EEC00AB8EEC11AB8EEC33A80EED7
:101DE000020A81EE021A83EE022A9FED103AC16ABE
:101DF00091ED014A91ED025A20EE030A21EE031AF9
:101E000022EE032A91ED003A31EE441A30EE430AF5
:101E100032EE452A80ED070A80ED081A80ED092A86
:101E20006FF00100704700BF6F12034235FA8E3C1D
:101E300010B5012000F090FC41F22C64C2F20004C5
:101E400038B90120012100F0C3FC2068022109F00B
:101E50005BFC022000F080FC002818BF10BD0220AF
:101E6000012100F0B5FC2068042109F04DFC10BDF3
:101E700080B5182001214FF0FF3209F085FC80BDAC
:101E8000002A08BF704770B51C4615460E4618B1AB
:101E9000012805D1022000E00120002100F098FC7B
:101EA00040F2886146F08000C2F200010870002014
:101EB0000122002300F022FD0020294622460123B2
:101EC00000F0F2FCBDE8704070470000F0B581B052
:101ED000044601200D46012600F02AFD14B1012C14
:101EE00004D102263046002100F072FC40F28866E0
:101EF000C2F2000645F08000374607F8010B0020CB
:101F0000314601220023012500F0F8FC0020314673
:101F10000222002300F0C8FC34B1012C09D140F2A8
:101F20008867C2F2000702252846012100F050FC14
:101F30003878C0B201B0F0BDB0B5044601F07F0002
:101F400040F28861C2F20001087001204A70012548
:101F500000F0EEFC14B1012C04D10225284600212A
:101F600000F036FC40F28861C2F20001002002223B
:101F7000002300F0C3FC24B1012C18BFB0BD022027
:101F800000E00120012100F023FCB0BD2DE9F04369
:101F900081B04DF2B408C2F201080646D8F800003C
:101FA00014460D466421002A08BF0A2409F016FBD6
:101FB00008B1FB242FE040F67479C2F20009D9F889
:101FC000000000E0006930B10178B142FAD1416807
:101FD000A942F7D11AE0142000F012FC88B107469C
:101FE00020461C21002209F04FFAB86058B1D9F8F8
:101FF00000003C7300243E707D603861C9F80070B9
:1020000005E0FE2403E0384600F06EFBFF24D8F81C
:10201000000009F059FB60B201B0BDE8F083000098
:102020007047000040F67472C2F20002126800E0CD
:102030001269002A04BF0020704713788342F7D149
:1020400053688B42F4D1906870470000D0E90212C7
:10205000081FB0FA80F14FF0020008BF0320022AE7
:1020600018BF48097047000040F2F4724CF68451E2
:10207000C2F200020128C2F2010118BF00220028AA
:1020800018BF1146012888BF00210846704700008C
:102090002DE9F04115464DF24402C2F201021278D8
:1020A000012A11D1A5B14DF2B408C2F201080746C8
:1020B000D8F800000E4664211C4609F08FFA58B18A
:1020C000FB2040B2BDE8F081FD2040B2BDE8F081C8
:1020D000FE2040B2BDE8F08138463146FFF7A2FF4E
:1020E000D8F800100646084609F0EEFA66B1304608
:1020F00029460022234609F083F9002818BF4FF033
:10210000FF3040B2BDE8F081FC2040B2BDE8F08174
:102110002DE9F0478AB04DF24407C2F20107387842
:1021200008B1FD248AE04CF21800C2F201006821D7
:10213000FEF734FB002400BFE0B200F03BFA0134AC
:10214000012CF9D040F6502042F22101C2F20000E9
:10215000C0F6000101600020002409F069FA4DF288
:10216000B401C2F201010028086066D0E8464FF0D1
:1021700001094046282187F80090FEF70FFB4CF636
:102180008456C2F201064FF00E0A30464146CDE9B0
:102190000244CDE90799CDF824A0049402F0DCFDB7
:1021A000304603F09DF942F2BD22C0F60002002045
:1021B000062100F051F842F25155C0F6000500200A
:1021C00000212A4600F048F8002001212A4600F0AC
:1021D00043F8002002212A4600F03EF83046032151
:1021E00002F05CFD40F2F476C2F200063046414651
:1021F000CDE9049A02F0B0FD304603F071F942F2E5
:102200008132C0F600020120082100F025F80120EB
:1022100000212A4600F020F8012001212A4600F082
:102220001BF8012002212A4600F016F83046112141
:1022300002F034FD87F8009000E0FF2460B20AB09D
:10224000BDE8F08780B540F65022C2F20002126865
:10225000002A18BF904780BD4DF24403C2F201032B
:102260001B78012B1EBFFD2358B270473AB10128DD
:102270004FF0FF0398BF0C2904D958B27047FE23D2
:1022800058B270474CF2180CC2F2010C342310FB08
:1022900003C0002340F8212058B2704780B54DF2AA
:1022A0004403C2F201031B78012B03D1FFF76EFE3A
:1022B00040B280BDFD2040B280BD00002DE9F04F4E
:1022C00093B003A80D3001904FF0000A0CAE00202F
:1022D00005E000BF0298002800F101004CD15FFA30
:1022E00080FB02905846FFF7BFFE0028F2D004465C
:1022F00009E000BF03F064FC0990384603A90022FE
:10230000002309F011F92046002102F0A7FD002862
:10231000E0D02046002132460AAB02F0AFFD002893
:10232000F1D10E980028304618BF043005683046B9
:10233000FFF78CFE804628464146FFF783FF814623
:1023400058464946FFF76EFE0028DCD00746DDE917
:102350000F02CDF80CA00028CDE908AACDE906AA05
:102360008DF80C80CDE904598DF81820C2D1019860
:102370000AA9FEF794F9BDE713B0BDE8F08F00009D
:102380002DE9F04F93B003A80D3001904FF0000AF3
:102390000CAE002005E000BF0298002800F101000B
:1023A0004CD15FFA80FB02905846FFF75DFE002893
:1023B000F2D0044609E000BF03F002FC0990384661
:1023C00003A90022002309F0AFF82046012102F002
:1023D00045FD0028E0D02046012132460AAB02F03C
:1023E0004DFD0028F1D10E980028304618BF04306A
:1023F00005683046FFF72AFE804628464146FFF72B
:1024000021FF814658464946FFF70CFE0028DCD0E4
:102410000746DDE90F02CDF80CA00028CDE908AA97
:10242000CDE906AA8DF80C80CDE904598DF8182065
:10243000C2D101980AA9FEF732F9BDE713B0BDE891
:10244000F08F00002DE9F04389B017464DF24402A9
:10245000C2F201021278012A04D10446012806D9E9
:10246000FF2000E0FD2040B209B0BDE8F08301F09C
:10247000FE001D460E46022802D00DB9FE20F2E7EE
:10248000DDF84080B8F1080F01D9FF20EBE72046C6
:10249000FFF7EAFD98B181460020032E0890CDE9B0
:1024A0000600CDE90400CDE90200019009D8DFE87B
:1024B00006F0020A0D110197002100200DE0FE2018
:1024C000D1E7FF20CFE70297002005E00197022027
:1024D000002102E0022002970421CDE90310002030
:1024E000002DCDF814808DF8180018BFB8F1000F3A
:1024F00005D001A8183029464246FEF7D0F84846D4
:1025000002F04EFD38B101A901F118026B464846B0
:1025100002F0D8FB28B101A9204600F0A5F8013847
:10252000A1E700209FE7000079B180B582B00A687A
:1025300091F804C04B1D0021CDF800C0FFF782FFC9
:1025400002B0BDE8804040B27047FE2040B2704704
:102550002DE9F04389B001AC04F118090025E846E3
:1025600004E000BF002D05F1010520D1EFB238468F
:10257000FFF77AFD0028F5D0064600BF384600F088
:1025800027F80028EED1304602F00AFD0028E9D0F5
:102590003846214600F02EF80028E3D03046214688
:1025A0004A46434602F08EFB0028E7D0DAE709B03E
:1025B000BDE8F0834DF29C1100EBC010C2F20101A6
:1025C00001EBC0000021C0F80014C0F804147047EB
:1025D0004DF29C1100EBC010C2F2010101EBC000F2
:1025E000D0F80014D0F80404081AB0FA80F04009BA
:1025F00070470000002904BF002070472DE9F0411A
:102600004DF29C1C00EBC012C2F2010C0CEBC2029A
:10261000D2F800E4D2F804349E451FD002F20445FB
:102620002C6800EBC0100CEBC00000EB44126401FE
:1026300050F804C0D2E901805769D2E90364C1E9C6
:1026400000C8C1E90447C1E90206D2E90620C1E990
:1026500006202868013000F01F002860BEEB030050
:1026600018BF0120BDE8F08101284FF0000238D8E2
:10267000B9B32DE9F0474DF29C1C00EBC012C2F239
:10268000010C0CEBC202D2F80034D2F804E401339E
:1026900003F01F0373451ED002F58069D9F800408E
:1026A00000EBC0100CEBC00000EB44124FEA441AE0
:1026B000D1E904C6D1E90078D1E9025440F80A70A2
:1026C0005661C2E9034CC2E90185D1E90610C2E9AD
:1026D0000610C9F80030B3EB0E0218BF0122BDE8A6
:1026E000F04710467047000080B509F085FF80BDB7
:1026F00006284FF0FF0212D801460620DFE801F05D
:10270000090F0F04060F08000A2002E0172000E05E
:10271000092080B503F008FC0022BDE8804050B2DB
:102720007047000006284FF0FF0212D8014606202D
:10273000DFE801F0090F0F04060F08000A2002E08D
:10274000172000E0092080B503F0F2FB0022BDE86D
:10275000804050B2704700000A2884BF00207047B4
:1027600080B540F6DC11C0F6010101EBC0025268F1
:1027700031F83010104603F017FA0138B0FA80F043
:10278000400980BDB9B10A2882BFFF2040B270471E
:1027900040F6DC12C0F6010232F830C000200023FF
:1027A0002CFA00F2D20709D10E2B03F1010300F13C
:1027B0000100F5D908E0FE2040B270474CF28002DB
:1027C000C2F2010242F82010002040B2704700001F
:1027D0000A2882BFFF2040B2704780B50A4640F603
:1027E000DC11C0F6010101EBC0035B6831F8301069
:1027F000184603F0DFF90020BDE8804040B2704782
:1028000080B509F06BFD80BD012882BFFF2040B27A
:10281000704740F63421C0F60101B7EE001A51F8B6
:102820003000B4EE410AF1EE10FAC8BFB0EE410A32
:1028300000689FED0C1AC16AB5EE400A0131F1EE55
:1028400010FAB8BFB0EE410A01EE101AB8EE411A04
:1028500020EE010ABCEEC00A80ED0D0A002040B255
:10286000704700BF00000000012882BFFF2040B277
:10287000704780B540F63421C0F6010101EBC0027B
:1028800051F83000918804F065FE0020BDE88040DA
:1028900040B270474CF62071C2F20101002818BF07
:1028A000002108467047000070B510B1FF2040B20B
:1028B00070BD1E4614460D46FFF7ECFF0028F5D00C
:1028C0002946224616B103F0BBFF02E0142303F0B1
:1028D000FDFE002818BF012040B270BD002A0FBFC6
:1028E000FE204CF2C403C2F2010303EB40101CBFF4
:1028F00040F82120002040B27047000070B510B1B0
:10290000FF2040B270BD1E4614460D46FFF7C2FFC1
:102910000028F5D02946224616B104F07FFA02E0DD
:10292000142304F027F8002818BF012040B270BD1E
:1029300070B5044608F0FAFC0546FF2608F0D8FCFE
:10294000411C05290BD80120884010F0310F0BD114
:1029500010F0060F0AD0204603F020F811E06FF0C7
:102960000041884218BF002670B270BD4FF47A70E3
:10297000B0FBF5F1B4FBF1F0A14288BF012008F0F3
:102980008DFC002670B270BD2DE9F04108F0CEFC40
:1029900004460BF011F84FF47A784EF21806B8FBA3
:1029A000F4F4CEF20006376804FB00F50BF004F8EF
:1029B00060433168854208BF394656F8042C01FB54
:1029C00008F10132B1FBF2F100FB08F0401A00F50A
:1029D0007A700021BDE8F08103288FBF002040B24B
:1029E00001A151F82000704778CF0120C0090020D4
:1029F000C0CF0120080A002080B582B001680A68B3
:102A0000D20614D5002201920A6801924968019108
:102A1000019907F019FF40F2F85100EBC000C2F233
:102A2000000101EB8000006A002818BF804702B057
:102A300080BD00003AB103284FF0FF0398BF08297A
:102A400004D958B27047FE2358B2704740F2F85389
:102A500000EBC000C2F2000303EB8000002340F84B
:102A6000212058B27047000070B5032802D9FF201A
:102A700040B270BD144602460D4600294FF0FE00DC
:102A800018BF002C01D140B270BD10461E46FFF7A2
:102A9000A3FF294622461EB105F012F940B270BDCF
:102AA00005F054F940B270BDFEE7000080B54CF669
:102AB0008450C2F2010002F087FA80BD80B54CF666
:102AC0008450C2F2010002F07FFA80BD80B540F26E
:102AD000F470C2F2000002F077FA80BD80B540F2D7
:102AE000F470C2F2000002F06FFA80BD4FF00301F3
:102AF00060B146F200420068C4F2000202F5806351
:102B0000984208BF0121801A08BF0146C8B2704729
:102B100080B5024603284FF0FF000BD851B140F2B8
:102B20006870C2F2000050F8220028B102691AB1A0
:102B30008068904740B280BD007900220A54FC2092
:102B400040B280BDB0B540F20800C2F2000000F013
:102B500017F840F268750024C2F2000503E000BFD8
:102B60000134042C09D055F824000028F8D0C1689D
:102B70000029F5D080688847F2E70020B0BD00004A
:102B800010B10179032902D9FF2040B2704740F209
:102B90006872C2F2000242F82100002040B2704781
:102BA00050B380B590F88010022902D80144097C06
:102BB000B1B900210FF2480C1CF8012083181B7CCE
:102BC000002B08BF042203D1022901F10101F3D136
:102BD00080F8802080F8842080F8A82080F8C02029
:102BE00000F1100100F14802012300F0F5F8002087
:102BF000BDE8804040B27047FF2040B2704700BF40
:102C0000000102000146006891ED241A90ED030ACC
:102C100091ED252A20EE011A20EE020A002081ED16
:102C2000241A81ED250A704700207047014600688C
:102C300091ED251A90ED020A002031EE400A81ED57
:102C4000250A704790F88010012902D051B901215E
:102C500000E0002180F8801080F8841080F8A8102F
:102C600080F8C010002070470146006891ED241ADA
:102C700090ED040A91ED252A20EE011A20EE020AB9
:102C8000002081ED241A81ED250A704701460122BA
:102C9000002081F8C3207047014690F8C100013040
:102CA00000F00302002081F8C1207047014600684F
:102CB00091ED251A90ED020A002030EE010A81ED17
:102CC000250A70470146006891ED241A90ED020A2A
:102CD000002031EE400A81ED240A70470146006869
:102CE00091ED241A90ED020A002030EE010A81EDE8
:102CF000240A70470146052081F88C00022200203A
:102D000081F8AC20704700000020704710B586465F
:102D100000284FF0000018BF002A00D110BDD2F8E3
:102D200004C08CF000404FEACC0343EA5073062BFA
:102D300010D80020DFE803F0050E0E0E04222B0051
:102D4000ECE79EF82600002818BF0120E1B391F8B7
:102D5000261024E0DEF82C0000EA0C00A0EB0C00AA
:102D6000B0FA80F04FEA501081B3C96A01EA0C0151
:102D7000A1EB0C01B1FA81F1490913E09EF828009A
:102D8000002818BF012019B391F8281007E09EF819
:102D90002700002818BF0120E1B191F82710002971
:102DA00018BF0121127A002A08BF10BD022A05D0DF
:102DB000012A07D181F00101084010BD80F0010017
:102DC000084010BD002010BD0021EBE70021E9E71D
:102DD0000021E7E70021E5E72DE9F04780460028DC
:102DE0004FF0FF001ED00E46E1B140F6E03A1C461F
:102DF00091460025C0F6010A03E000BF1035B02D52
:102E00000FD00AEB0507787A2042F7D030464946C2
:102E10003A46FFF77BFF0028F0D0F9684046884724
:102E2000ECE7002040B2BDE8F08700002DE9F0415A
:102E30000022C1E90022C1E90222C1E904228A611B
:102E400050F8015F037C90F83C60013BDFB2FC006E
:102E500040F20133032F4FF00007D0F80480D0F880
:102E600008E0D0F80CC0C0F2020338BF23FA04F720
:102E70000F75447C013CE4B2E700032C4FF00004E2
:102E800038BF23FA07F44C75847C013CE4B2E700B8
:102E9000032C4FF0000438BF23FA07F48C75C47C70
:102EA0000E70013CE4B2E600032C4FF0000438BF82
:102EB00023FA06F4CC75047D4D60013CE4B2E500D4
:102EC000032C4FF0000438BF23FA05F40C76447D40
:102ED000C1F80880013CE4B2E500032C4FF0000487
:102EE00038BF23FA05F44C76847DC1F80CE0671EE8
:102EF000FFB2FE00032F4FF0000738BF23FA06F79A
:102F00008F76C07DC1F810C00138C0B2C700032859
:102F10004FF0000038BF23FA07F2CA76BDE8F0810F
:102F200080B506F0E7F980BD90F83D0070470000DD
:102F300070B52DED028B20B30446FFF725FD054645
:102F40000E460DF00AFC9FED1F8A00EE100A80EE7F
:102F5000080AE068281A66F1000184ED010A0DF004
:102F6000FCFB00EE100A80EE080A94F88000E56091
:102F7000042884ED020A06D3204600F02DF9FC2037
:102F80001BE0FF2019E094F8A80040F26C45C2F263
:102F9000000505EB001081682046884794F88400FE
:102FA00005EB001041682046884794F8C00005EB07
:102FB0000010C16820468847002040B2BDEC028B5B
:102FC00070BD00BF00247449B0B5054600284FF01D
:102FD000FF000BD00C4649B12846C421FDF7DEFBAB
:102FE0002C60FFF7AFFDFFF78FFE002040B2B0BDB1
:102FF00080B5417C69B1042280F88C20002200F168
:103000001001C0E9242200F148020223FFF7E4FE88
:1030100080BD032180F88C1080BD000080B5417C0C
:1030200061B3012280F8AC20B0F93020036852422D
:1030300000EE102AB0F9322090ED021A03EE102AA9
:10304000B8EEC00A93ED012AB8EEC33A21EE000AA9
:1030500021EE031A22EE000A22EE011AB7EE082A28
:1030600000F1100121EE021A00F14802042380ED64
:103070002C0A80ED2D1AFFF7AFFE80BD002180F8ED
:10308000AC1080BD80B5417C71B190F83630012222
:1030900000F1100180F8C22080F8C33000F148022E
:1030A0000823FFF799FE80BD002180F8C11080BD84
:1030B00090F824200168032A0AD0022A0FD0012A9E
:1030C00017D1097D80F88C10002180F88D1013E055
:1030D000897D80F88C10012180F88D100CE04A7DEC
:1030E00080F88C20022280F88D200969C0F89C109D
:1030F00002E0032180F88C10D0E90512C0E9241207
:103100007047000090F825200168032A05D0022AA4
:1031100005D0012A06D1173102E0193100E018313B
:10312000097800E0002190ED070A90ED081AB8EE4A
:10313000002A20EE020ABFEE082A21EE021A80F8C9
:10314000AC1080ED2C0A80ED2D1A704790F82610F7
:10315000027C012980F8C12005D002290AD0032968
:1031600004D1022107E0002180F8C2100021A0F85C
:10317000C21002E0012180F8C11090F82710012947
:1031800006D003290AD0022905D10022012107E037
:103190000021A0F8C2100021002201E0012101223B
:1031A00090F8283080F8C210032B80F8C3200AD092
:1031B000022B0CD0012B19BF002180F88C100121AB
:1031C00080F88D107047022180F88D107047002123
:1031D00080F88D1070470000032180F88C100021CA
:1031E00080F8AC1080F8C1107047000010B504469C
:1031F00000F00AF8002818BF10BD2046FFF7D0FCE9
:103200002046FFF795FE10BD78B32DE9F04F83B04F
:10321000044654F8100F0190606B04F11C0B0290EF
:1032200001989BE8C00F04F1040EA06304F1540060
:103230009EE82E5080E8C00F0298A5640025E16347
:1032400022646364C4F84CC0C4F850E0E06600BF78
:10325000E8B22146FFF75CFC0135042DF8D10020CF
:1032600003B0BDE8F04F40B27047FF2040B2704756
:1032700080B500EE100AB8EE400A10EE100A0DF00C
:1032800017FA9FED110B53EC102B0CF0A5FE0CF070
:103290006FFB00EE100A0BF0DBFF9FED0D1A9FEDA8
:1032A0000E2A20EE010A9FED0B1AB0EEC00A30EE96
:1032B000010AB4EE420AF1EE10FAC8BFB0EE420ABB
:1032C00080BD00BF00BF00BFFCA9F1D24D62503FDE
:1032D000CDCC4C3E9A99193FCDCC4C3F2DE9F047CF
:1032E0002DED048B804600284FF0FE0000F0068193
:1032F0000E46002900F00281D8F800009FED821AE6
:10330000101A00EE100AB8EE400A80EE010A317978
:1033100040461546C8F8002088ED010A00F0FEF886
:1033200008B1FD20EAE0404606F008FA98F81800D7
:1033300005280AD8DFE800F0030B03035822002019
:10334000C8E90700C8F8240068E0FD20D6E096ED43
:10335000020A96ED031A96ED052A96ED043A20EE40
:10336000020A22EE011A22EE033A88ED070A88EDDE
:10337000081A88ED093A88ED0A2A4FE098ED5B0AB1
:103380009FED641A08F5FC6480EE010A9FED621A55
:1033900094ED012A20EE010A30EE428AB0EE480A8E
:1033A0000BF02CFEB0EE409AB0EE480A0BF050FF46
:1033B00096ED061A96ED072A29EE013A20EE024A0A
:1033C00020EE010A29EE021A33EE443A30EE010AE9
:1033D00094ED008A284688ED073A88ED080AFFF741
:1033E00047FF28EE000A17E096ED070A96ED061A49
:1033F000B1EE400AB1EE411A88ED070A88ED081ACD
:10340000D8ED011AD8ED5B0A9FED400A9FED401AF6
:1034100008F2AC5005F022FE88ED090A98ED070A83
:1034200008F5C16004F00AFD88ED070A98ED080A66
:1034300008F5C56004F002FD88ED080A98ED090A58
:1034400008F5C96004F0FAFC404688ED090A00F06E
:10345000EBF89FED2F8A6FF07F094FF0000A40F2E2
:10346000BC47002408EB040595ED1E0AD5ED6B0A58
:1034700008EB0A06D8ED011A06F53770B0EE481AC7
:1034800085ED220A05F0EAFDD5ED6F0AD8ED011AA7
:1034900006F57370B0EE481A85ED020A05F0DEFD00
:1034A00008EB090606F5ED6085ED2B0A04F0C6FC75
:1034B00005F5FA6080ED000A95ED160AD5ED770A5C
:1034C000D8ED011A08EB0700B0EE481A85ED260A80
:1034D00005F0C4FD06F5DD6085ED2F0A04F0AEFCB5
:1034E000043405F5F86009F120090AF13C0A102CB2
:1034F00007F13C0780ED000AB4D1002040B2BDECDA
:10350000048BBDE8F08700BF00007A440AD703406F
:103510000000000000003443DB0F49402DE9F0417A
:10352000B0B30446007E884688422DD0B8F1050F1E
:1035300008D1052806D01046FDF774F84FF07E50EC
:10354000C4F8E00704F2BC46042500BFA6F1F0076A
:10355000384605F083FEA6F5F07005F07FFE304694
:1035600005F07CFE384605F079FE013D06F13C068B
:10357000ECD104F5197004F5F67605F06FFE3046CF
:1035800005F06CFE84F81880002040B2BDE8F081A0
:10359000FE2040B2BDE8F081F0B581B0044600F2F3
:1035A000BC764FF4947500BFD4F8040696ED010A7A
:1035B00028442038371D05F083F8D4F8040696ED2A
:1035C000050A284405F07CF80835B5F5A47F3E4689
:1035D000EAD1D4F8040600F5847004F045FFD4F86D
:1035E000040600F5947004F03FFFD4F8040600F5DB
:1035F000A07004F039FF04F2B4714FF4A87500BF55
:10360000D4F8040691ED010A28440E1D05F058F87F
:10361000D4F80406284404F027FF0835B5F5B07F38
:103620003146EDD101B0F0BD2DE9F04F81B02DED67
:10363000028B8AB0077E0446012F35D1E06920F065
:1036400000400DF035F89FED220B55EC106B324623
:103650002B460DF06DF838BB206A20F000400DF0CD
:1036600027F832462B460DF063F8E8B9606A20F07F
:1036700000400DF01DF832462B460DF059F898B970
:1036800094F8E80504F5F563002804BF012084F8E8
:10369000E8050020C4E91200C4E914000FCB04F1CE
:1036A000680C8CE80F0014E20020052F84F8E80570
:1036B00000F20F820120B84010F00D0F14D000204E
:1036C000C4E91200C4E91400C4E91A002067FFE14C
:1036D0009A9999999999B93FCC3B7F669EA0E63F0C
:1036E000CD3B7F669EA0E63FD4E9070A656A0CF0F1
:1036F000DFFF8046284689460CF0DAFF1FED0A0BF3
:1037000006465BEC102B5B460F460292CDF814B0D8
:103710000CF062FC42464B460CF05CF902460B464C
:103720000CF05AFC8146504688460CF0C1FF1FED54
:10373000140B05468A4653EC102B30463946CDE92A
:1037400003230CF049FC2A4653460CF043F9024689
:103750000B460CF041FC02460B46484641460CF035
:1037600039F941EC100B0BF03BFE51EC100B0CF057
:10377000FFF8A064D4E90708656A0CF099FF0746D2
:1037800028468A460CF094FF029A5B460646894614
:103790000CF022FC3A4653460CF01CF902460B464C
:1037A0000CF01AFC824640468B460CF081FFDDE9A6
:1037B000032305460F46304649460CF00DFC0246F1
:1037C0000B46284639460CF085FE02460B460CF0A7
:1037D00003FC02460B46504659460CF0FBF841EC00
:1037E000100B0BF0FDFD51EC100B0CF0C1F8E06478
:1037F000D4E90701656A01910CF05AFF0746284693
:1038000089460CF055FFDDF80880059B42460646C8
:103810008B460CF0E1FB02460B46384649460CF05D
:1038200059FE02460B460CF0D7FB814601988A46AA
:103830000CF03EFFDDE9032307460D4630465946AE
:103840000CF0CAFB02460B46384629460CF042FEF5
:1038500002460B460CF0C0FB02460B46484651465A
:103860000CF0B8F841EC100B0BF0BAFD51EC100B5A
:103870000CF07EF82065D4E9070A656A0CF018FFA1
:103880000746284689460CF013FF059B424606462C
:103890008B460CF0A1FB02460B46384649460CF01D
:1038A00019FE02460B460CF097FB814650468846AF
:1038B0000CF0FEFE0D465946DDF80CA0DDF810B008
:1038C0000746304652465B460CF086FB3A462B468E
:1038D0000CF080F802460B460CF07EFB02460B46CD
:1038E000484641460CF076F841EC100B0BF078FDA1
:1038F00051EC100B0CF03CF86065D4E90780666A67
:103900000CF0D6FE0546304689460CF0D1FE5246F4
:103910005B4606460F460CF05FFB2A464B460CF012
:1039200059F841EC180B40460CF0C2FE029A059B78
:1039300005468846304639460CF04EFB2A4643463B
:103940000CF048F841EC110BB0EE480AF0EE680AB2
:103950000BF0FEF851EC100B9FED9F0B53EC102B6E
:10396000CDE900230CF038FB0CF002F8A066D4E996
:1039700007A0666A0CF09CFE054630468B460CF0AC
:1039800097FEDDF80C90049B4A4606460F460CF065
:1039900023FB02460B46284659460CF09BFD41ECA2
:1039A000180B50460CF084FEDDF80880059B054698
:1039B0008A463046394642460CF00EFB2A465346AC
:1039C0000CF008F841EC110BB0EE480AF0EE680A72
:1039D0000BF0BEF8DDE9002351EC100B0CF0FCFA03
:1039E0000BF0C6FFE066D4E907A0666A0CF060FE43
:1039F000054630468B460CF05BFE4A46DDF81090DB
:103A000006464B460F460CF0E7FA02460B462846A0
:103A100059460CF05FFD41EC180B50460CF048FE87
:103A20004246DDF8148005468A463046394643460C
:103A30000CF0D2FA02460B46284651460CF04AFDDD
:103A400041EC110BB0EE480AF0EE680A0BF080F87A
:103A5000DDE9002351EC100B0CF0BEFA0BF088FFEF
:103A60002067D4E907A0666A0CF022FE05463046BE
:103A70008B460CF01DFE039A4B4606460F460CF093
:103A8000ABFA2A465B460BF0A5FF41EC180B5046FB
:103A90000CF00EFE029A05468A46304639464346E9
:103AA0000CF09AFA02460B46284651460CF012FDDD
:103AB00041EC110BB0EE480AF0EE680A0BF048F842
:103AC000DDE9002351EC100B0CF086FA0BF050FFEF
:103AD00060679FED430A04F168000021421892EDEF
:103AE000001A0431B5EE401AF1EE10FABCBF31EE07
:103AF000001A82ED001A1029F0D19FED3A1A9FEDBD
:103B00003A2A9FED3A3A9FED3A4A9FED3A5A002001
:103B100006A90AE0F1EE600A36EE076AC2ED160A5F
:103B20000130042882ED1E6A4DD004EB800292ED34
:103B30001A7A92ED6B6A01EB800337EE467AB4EEA7
:103B4000417AF1EE10FA83ED007A08DD37EE027A61
:103B5000B4EE417AF1EE10FAF8DC83ED007A93EDE1
:103B6000007AB4EE437AF1EE10FA08DA37EE007A12
:103B7000B4EE437AF1EE10FAF8DB83ED007AB4EE9E
:103B8000447AF1EE10FA0BDDB4EE417AF1EE10FA60
:103B900006DC936C36EE076A936536EE036ABFE780
:103BA000D2ED120AB4EE457AF1EE10FAB2DAB4EEC2
:103BB000437AF1EE10FAADDB36EE076AC2ED160A73
:103BC00036EE016AACE70AB0BDEC028B01B0BDE88D
:103BD000F08F00BF00BF00BF00000000DCA54C401C
:103BE0000000B443000034430000B4C3000034C3F9
:103BF0000000B4420000B4C22DE9F0472DED0C8B5B
:103C000082B0002800F0DD809FED739A9FED73AACB
:103C10009FED73BA9FED73CA9FED6D8B9FED72DAC6
:103C2000824600256FF00F066FF00F07DAF80406E2
:103C3000284400F5847004F093FDDAF80406284463
:103C400000F5847004F0AEFC00F108030AEB4504B3
:103C50000ECB406904F1EC0C8CE80E00C4F8F800BF
:103C6000DAF80406284400F5947004F079FDDAF8D7
:103C70000406284400F5947004F094FC00F1080355
:103C80000ECB406904F5967C8CE80E00C4F8380130
:103C900094ED4B0A0AEB070480EE090A0AEB0600D2
:103CA00020EE0A0A84ED6F0A90ED501A81EE0B1A8D
:103CB00084ED731A90ED401A04F2FC5081EE0C1A58
:103CC00090ED002A30EE420A10EE100A84ED7B1AC5
:103CD0000CF0EEFC41EC100BB0EE481AF0EE681A56
:103CE0000BF034FA51EC100B0BF042FE00EE100A10
:103CF000B5EE400AF1EE10FA05F1080530EE0D1AA6
:103D0000B8BFB0EE410A0437202D06F1100684ED4D
:103D10006F0A8BD19FED358A9FED359A0AF2FC58D8
:103D200000264FF4A877D025E94605E00436083789
:103D3000042E05F1100532D159F806000028F5D0FF
:103D4000DAF80406384404F00BFDDAF804063844C7
:103D500004F028FC00F1080C0AEB86019CE81C101A
:103D600001F1CC0E8EE81C100AEB050292ED000A60
:103D70000AEB060420EE080A80EE090AB0EE481AA3
:103D800049F8060084ED690A91ED330A08EB060153
:103D9000D1ED000A00F0F0FA84ED630AC6E79AED6F
:103DA000630A0020002407F01DFA9AED641A8AEDD8
:103DB000650AB0EE410A012007F014FA8AED660A9E
:103DC00000E0FE2460B202B0BDEC0C8BBDE8F087D1
:103DD0000000000000807640DB0F494000003443C3
:103DE0000000A04300401C460000B443DB0FC94064
:103DF0000000704290ED001AF5EE400AF1EE10FA64
:103E000031EE000A10DDB4EE600AF1EE10FAA2BF46
:103E100030EE600A80ED000A7047B5EE400AF1EE20
:103E200010FAB8BF30EE200A80ED000A704700009B
:103E3000B5EE401AF1EE10FA30EE600AD8BF7047C6
:103E4000B6EE002A21EE022AB4EE420AF1EE10FA92
:103E5000C4BF30EE410A7047B1EE422AB4EE420AC6
:103E6000F1EE10FAB8BF30EE010A704790ED001A7B
:103E7000B4EE601AF1EE10FAC8BFC0ED000A90ED82
:103E8000001AB4EE401AF1EE10FAB8BF80ED000A45
:103E90007047000040F22000C2F2000070470000AE
:103EA00080B54CF60C60C2F2010001F017FC80BD39
:103EB00080B540F67C00C2F2000001F00FFC80BD2E
:103EC00080B54CF6AC50C2F2010001F007FC80BD99
:103ED00080B540F61C00C2F2000001F0FFFB80BD7F
:103EE00080B54CF66C60C2F2010001F0F7FB80BDBA
:103EF000D0F800C06FF00F024AF6AB2352FA8CF2F2
:103F0000CAF6AA230146A2FB0330000905A31B5CE5
:103F100040F2FF302CEA00005F2A88BF0430C1E97C
:103F20001603704700061016000610168269816A93
:103F3000B2F5005F06D06AB9022912D0012914D067
:103F4000D1B90EE0032917D8DFE801F0020B020F08
:103F50000120704703293CBF012070471CBF00208F
:103F60007047C06AC0F300607047C06AA0F1C070BB
:103F7000B0FA80F0400970470020704780B5D0F853
:103F800000C0D0F808E0DCF80000BEF1400F20F4DB
:103F90008020CCF800000846CCF8043004BF10465E
:103FA0000A46CCF80800CCF80C2080BD10B5E8B16A
:103FB0004DF24504C2F20104207810B1FD2040B258
:103FC00010BD07F03FFC41F23061C2F20001086011
:103FD00060B143F6F572C0F6000202200321FEF73D
:103FE00029FD01202070002040B210BDFE2040B20B
:103FF00010BD000080B541F23060C2F200000068E0
:10400000012107F081FB80BD70470000002843D0EC
:10401000B0B50446451C02202070204600F05CF834
:10402000E869296A6A6AAB6A2860B4F92D00AA6057
:10403000EB60696003F0F0FEB4F92F10607408467D
:1040400003F0EAFEB4F93110A074084603F0E4FE70
:10405000B4F93310E074084603F0DEFEB4F935100D
:104060002075084603F0D8FEB4F93710607508468D
:1040700003F0D2FEB4F93910A075084603F0CCFE67
:10408000B4F93B10E075084603F0C6FE2076002028
:10409000BDE8B04040B27047FE2040B2704700001B
:1040A000B0B103210170002180F83D10C0F801106B
:1040B000C0F80510C0F80910C0F80D10C0F81110B4
:1040C000C0F81510C0F81910C0F81D1048B270479C
:1040D000FE2148B2704700002DE9F0472DED088B16
:1040E000002800F01A814CF23411C2F201014B7821
:1040F0008F78012267F30A2300EE103AB8EEC00A67
:1041000000F11D0480F83D2010EE102A2260CA78CC
:10411000FB0862F34A1300EE103AB8EEC00A10EE44
:10412000103AE3600B794F799B0043EA921207F053
:10413000010342EA832200EE102AB8EEC00A10EE14
:10414000102A62608A797B0862F3CA1301EE103A82
:10415000B8EEC11A11EE103AA3600F7ACB794E7AFD
:1041600012097F0063F30A1247EAD31306F003072C
:104170008D7A43EA4723A0F82D30B308CF7A65F350
:104180008A13A0F83730FB000F7B4E7B43EA5513B0
:10419000A0F8353066F30A278B7BA0F83370F70858
:1041A000CE7B63F34A17A0F83170B7000E7C47EA64
:1041B000931306F0010743EA8723497C9FED5E8A4B
:1041C0009FED5E9AA0F82F307308BFEE00AAB7EEFD
:1041D00000BA61F3CA13F0EE480AB0EE491AF0EEE5
:1041E0004A1AB0EE4B2AA0F83920A0F83B30A0F8CC
:1041F000392006F0E9FF216810EE100A00EE101ACF
:10420000F0EE480AB0EE491AF0EE4A1AB0EE4B2A28
:10421000606006F0D9FFA16810EE100A00EE101AD7
:10422000F0EE480AB0EE491AF0EE4A1AB0EE4B2A08
:10423000206006F0C9FFE16810EE100A00EE101AC7
:10424000F0EE480AB0EE491AF0EE4A1AB0EE4B2AE8
:10425000A06006F0B9FF206810EE108AC4F80C8048
:104260000CF026FA9FED300B074659EC10AB524686
:104270004B460E460CF063FA58B99FED2D0B3846AD
:1042800053EC102B31460CF04CFA002804BF0020F0
:10429000206060680CF00CFA52464B4606460F460A
:1042A0000CF04DFA58B99FED220B304653EC102B11
:1042B00039460CF036FA002804BF00206060A06880
:1042C0000CF0F6F952464B4606460F460CF037FA0C
:1042D00058B99FED170B304653EC102B39460CF0B4
:1042E00020FA002804BF0020A06040460CF0E0F94E
:1042F00052464B4606460F4600250CF020FA68B998
:104300009FED0B0B304653EC102B39460CF009FA9D
:10431000002804BF0025E56000E0FE2568B2BDEC82
:10432000088BBDE8F08700BF7B14AE47E17A84BFFD
:104330007B14AE47E17A843F0080B04300E0D34471
:1043400080B5012001F054FB80BD000080B508203D
:1043500001F04EFB80BD000080B5102001F048FB4D
:1043600080BD000080B5202001F042FB80BD000030
:1043700072B600BFFEE7000030EE600AB5EE400AFC
:10438000F1EE10FABCBF30EE010A7047B4EE410AFC
:10439000F1EE10FAA8BF30EE410A704770B52DED6E
:1043A0000E8B044600284FF0FF0000F0B6810D464A
:1043B000002900F0B281FEF7E7FAD4E90023801A61
:1043C00099410CF0CAF99FEDD70A01EE100A81EE6F
:1043D000000A84ED020AFEF7D7FA2A78C4E9000140
:1043E0002046114600F05EFB204606F0DDFE94ED0F
:1043F00002DA95ED010A95ED02EA04F5367004F54E
:10440000287120EE0DAA06F027FF94ED141AB0EEE5
:10441000408A9FEDC59A94ED740A38EE011A7AEE3F
:10442000010AB0EE491AFFF703FD94ED141AB0EE3D
:1044300040BA94ED750A38EE011A7AEE010AB0EE30
:10444000491AFFF7F5FC607C02280BD0012800F028
:10445000AC80002840F048810020C4E99300C4F8F3
:10446000540241E19FEDB09A04F5F2752846B0EE92
:104470004A0AF0EE490AFFF7BDFC94ED790A9FED78
:10448000AB1AB4EE410AF1EE10FA05DD9FEDA82A51
:1044900030EE020A85ED000A95ED003A9FEDA52A5F
:1044A000B1EE484AB4EE423AF1EE10FABCBF33EE38
:1044B000093A85ED003A9FED9E3AB4EE428A33EE1A
:1044C000485AF1EE10FAB8BFB0EE454AB4EE424A8F
:1044D00094ED796A34EE095AF1EE10FAB8BFB0EEF5
:1044E000454A34EE064AB4EE414A34EE033AF1EE60
:1044F00010FAC8BFB0EE434AB4EE424A34EE091A8D
:10450000F1EE10FAB8BFB0EE414AE06894ED151A2A
:1045100041782DEE0E0A30EE010A84ED144A84ED46
:10452000150A39B1D0ED460A90ED470A04F154005E
:10453000FFF79CFCD4ED021A94ED130AD4EDB20AF5
:1045400094EDB31A04F1680004F088FD9FED7AAA97
:1045500084ED930AD4ED021AD4ED0D0A94ED140AF9
:1045600004F1E000B0EE4A1A04F078FDD4ED021A2E
:10457000D4ED0A0A04F58E70B0EE4A1AB0EE408A05
:1045800004F06CFD84ED940AD4ED021AD4ED0C0A0B
:1045900094ED150A04F5AC70B0EE4A1A04F05EFD15
:1045A000D4ED021AD4ED090A73E020462946B0EE94
:1045B00040CA04F1500600F0C1F8E068007838B154
:1045C0003046B0EE4C0AF0EE4B0AFFF74FFC1BE012
:1045D00096ED000A9FED551AB4EE410AF1EE10FA7D
:1045E00005DD9FED531A30EE010A86ED000A96EDC7
:1045F000000A9FED501AB4EE410AF1EE10FABCBF6A
:1046000030EE090A86ED000AE068417839B1D0ED54
:10461000460A90ED470A04F15400FFF727FCD4ED59
:10462000021A94ED130AD4EDB60A94EDB71A04F108
:10463000680004F013FD9FED40AA84ED930AD4EDC9
:10464000021AD4ED0D0A94ED140A04F1E000B0EE64
:104650004A1A04F003FDD4ED021AD4ED0A0A04F557
:104660008E70B0EE4A1AB0EE408A04F0F7FC84ED8A
:10467000940AD4ED021AD4ED0C0A94ED150A04F54F
:10468000AC70B0EE4A1A04F0E9FCD4ED021AD4ED95
:10469000A60AB0EE409A04F5CA70B0EE4A1A04F0C9
:1046A000DDFCE06884ED950A90F8041169B194EDA1
:1046B000A72A90ED421A94ED943A38EE422A21EE60
:1046C000021A33EE011A84ED941A90F8051159B1CB
:1046D00094EDA51A90ED432A39EE411A22EE011A03
:1046E00030EE010A84ED950A94ED930A04F5F67014
:1046F00003F0A4FB84ED930A94ED940A04F503708F
:1047000003F09CFB84ED940A94ED950A04F50B707C
:1047100003F094FB002084ED950A40B2BDEC0E8BB3
:1047200070BD00BF00247449DB0FC940DB0F494056
:10473000DB0FC9C0DB0F49C00000000000284FF0AC
:10474000FF0218BF002901D150B270474A78022AEF
:1047500019D0AAB991ED010A91ED021A90ED022A41
:1047600090ED143A90ED154A20EE020A22EE011A5D
:1047700033EE000A34EE011A80ED140A80ED151AAA
:10478000002250B27047CA6802650969002241657B
:1047900050B27047002808BF7047C16891F8FB20ED
:1047A000022A05D0012A08D05AB990EDA90A06E0DC
:1047B00090EDAA0AB1EE400A01E090EDA80A80ED62
:1047C0000C0A91F8FC20022A05D0012A06D04AB929
:1047D00000F5297204E000F52A7201E000F5287264
:1047E0001268426391F8F820022A05D0012A06D007
:1047F0004AB900F5257204E000F5277201E000F5E2
:1048000026721268426291F8F910022905D0012936
:1048100006D049B900F5257104E000F5277101E0E3
:1048200000F526710968816200F52B7C9CE80E106A
:104830003C3080E80E10704710B52DED028B00283B
:1048400000F09E800446C1600020607404F168009E
:1048500001F158020121B0EE408A04F0B7FCE16892
:1048600004F1A40001F138020121B0EE480A04F07D
:10487000ADFCE16804F1E00001F198020121B0EE25
:10488000480A04F0A3FCE16804F58E7001F1780297
:104890000121B0EE480A04F099FCE16804F5AC701F
:1048A00001F1D8020121B0EE480A04F08FFCE16862
:1048B00004F5CA7001F1B8020121B0EE480A04F013
:1048C00085FCE06890ED4B0A90ED4C1AD0ED440A5F
:1048D00030EE011A84ED750A04F5F670B0EE480A60
:1048E00084ED741A03F0E8FAE068B0EE480AD0EDFF
:1048F000440A04F5037003F0DFFAE068B0EE480AFA
:10490000D0ED440A04F50B7003F0D6FAFDF700FC75
:10491000E0688178022902D10E3003F07DFEE06864
:104920008178012906D1063003F052FCE068063098
:1049300003F060FBE0680179022902D12E3003F018
:104940006BFEE068C178022902D1263003F064FED4
:10495000E0680179012906D11E3003F039FCE068D6
:104960001E3003F047FBE068C17801290AD11630F8
:1049700003F02EFCE068163003F03CFB002002E060
:10498000FF2000E0002040B2BDEC028B10BD000013
:1049900010B50446C0688178022908D10E3003F0B2
:1049A00063FDE06894ED930A0E3003F089FEE06841
:1049B000817801291CD1D0F8401194ED930AC4F8F4
:1049C0006012D0F84811C4F86812D0F84411C4F845
:1049D0006412D0F83C11C4F85C1290ED5D1A04F535
:1049E000167120EE010A063084ED960A03F05CFB96
:1049F000E0680179022908D12E3003F035FDE06826
:104A000094ED940A2E3003F05BFEE068C178022931
:104A100008D1263003F028FDE06894ED950A263091
:104A200003F04EFEE068C17801291CD1D0F868116E
:104A300094ED950AC4F88812D0F87011C4F8901259
:104A4000D0F86C11C4F88C12D0F86411C4F8841238
:104A500090ED5F1A04F5207120EE010A163084ED06
:104A6000A00A03F021FBE0680179012918BF10BDFD
:104A7000D0F8541194ED940AC4F87412D0F85C1173
:104A8000C4F87C12D0F85811C4F87812D0F850113C
:104A9000C4F8701290ED5E1A20EE010A84ED9B0AB4
:104AA00010BD0000B0B52DED028BC8B30446407CAC
:104AB0000D46884234D004F1680004F0CFFB04F1C5
:104AC000A40004F0CBFB04F1E00004F0C7FB04F504
:104AD0008E7004F0C3FB04F5AC7004F0BFFB04F56A
:104AE000CA7004F0BBFB9FED108A04F5F670B0EEBF
:104AF000480A03F033FA04F50370B0EE480A03F0F5
:104B00002DFA04F50B70B0EE480A03F027FA04F111
:104B10005000FCF7C3FBD4E9A8016574C4E9140193
:104B2000BDEC028BB0BD00BF0000000010B5002836
:104B300000F088800446C0688178022911D10E30C7
:104B400003F00EFEE0680E3003F02CFD48B100F1DA
:104B500008030ECB406904F5327C8CE80E00C4F8E3
:104B6000D402E0688178012911D1063003F00EFCEF
:104B7000E068063003F06CFA48B100F11C030ECB7C
:104B8000806A04F5327C8CE80E00C4F8D402E06838
:104B90000179022911D12E3003F0E2FDE0682E30B8
:104BA00003F000FD48B100F108030ECB406904F5A5
:104BB000367C8CE80E00C4F8E402E068C178022973
:104BC00011D1263003F0CCFDE068263003F0EAFC7A
:104BD00048B100F108030ECB406904F53A7C8CE83B
:104BE0000E00C4F8F402E0680179012911D11E30E9
:104BF00003F0CCFBE0681E3003F02AFA48B100F164
:104C00001C030ECB806A04F5367C8CE80E00C4F8D9
:104C1000E402E068C178012911D1163003F0B6FB37
:104C2000E068163003F014FA48B100F11C030ECB13
:104C3000806A04F53A7C8CE80E00C4F8F402002087
:104C400040B210BDFF2040B210BD000010B380B5CF
:104C50008B68D1E900C2C0F89C32C0E9A5C24B699B
:104C6000D1E903C2C0F8A832C0E9A8C201F1280CFA
:104C70009CE80C1000F52F7E8EE80C10D1E906C3DD
:104C8000D1E90821C0E9ABC3C0E9AD21FFF782FD3E
:104C9000BDE880404FF0FF307047000090F82020C2
:104CA000013A012A04D8006800F11402002004E04F
:104CB00000F1240201204FF4802113681943116090
:104CC0007047000010B590F820E0D0F800C0AEF1B9
:104CD000010EBEF1010FDCF808E00ED81EF0E05F17
:104CE00011D0CEF3016E012000FA0EF018608B682F
:104CF0007BB1486843EAC0030DE000F124010120C4
:104D00004FF4802223E000F1240101204FF400122F
:104D10001DE008684305D1E9030403430CEB0E10C2
:104D2000C0F88031C0F88441097D012905D100F522
:104D3000C2710B6843F480730B605168C0F88C112A
:104D4000126800F5C071C0F88821002001220B68AC
:104D50001A430A6010BD0000B0B590F82020013A57
:104D6000012A2FD846F20060C4F20000026842F027
:104D700001020260026822F47C520260D1F814E061
:104D8000CC694A6A0368012C43EA022202600EF0F1
:104D90001F024FF0010303FA02F2C3696FEA020C2B
:104DA00023EA0203C36113D02CBBC36803EA0C03DC
:104DB000C360CB688C8844EA034300EBCE042364D1
:104DC0000B4611E0416A41F4802141620120B0BDEF
:104DD000C3681343C3600B688C8844EA034300EB49
:104DE000CE04236401F10C038C681B8843EA04435E
:104DF00000EBCE04636443688D6943EA0204D1F892
:104E000010E0096A002D08BF03EA0C0444604369FE
:104E1000BEF1000F43EA020408BF03EA0C040129B3
:104E2000446102D1C1691143C161016821F00101EE
:104E300001600020B0BD000080B5FDF757FE0328DB
:104E400008BF80BD4CF21801C2F20101342210FBF0
:104E50000210006B002818BF804780BD90F820200A
:104E6000013A012A84BF00207047006810220029FF
:104E700008BF0C22805800F00300704710B590F86E
:104E80002040013C012C0AD8046871B12469A407B0
:104E90000ED100F1240101204FF4001276E000F160
:104EA000240101204FF4802270E0E468A40771D04F
:104EB000046804EB011CDCF8B0410CF5D87E14F05A
:104EC00004049460DCF8B04119BFE4085460640D38
:104ED0001460DEF800400CF5DA7E04F00204D460C1
:104EE000DCF8B44124075ABFDEF8004004F00F0498
:104EF00008241461DEF800400029C4F307249461FB
:104F0000DEF800404FEA14445461DCF8B8211A700E
:104F1000026802EB0112D2F8B8214FEA12225A704D
:104F2000026802EB0112D2F8B8214FEA12429A70DD
:104F3000026802EB0112D2F8B8214FEA1262DA706D
:104F4000026802EB0112D2F8BC211A71026802EB6E
:104F50000112D2F8BC214FEA12225A71026802EB08
:104F60000112D2F8BC214FEA12429A71026802EB98
:104F70000112D2F8BC214FEA1262DA71006814BF44
:104F800000F1100100F10C01002020220B681A43EF
:104F90000A6010BD00F1240101204FF40012F5E772
:104FA00090F820100139012984BF00207047006863
:104FB000816882688068C1F38061C2F3C062114475
:104FC000C0F30070084470472DE9F04F81B00446EB
:104FD00000684669D0F804908768D0F80CB0D0F823
:104FE00010A0D0F81880F10703D1002530071CD499
:104FF00023E0F90710D00121BA07816009D47807AE
:1050000000F1AA80380700F1B080204600F096FA3F
:1050100002E0204600F0A4FA0025F80500F18480A3
:10502000F80300F1AA80300707D51BF0100004D068
:10503000206845F400751021C160700708D51BF089
:10504000080005D020680821C160204600F0EEF974
:10505000B00706D52068C068800702D0204600F05F
:10506000F7F9700607D51AF0100004D0206845F44F
:10507000806510210161B00608D51AF0080005D03E
:10508000206808210161204600F0F4F9F00606D5F9
:1050900020680069800702D0204600F0FDF9B003C7
:1050A00008D519F0100005D0206810214160204675
:1050B00000F004FAF00308D519F0080005D02068C4
:1050C00008214160204600F0A5FA300440F18F80AD
:1050D0005FEA497040F1888006F4807008EA102089
:1050E00028435FEA8871014648BF41F00201B205DA
:1050F00058BF01465FEA48700D4648BF45F00405B9
:10510000700558BF0D4630056ED518F070006BD095
:1051100010380009052862D8DFE800F0035356591B
:105120005C5F45F008055AE020684FF48071BA05CD
:1051300081600AD4780512D4380519D4204600F0CD
:1051400021FAF8037FF56FAF17E0204600F02CFA44
:10515000F8037FF568AF10E04FF400655DE705F5F3
:105160000055F8037FF55FAF07E04FF4805554E733
:1051700005F58045F8037FF556AF20684FF4803180
:10518000BA0381600AD478030FD4380313D42046BD
:1051900000F01CFA30073FF548AF4EE7204600F01C
:1051A00027FA30073FF541AF47E705F500453007DF
:1051B0003FF53BAF41E705F5803530073FF535AFAB
:1051C0003BE745F010050AE045F0200507E045F013
:1051D000400504E045F0800501E045F48075206855
:1051E000816921F0700181612068042141602DB145
:1051F000606A284360622046FFF71EFE01B0BDE8EA
:10520000F08F0000B0B5C8B1044690F8200010B986
:10521000204600F071F82068016841F0010101604A
:1052200000F0CEFC054600BF20684168C90707D1E1
:1052300000F0C6FC401B0B28F6D312E00120B0BDE5
:10524000016821F00201016000F0BAFC054600BFD0
:105250002068416889070DD500F0B2FC401B0B287F
:10526000F6D3606A052140F400306062012084F8C2
:105270002010B0BD217E0268012922F0800208BF03
:1052800080320260617E0268012922F0400208BF7C
:1052900040320260A17E0268012922F0200208BF8C
:1052A00020320260E17E0268012922F0100218BF5C
:1052B00010320260217F0268012922F0080208BF33
:1052C00008320260617F0268012922F0040208BFEF
:1052D00004320260D4E901C2D4E9033561691A439A
:1052E0002A431143ACF101021143C16100200121A5
:1052F000606284F82010B0BDB0B586B0006846F694
:105300000002C4F2000200219042CDE90411CDE96F
:105310000211019136D046F20041C4F200018842E8
:1053200040F082804CF2C001C2F201010A6843F6EB
:105330004000C4F20200531C0B6052B900210091DE
:10534000016841F000710160016801F00071009195
:1053500000990021009150F8101C152441F008011B
:1053600040F8101C50F8100C142500F008000090B4
:1053700000980320019040F20040C4F2020000F5C2
:10538000006036E043F64000C4F20200009101687C
:1053900041F080610160016801F080610091009935
:1053A0004CF2C001C2F201010A68531C0B6052B9F1
:1053B00000210091016841F000710160016801F075
:1053C0000071009100990021009150F8101C4124B7
:1053D00041F0020140F8101C50F8100C402500F07C
:1053E0000200009000986020019040F20040C4F25A
:1053F000020002210291002103910321049109215D
:10540000059101A900F002FB28460521002200F0C9
:1054100093FD284600F08CFD20460521002200F077
:105420008BFD204600F084FD06B0B0BD80B5FDF7D1
:105430005DFB032808BF80BD4CF21801C2F20101D8
:10544000342210FB0210C069002818BF804780BDBD
:1054500080B5FDF74BFB032808BF80BD4CF2180157
:10546000C2F20101342210FB02108069002818BF2B
:10547000804780BD80B5FDF739FB032808BF80BD9C
:105480004CF21801C2F20101342210FB0210406AF2
:10549000002818BF804780BD80B5FDF727FB032893
:1054A00008BF80BD4CF21801C2F20101342210FB8A
:1054B0000210006A002818BF804780BD80B5FDF744
:1054C00015FB032808BF80BD4CF21801C2F2010190
:1054D000342210FB0210806A002818BF804780BD6C
:1054E000B0B5044690F8200001281DD1022084F8B0
:1054F00020002068016821F00101016000F060FBDC
:10550000054600BF20684068C00713D000F058FB74
:10551000401B0B28F6D3606A40F40030606205201F
:1055200084F820000120B0BD606A40F40020606271
:105530000120B0BD00206062B0BD000080B5FDF765
:10554000D5FA032808BF80BD4CF21801C2F2010150
:10555000342210FB0210C068002818BF804780BDAD
:1055600080B5FDF7C3FA032808BF80BD3421484346
:105570004CF21801C2F201010858002818BF8047F8
:1055800080BD000080B5FDF7B1FA032808BF80BDDB
:105590004CF21801C2F20101342210FB0210006922
:1055A000002818BF804780BD80B5FDF79FFA03280B
:1055B00008BF80BD4CF21801C2F20101342210FB79
:1055C00002104068002818BF804780BD80B5FDF7F5
:1055D0008DFA032808BF80BD4CF21801C2F2010108
:1055E000342210FB02104069002818BF804780BD9C
:1055F00080B5FDF77BFA032808BF80BD4CF2180187
:10560000C2F20101342210FB02108068002818BF8A
:10561000804780BD80B5FDF769FA032808BF80BDCB
:105620004CF21801C2F20101342210FB0210C06AD0
:10563000002818BF804780BD70B5866D044600F015
:10564000BFFA94F83510022925D105462068216C4F
:10565000026822F016020260426922F08002426172
:1056600009B9A16C19B1016821F008010160016854
:1056700021F00101016000BF20680068C0070ED062
:1056800000F09EFA401B0628F6D320206065032018
:1056900084F835000CE080206065012008E0E06DB2
:1056A0003F2101FA00F0B060012084F835000020AD
:1056B000002184F8341070BD90F83510022909D10A
:1056C000052180F835100068016821F001010160B2
:1056D000002070478021416501207047F0B581B0FE
:1056E00004460020009040F20000C2F20000026870
:1056F000D4E9166048F2B51337680821C1F64E3375
:1057000081403942A2FB03250CD0226813685B0755
:1057100008D5136823F004031360B160616D41F094
:105720000101616501218140394208D02268526936
:10573000120604D5B160616D41F00201616504217A
:105740008140394208D022681268920704D5B160BE
:10575000616D41F00401616510218140394215D02D
:1057600020680268120711D5B1600268016852030F
:1057700006D4C90506D4016821F00801016001E0E2
:10578000080342D4216C09B120468847E16D2020EE
:1057900000FA01F23A4244D020680368DB0640D5A3
:1057A000B26094F835300268052B1ED122F0160243
:1057B0000260426922F080024261226C0AB9A26C46
:1057C0001AB1026822F0080202603F208840B060EF
:1057D000012084F83500216D0020002984F8340070
:1057E00040D02046884701B0F0BD0168520310D474
:1057F000C90512D4016821F010010160012084F86C
:105800003500002084F8340007E0A16C0029BBD1EA
:10581000BCE7080301D4616C00E0E16B09B12046EC
:105820008847606DF0B1606DC00717D0052084F81F
:1058300035002068A90A026822F00102026000BF58
:10584000009A01328A42009202D80268D207F7D148
:10585000012084F83500002084F83400E16C09B19F
:105860002046884701B0F0BD2DE9F041044600F024
:10587000A7F9C4B10546022084F83500002021684C
:1058800084F83400086820F0010008602668306859
:10589000C0070BD000F094F9401B0528F6D903216E
:1058A0002022032042E00120BDE8F081306848F268
:1058B0003F01CFF21001251D00EA010C2ECDD4E9E5
:1058C000050E41EA0C01114319432943D4E9077835
:1058D000084340EA0E01606A3943042841EA08019E
:1058E00003D1D4E90B2311431943316071690428B2
:1058F00021F0070141EA00050CD1D4E90A1045EA7C
:10590000010538B12046FEF711FB18B101214022F4
:1059100001200BE020467561FEF7EAFAE16D3F22B7
:1059200002FA01F18160002201210020626584F801
:105930003510BDE8F0810000B0B5044690F83400A1
:10594000012828D0012084F83400A56D94F8350092
:1059500001281DD1022084F8350000206065204612
:10596000FEF70CFBE26D3F23206803FA02F2216C84
:10597000AA60026842F01602026019B1016841F0A3
:1059800008010160016841F0010101600020B0BD23
:10599000002084F834000220B0BD0000B0B50446F9
:1059A00000F00EF905464CF21000C2F2010000783A
:1059B000611C18BF044400BF00F002F9401BA04264
:1059C000FAD3B0BD70B54CF2800604460025C2F291
:1059D000010603E00135102D08BF70BD24FA05F063
:1059E000C007F7D056F82500002818BF8047F1E718
:1059F00080B543F61441C4F201010A68024208BFAF
:105A000080BD0860FFF7DEFF80BD00002DE9F04F8C
:105A100083B000F13E4202F1FF724FEAB22241F63A
:105A200000470192C4F2020708224FF0010E002540
:105A30004FF0000A4FF00008B84208BF072200925A
:105A40000AE000BF08F101080AF1040AB8F1100FDA
:105A500005F1020500F0A4800C680EFA08FB14EAB8
:105A60000B09EFD04C6804F0030CACF1010EBEF151
:105A7000010F11D80322876802FA05F6CA68B743F6
:105A8000AA403A4382604268C4F3001722EA0B023C
:105A900007FA08F73A434260BCF1030F1CD0C26812
:105AA00003238E6803FA05F7BA4306FA05F73A436B
:105AB000BCF1020FC2600FD16FF0030202EA58027C
:105AC00002440AF01C060F23176A03FA06F40B6956
:105AD000A743B3403B431362026803234F68AB40C4
:105AE0009A4307F00303AB401A4317F4403F4FF0CB
:105AF000010E0260A6D0002243F644030292C4F2D3
:105B000002031A6843F6004442F480421A601A689D
:105B1000C4F2010402F480420292029A28F00302C5
:105B20004FF6084B2244CFF6FF7B52F80B300AF0B9
:105B30000C070F26BE4023EA060C019B009E072B94
:105B400038BF1E4606FA07F747EA0C0342F80B3047
:105B5000A2684B6842EA090743F60C4CDE0258BFC4
:105B600022EA0907A760C4F2010CDCF800209E02BB
:105B700042EA090758BF22EA0907CCF800706268B8
:105B80009E0342EA090758BF22EA090767602268B4
:105B9000DB0342EA090358BF22EA0903236051E705
:105BA00003B0BDE8F08F00000069084018BF012075
:105BB00070470000002A08BF090481617047000097
:105BC0004DF6AC10C2F2010000687047F0B581B02C
:105BD000B0B3044690F83D0028B9002084F83C009A
:105BE000204600F0BFF8242084F83D0020680168BA
:105BF00021F001010160016841F400410160016888
:105C000021F40041016000F061FA48F28041C0F2E5
:105C10001E0140F60012656888424FF00001C0F294
:105C20003D0248F2A16C4FF0000338BF01219042C1
:105C3000C0F2010C38BF0123654538BF0B4613B1D4
:105C4000012001B0F0BD4DF68361C4F21B31A0FB11
:105C5000011221684FEA924E4B684FF4967623F07A
:105C60003F0343EA92434B6044F6D3530F6A0EFB63
:105C700006F6C1F26203A6FB033627F03F03B7091D
:105C8000654538BF970C7A1C1A430A62CA6948F204
:105C9000A0674CF6FF73C0F20107BD4222EA030C75
:105CA0000AD801386A00B0FBF2F001306FF31F3000
:105CB000042898BF04202BE0A368A0F1010E9BB13B
:105CC00019206843BEFBF0F00422013062F31F305C
:105CD000000512D09BB119206843BEFBF0F00422EE
:105CE000013062F31F3011E005EB4500BEFBF0F020
:105CF00001306FF31F300005ECD1012008E005EB07
:105D00004500BEFBF0F001306FF31F3040F400405F
:105D100040EA0C00C8610868D4E9072320F0C000FD
:105D2000104318430860886848F2FF3204F10C07FA
:105D300090438CCF18431043A6698860C86820F050
:105D4000FF0038433043C860086840F00100086035
:105D500000202021206484F83D10206384F83E0058
:105D600001B0F0BDB0B586B0006845F60001C4F2E0
:105D7000000100248842CDE90444CDE902440194A5
:105D800031D045F20041C4F20001884254D10024D0
:105D900043F630050094C4F20205286801A940F0DA
:105DA00002002860286800F00200009000984FF47C
:105DB000407001901220CDE90204032004900420D9
:105DC000059040F20040C4F20200FFF71FFE00946D
:105DD000286940F400102861286900F40010009040
:105DE000009806B0B0BD43F630050094C4F2020539
:105DF0002868122140F020002860286800F0200068
:105E0000009000980320019004900420059040F237
:105E10000040C4F20200CDE9021400F5805001A94F
:105E2000FFF7F4FD0094286940F480002861286998
:105E300000F480000090009806B0B0BD4CF2100055
:105E40004DF6AC11C2F20100C2F2010100780A68FD
:105E5000104408607047000080B543F60040C4F26B
:105E60000200016841F400710160016841F4806141
:105E70000160016841F480710160032000F06CF85A
:105E80000F2000F005F800F02BF8002080BD000086
:105E9000B0B54CF21002C2F2010240F200011278D9
:105EA000C2F200014FF47A730968B3FBF2F20446C0
:105EB000B1FBF2F1084601F05DF80F2C4FF001053F
:105EC0000CD858B94FF0FF3021460022002500F0D1
:105ED00033F840F2AC40C2F2000004602846B0BD86
:105EE00080B582B0002043F640010190C4F2020167
:105EF0004A6842F480424A604A6802F48042019251
:105F0000019A00900868002240F0805008600868FC
:105F10000F2100F08050009000986FF0010000F019
:105F20000BF802B080BD000080B504F025FF80BDF5
:105F300080B504F035FF80BD70B514460D460646A9
:105F400004F03EFF2946224603F072F8014630462F
:105F500004F03EFF70BD000080B504F053FF80BD2B
:105F60002DE9F041002800F08B8043F60808C4F2C8
:105F700002080446D8F8F8030D4600F007008842EE
:105F800007D288F8F853D8F8F80300F00700A842C1
:105F900076D12068810717D5410705D5D8F80010BC
:105FA00041F4E051C8F80010010705D5D8F80010F9
:105FB00041F46041C8F80010D8F80010A26821F040
:105FC000F0011143C8F80010C0073FD1D8F8F8031A
:105FD00000F00700A84207D988F8F853D8F8F8036A
:105FE00000F00700A8424BD12068410707D5D8F838
:105FF0000010E26821F4E0511143C8F800100007D6
:1060000008D5D8F80000216920F4604040EAC100BA
:10601000C8F8000000F07EF8D8F8001040F6C4126E
:10602000C1F30311C0F60102515C40F2000220FAF4
:1060300001F140F2AC40C2F200000068C2F200027E
:106040001160FFF725FF0020BDE8F0816068811E28
:10605000022907D258F8081C89015CBF0120BDE85D
:10606000F08110E0012807D158F8081C89035CBFB3
:106070000120BDE8F08106E058F8081C890702D429
:106080000120BDE8F081D8F8001021F00301084399
:10609000C8F80000FFF794FD064641F2883700BFBC
:1060A000D8F80000616800F00C00B0EB810F8DD0D3
:1060B000FFF786FD801BB842F2D90320BDE8F081CE
:1060C00040F20000C2F200000068704780B5FFF7A0
:1060D000F7FF43F60801C4F20201096840F6D41242
:1060E000C1F38221C0F60102515CC84080BD0000AE
:1060F00080B5FFF7E5FF43F60801C4F20201096825
:1061000040F6D412C1F34231C0F60102515CC840DE
:1061100080BD000010B543F60404C4F202046068B8
:1061200000F00C0008280AD0042819BF42F20040F1
:10613000C0F2F40041F60030C0F2B70010BD206894
:1061400021682368490241F60031C0F2B70100F02E
:106150003F02C3F388105CBF42F20041C0F2F40179
:10616000A1FB00010023FAF7C5F821680222C1F360
:10617000014102EB4101B0FBF1F010BD2DE9F0410E
:1061800082B0002800F0A2800446007843F60006A2
:10619000C007C4F2020643D0B06800F00C00042827
:1061A00005D1306880033BD56068C8BB8EE0B0681D
:1061B00000F00C00082802D170684002F1D4656834
:1061C000B5F5A02F0AD0B5F5803F0BD0306820F48C
:1061D00080303060306820F4802006E0306840F481
:1061E00080203060306840F480303060FFF7E8FC99
:1061F000002D054611D000BF3068800310D4FFF792
:10620000DFFC401B6428F7D922E100BFFFF7D8FC70
:10621000401B64284FF0030055D830688003F5D444
:10622000207880071AD5B06810F00C0F09D0B0683C
:1062300000F00C00082840F08A807068400200F1ED
:1062400086803068800702D5E06801283ED130683A
:10625000216920F0F80040EAC10030602078000792
:1062600038D4207840074CD4A5695DB3B06800F0FD
:106270000C00082840F09E80012D27D07068E1694D
:1062800000F480028A4221D1216A00F03F028A4252
:106290001CD147F6C071626A0140B1EB821F15D173
:1062A000A26A0023CFF6FF7303EBC23200F4403141
:1062B0006FF30F02914209D1E16A00F07060B0EB18
:1062C000016F03D1002002B0BDE8F081012002B0CF
:1062D000BDE8F0816069002840F20000C4F2472068
:1062E00057D00121C0F8801EFFF76AFC054600BFA9
:1062F000706F8007B5D4FFF763FC401B0228F7D905
:10630000A6E0306C10F080580AD100200190306C6B
:1063100040F080503064306C00F080500190019863
:1063200047F20007C4F200073868C00524D4386873
:1063300040F480703860FFF743FC05463868C005BC
:106340001AD4FFF73DFC401B0228F7D980E0E06833
:10635000002851D00020C4F2472001210160FFF73E
:106360002FFC0546306880073FF571AFFFF728FC2A
:10637000401B0228F6D96BE0A568052D50D0012DF1
:1063800052D0306F20F001003067306F20F00400F1
:106390004DE00021C0F8801EFFF712FC054600BF4B
:1063A000706F80077FF55DAFFFF70AFC401B022886
:1063B000F6D94DE00027C4F2472700203866FFF7E2
:1063C000FFFB022D05460BD13068800158D5FFF741
:1063D000F7FB401B02284FF00300F5D973E700BF1D
:1063E000306880017FF56EAFFFF7EAFB401B0228A3
:1063F0004FF00300F4D966E70020C4F247200021E3
:106400000160FFF7DDFB0546306880077FF526AFAA
:10641000FFF7D6FB401B02284FF00300F4D952E7E8
:10642000306F40F004003067306F40F0010030679B
:10643000FFF7C6FB002D054641F2883714D000BF98
:10644000306F800713D4FFF7BBFB401BB842F7D96E
:10645000032002B0BDE8F081FFF7B2FB401BB84259
:106460004FF003003FF62FAF306F8007F4D4B8F140
:10647000000F7FF4F9AE306C20F080503064F3E60A
:1064800004F11C052FCD08430021CFF6FF7140EA2F
:10649000821001EBC3316FF30F0140EA056008433E
:1064A000706001203866FFF78BFB0446306880017E
:1064B0003FF508AFFFF784FB001B02284FF00300F5
:1064C000F4D900E780B503F0A9F8022808BF80BD21
:1064D0004CF2C401C2F2010101EB401080690028B6
:1064E00018BF804780BD000070B538B10446406ACF
:1064F00030B10020206104F1140007E0012070BDDC
:106500006068B0F5827F03D004F11C0000210160B7
:106510000026A66294F8510020B9204684F8506005
:1065200000F03CF8022084F8510094E80F0001F4D8
:106530008271056802F4044225F0400505601144AB
:1065400003F400622369114403F0020263691144F9
:1065500003F00102A369E569114403F400721144D8
:1065600005F03802256A114405F08002A56A11433E
:1065700005F4005211430160626A042101EA1341EB
:1065800002F0100211444160C16921F40061C1614F
:106590000120666584F85100304670BD2DE9F04F4A
:1065A00087B0044643F200070068C4F201070026E2
:1065B000B8420696CDE904660396029602D007B06B
:1065C000BDE8F08F43F630000196C4F20200416945
:1065D00002AD41F480514161416946F2404801F405
:1065E000805101910199019601684FF0020941F033
:1065F0000201016001684FF0030A01F002010191FC
:106600000199019601684FF0050B41F0010101600D
:106610000068294600F001000190019818200290BE
:1066200007F55440C4F20208CDE90396CDF814A052
:10663000CDF818B0FFF7EAF98020CDE9020904A8E7
:1066400080E8400C07F550402946FFF7DFF94CF68B
:10665000AC55C2F201054FF440304FF0C0674FF423
:106660008069C5E908062846C5E90087C5E90266CC
:10667000C5E90496C5E90666FFF7F6F8002818BFD5
:10668000FDF776FEE564AC6340F61C0508F11800E2
:10669000C2F200054021C5E9000705F1080000220B
:1066A00080E806024FF40030C5E908022846C5E933
:1066B0000522EA61FFF7D8F8002818BFFDF758FE59
:1066C000A564AC6307B0BDE8F08F00002DE9F04190
:1066D00082B0044690F85100012815D10E460029D9
:1066E0004FF0010060D01746002A5DD060681D465B
:1066F000B0F5827F02D1A068002858D0FFF760FA79
:1067000094F85010012903D1022002B0BDE8F081B5
:106710008046012084F85000042084F851000020B5
:106720006065A663A787E7872063A086E086A168E7
:106730002064B1F5004F606408D12068016821F041
:1067400040010160016821F4804101602068016816
:10675000490603D4016841F040010160E168E08F1F
:1067600091B3002855D06E1C0BE000BFC068A16B30
:1067700021F8020BA163E08F0138E087E08F002849
:1067800047D020688168C907F0D1FFF719FA002EB9
:10679000F4D0A0EB0800A842F0D3012084F8510007
:1067A000002084F85000032002B0BDE8F0810420EE
:1067B00084F851002046314632463B46009500F0B1
:1067C0009FF902B0BDE8F08118B36E1C0BE000BF6A
:1067D000007BA16B0870A06B0130A063E08F0138D3
:1067E000E087E08FA8B120688168C907F0D1FFF782
:1067F000E7F9002EF5D0A0EB0800A842F1D3012064
:1068000084F85100002084F85000032002B0BDE855
:10681000F08120462946424602F072FE00281CBF45
:1068200020206065012084F85100002084F8500089
:10683000606D002818BF012002B0BDE8F0810000A3
:1068400010B5044690F8510001281CBF022010BD6D
:1068500013460A4600294FF0010018BF002B00D153
:1068600010BDA06858B96168B1F5827F07D10420D6
:1068700084F851002046114600F03EFA10BD94F80D
:106880005010012904BF022010BD012184F85010CE
:10689000042184F851100021B0F5004F6165A26316
:1068A000A387E387C4E91011A186E18608D1206897
:1068B000036823F040030360036823F4804303600C
:1068C000E06C49F2A93E49F2CD33C0F6000EC0F6A5
:1068D0000003C0E90F3E49F28533C0F60003D4F847
:1068E00000C0C0E91331E38F0CF10C01FFF724F86D
:1068F00040B1606D40F010006065002084F85000E9
:10690000012010BD21680868400603D4086840F0E3
:1069100040000860002084F850004A6842F02002DD
:106920004A604A6842F001024A6010BD80B502F038
:1069300075FE022808BF80BD4CF2C401C2F20101FD
:1069400001EB40104068002818BF804780BD000060
:1069500080B502F063FE022808BF80BD4CF2C4017E
:10696000C2F2010101EB40100069002818BF804706
:1069700080BD00002DE9F04182B01D4616460F464D
:106980000446FFF71DF994F8511001290DD18046F6
:10699000002F4FF0010018BF002E02D102B0BDE859
:1069A000F08194F85000012803D1022002B0BDE824
:1069B000F081012084F85000032084F85100002069
:1069C00060652763A686E686A063A087E087A16846
:1069D000C4E91000B1F5004F08D12068016821F02A
:1069E00040010160016841F4804101602068016854
:1069F000490603D4016841F0400101606168731EDB
:106A0000E268B1FA81F1B3FA83F349095B09B2F59F
:106A1000006F41EA030124D139B1216B0988C160BB
:106A2000B81C2063E08E0138E086E08E002846D056
:106A30006E1C09E0216B31F8022BC2602163E08EED
:106A40000138E086E08ED0B3206881688907F1D4F0
:106A5000FFF7B6F8002EF5D0A0EB0800A842F1D35E
:106A600023E039B139780173206B01302063E08E67
:106A70000138E086E08E10B36E1C0AE0216B0978C5
:106A80000173206B01302063E08E0138E086E08ED8
:106A9000A8B1206881688907F0D4FFF791F8002E2B
:106AA000F5D0A0EB0800A842F1D3012084F85100F2
:106AB000002084F85000032002B0BDE8F081204699
:106AC0002946424602F064FD00281CBF2020606574
:106AD000A06838B9002001902068C16801918068E1
:106AE00001900198012084F85100002084F85000A2
:106AF000606D002818BF012002B0BDE8F0810000E1
:106B00002DE9F04381B01E4615460F460446FFF7B7
:106B100057F894F851108146012909D06068B0F502
:106B2000827F14D104294FF0020007D1A16829B94E
:106B3000002F4FF0010018BF002D02D101B0BDE8B9
:106B4000F083002EFAD094F85000012803D10220DF
:106B500001B0BDE8F083012084F8500094F85100A2
:106B6000002104281CBF052084F851006165A5633D
:106B7000E687A6872763E6862068A6862164616487
:106B80000168490603D4016841F040010160616871
:106B9000731EE268B1FA81F1B3FA83F3DDF8208065
:106BA00049095B09B2F5006F41EA030139D139B1F6
:106BB000216B0988C160B81C2063E08E0138E08633
:106BC000012608F1010500BFE08E10B9E08F002812
:106BD0006CD02068816889070CD5E18E012E09D11F
:106BE00041B1216B002631F8022BC2602163E18E96
:106BF0000139E1868168C9070AD0E18F41B1C068D7
:106C0000A16B012621F8020BA163E08F0138E08718
:106C1000FEF7D6FF002DD7D0A0EB09004045D3D317
:106C20003AE039B139780173206B01302063E08E8E
:106C30000138E086012608F1010500BFE08E08B9A1
:106C4000E08F98B32068816889070DD5E18E012E09
:106C50000AD149B1216B002609780173206B0130FC
:106C60002063E08E0138E08620688168C9070BD078
:106C7000E18F49B1C068A16B01260870A06B01309B
:106C8000A063E08F0138E087FEF79AFF002DD5D092
:106C9000A0EB09004045D1D3012084F85100002029
:106CA00084F85000032001B0BDE8F083204641463F
:106CB0004A4602F06DFC40B120206065002084F857
:106CC0005000012001B0BDE8F083A06838B9002071
:106CD00000902068C16800918068009000980120B1
:106CE00084F85100002084F85000606D002818BF1F
:106CF000012001B0BDE8F08370B5044690F8510062
:106D0000012806D100294FF0010018BF002A0CD13C
:106D100070BD6568B5F5827F0ED104284FF0020082
:106D2000F6D1A568002DEDD0F2E7002B08BF70BDAD
:106D300094F85000012801D1022070BD012084F890
:106D4000500094F85100002604281CBF052084F848
:106D5000510066652163A386E386A263A387E38768
:106D6000C4E9106694F8510049F2A93149F2C133DF
:106D7000C0F60001C0F60003042808BF0B4649F224
:106D8000CD3049F2A541C0F60000C0F6000108BFB1
:106D90000146E06C2568C0E90F1349F28531C0F661
:106DA0000001C0E91316E38F05F10C01FEF7C4FDE5
:106DB00038B1606D40F010006065012084F85060CB
:106DC00070BD2268216BA06C536843F001035360CF
:106DD000C0E90F66C0E91366E38E0C32FEF7ACFD26
:106DE00040B1606D40F010006065002084F85000F4
:106DF000012070BD21680868400603D4086840F08F
:106E000040000860002084F850004A6842F02002E8
:106E10004A604A6842F002024A6070BD10B50446FA
:106E200090F8510001280AD100294FF0010018BF45
:106E3000002A00D110BD94F85000012801D1022091
:106E400010BD012084F850000320002384F8510075
:106E500063652163A286E286A363C4E91033A38736
:106E6000E387A068B0F5004F08D12068026822F0DF
:106E700040020260026842F480420260A06C49F263
:106E8000B53C49F23542C0F6000CC0F60002C0E93C
:106E90000F2C49F28532C0F60002D4F800E0C0E9B8
:106EA0001323E38E0EF10C02FEF746FD40B1606D38
:106EB00040F010006065002084F85000012010BDF3
:106EC00021680868400603D4086840F04000086064
:106ED000002084F850004A6842F020024A604A6864
:106EE00042F002024A6010BD80B502F097FB022812
:106EF00008BF80BD4CF2C4014001C2F20101085834
:106F0000002818BF804780BD80B502F087FB0228AB
:106F100008BF80BD4CF2C401C2F2010101EB401078
:106F2000C068002818BF804780BD000080B502F00F
:106F300075FB022808BF80BD4CF2C401C2F20101FA
:106F400001EB40108068002818BF804780BD00001A
:106F500080B502F063FB022808BF80BD4CF2C4017B
:106F6000C2F2010101EB40104069002818BF8047C0
:106F700080BD000080B502F0CBFD80BD70470000F1
:106F800070470000B0B590F83C20012A04BF0220F1
:106F9000B0BD01F108053CCDD1E900CE23F47C530E
:106FA00022F470521A432EF4F0431A432CF4E043B7
:106FB0001A4324F4C0431A432A43C96922F4804285
:106FC000036811435964002180F83C100846B0BDA5
:106FD00010B590F83C20012A4FF0020252D0012354
:106FE00080F83C3080F83D200268D2F804E0D2F806
:106FF00008C00C682EF07003234341F2FF74C4F202
:107000000004A24253600DDC40F2FF73C4F200039F
:107010009A4215DCB2F1804F29D040F20043C4F20D
:10702000000322E040F2FF33C4F201039A4212DC73
:1070300041F60003C4F200039A4218D0002312E084
:1070400040F60003C4F200039A4210D040F6004319
:10705000C4F2000309E044F20003C4F201039A42BF
:1070600005D040F20043C4F201039A4204D14968BA
:107070002CF08003194391600121002280F83D101B
:1070800080F83C20104610BD002804BF0120704746
:1070900010B5044690F83D0028B9002084F83C0063
:1070A000204600F01FF8022084F83D002068211DD2
:1070B00002F0B4FD012084F8460084F83E0084F814
:1070C0003F0084F8400084F8410084F8420084F8CE
:1070D000430084F8440084F8450084F83D00002013
:1070E00010BD000080B586B0006844F20042C4F2D2
:1070F000010200219042CDE90411CDE90211019174
:107100003AD00021C4F20101884243D1002043F665
:1071100044010090C4F202010A6842F001020A60D0
:107120000A6802F001020092009A009051F8140CD3
:1071300040F0100041F8140C51F8140C012100F03B
:107140001000009000984FF4C0400190022002907F
:10715000CDE9031041F200000591C4F2020001A93B
:10716000FEF754FC182005210022FEF7E5FE18204A
:10717000FEF7DEFE06B080BD43F644000091C4F287
:107180000200016841F400310160006800F4003041
:107190000090009806B080BD10B5044690F83C0001
:1071A00001284FF0020008BF10BD012284F83C20E6
:1071B00084F83D0020684FF6777382689A438260B6
:1071C0000A684F2A0FDC1F2A22DD202A23D0302A0A
:1071D00021D0402A4DD14B68CA68194602F09EFE64
:1071E000206840213BE06F2A17DDB2F5005F20D018
:1071F000B2F5805F2AD0702A3BD1D1E9012CCB684F
:10720000614602F0B3FD2068816841F077011AE021
:107210000AB1102A2DD1114621E0502A18D0602A37
:1072200027D14B68CA68194602F08AFE206860219F
:1072300015E0D1E9012CCB68614602F097FD20688A
:10724000816841F48041816000200BE0002009E06A
:107250004B68CA68194602F061FE2068502102F0AE
:1072600091FD0020012184F83D10002184F83C109C
:1072700010BD0120F6E7000070470000B0B50446DD
:107280000068C168026902EA0105A9071DD4680700
:1072900031D4280747D4E8065CD4E80773D1280620
:1072A0007BD4680606D520686FF040010161204656
:1072B00000F0E4F9A80658BFB0BD20686FF02001C7
:1072C00001612046FFF75CFEB0BD6FF00201016175
:1072D000012121778069800703D02046FFF7CCFF8A
:1072E00005E0204600F0B6F8204600F031F9002015
:1072F00020776807CDD520686FF004010161022175
:107300002177806910F4407F03D02046FFF7B4FF57
:1073100005E0204600F09EF8204600F019F9002014
:1073200020772807B7D520686FF008010161042194
:107330002177C069800703D02046FFF79DFF05E055
:10734000204600F087F8204600F002F90020207760
:10735000E806A2D520686FF01001016108212177AD
:10736000C06910F4407F03D02046FFF785FF05E099
:10737000204600F06FF8204600F0EAF80020207761
:10738000E8073FF48CAF20686FF0010101612046EF
:1073900000F072F928067FF584AF20686FF0800155
:1073A00001612046FFF7EAFD68067FF583AF7AE7C3
:1073B00080B586B0006844F20042C4F201020021A8
:1073C0009042CDE90411CDE9021101911FD00021B5
:1073D000C4F2010188423BD10020009043F6300006
:1073E000C4F2020001684FF0020C41F0100101608C
:1073F0000068012100F01000009000984FF4007028
:10740000019041F20000C4F20200012318E043F6AB
:1074100030000091C4F202000268032342F020020F
:10742000026000684FF0000C00F02000009000980F
:107430004020019041F20000C4F2020000F580609B
:107440000222CDE9022101A9CDE904C3FEF7DEFA4B
:1074500006B080BD70470000B0B5044690F83C000F
:10746000012804BF0220B0BD0D464FEAB201012041
:10747000032984F83C0037D8DFE801F0020A122221
:107480002068294602F086FC206850F8181F0EE09C
:107490002068294602F0B0FC206850F8181F16E05A
:1074A0002068294602F0DEFC206850F81C1F41F0DD
:1074B00008010160016821F00401016029690FE001
:1074C0002068294602F002FD206850F81C1F41F494
:1074D00000610160016821F480610160296909028D
:1074E0000268114301600020002184F83C10B0BD07
:1074F000002804BF0120704710B5044690F83D00F5
:1075000028B9002084F83C00204600F01FF8022033
:1075100084F83D002068211D02F080FB012084F8E2
:10752000460084F83E0084F83F0084F8400084F868
:10753000410084F8420084F8430084F8440084F851
:10754000450084F83D00002010BD00007047000099
:107550007047000010B5044641B1082909D004293C
:1075600014BF04F1410004F13F0004E004F13E00C7
:1075700001E004F14000007801281CBF012010BD8B
:10758000022041B1082909D0042914BF84F8410020
:1075900084F83F0004E084F83E0001E084F84000F5
:1075A0002068012202F0D0FB206841F2FF71C4F292
:1075B000000188420FDC40F2FF71C4F200018842F2
:1075C00017DCB0F1804F49D040F20041C4F2000115
:1075D000884243D049E040F2FF32C4F201029042B7
:1075E00014DC41F60003C4F20003984236D00023B5
:1075F00014E040F60001C4F2000188422ED040F6AB
:107600000041C4F20001884228D02EE044F2000379
:10761000C4F20103984221D040F20043C4F20103B6
:10762000984222D1436C884243F400434364C2DD54
:10763000904207DC41F60001C4F2000188420DD0FF
:10764000002107E044F20001C4F20101884205D0A4
:1076500040F20041C4F20101884206D1816801F084
:107660000701062904BF002010BD016841F0010197
:107670000160002010BD000070470000704700004E
:107680007047000080B503F0DFF8052808BF80BD13
:1076900040F2F85100EBC000C2F2000101EB8000A3
:1076A0000069002818BF804780BD0000B0B582B0D7
:1076B000036804461868D9685A6900F02F05202D20
:1076C00001F0200505D125B1204603F0E7F802B00E
:1076D000B0BD5FEA007C1EBF02F0010E01F49072A3
:1076E00012EB0E024AD1226B0840C1063DD5012A99
:1076F0003BD10020019018680190586801900198D2
:107700005869400642D4A08DE18DE28D002A1CBF4D
:10771000401A5FEA004101D102B0B0BD216851E8D2
:10772000031F226821F4907142E80313002BF5D166
:10773000216851E8051F226821F0010142E8051384
:10774000002BF5D1202184F842100021216300BFD5
:10775000216851E8031F226821F0100142E8031359
:10776000002BF5D10221616354E0010654D4400698
:10777000D2D5204603F04EF802B0B0BDC20718BF04
:1077800011F480725DD1420761D467E0E06B01685B
:1077900049688AB2002A44D0A38D9A4241D2E18539
:1077A000C069B0F5807F30D0206850E8030F2168B1
:1077B00020F4807041E80302002AF5D1206850E8E7
:1077C000050F216820F0010041E80502002AF5D1EB
:1077D000206850E8050F216820F0400041E80502CC
:1077E000002AF5D1202084F842000020206300BF49
:1077F000206850E8030F216820F0100041E80302E0
:10780000002AF5D1E06BFDF717FF02206063A08D21
:10781000E18D401A81B20FE0204603F067F902B013
:10782000B0BDA18D91427FF477AFC069B0F5807F84
:107830007FF472AF022060632046FFF721FF02B0A1
:10784000B0BD626C42F001026264420706D5BEF12F
:10785000000F03D0626C42F002026264820706D518
:10786000BEF1000F03D0626C42F004026264BCF10E
:10787000000F06D55EEA050203D0626C42F00802F2
:107880006264626C002A3FF447AF0840800602D56C
:10789000204603F003F820684069616C00F0400066
:1078A00001F00801401827D0204602F08BFF206825
:1078B000406940061BD500BF206850E8050F2168CD
:1078C00020F0400041E80502002AF5D1E06B70B1DC
:1078D0004AF27961C0F600010165FDF7EDFE00286E
:1078E0003FF41AAFE06B016D884702B0B0BD20468F
:1078F000FFF7C8FE02B0B0BD2046FFF7C3FE002070
:10790000606402B0B0BD0000002804BF01207047D1
:1079100010B5044690F8410028B9002084F84000D2
:10792000204600F021F8242084F841002068C16836
:1079300021F40051C160204603F014F82068016969
:1079400021F490410161416921F02A014161C1683E
:1079500041F40051C16000202021606484F841108E
:1079600084F84210606310BD2DE9F04387B00446EF
:10797000006840F6FF71C4F2010188424FF0000137
:107980000691CDE90411CDE902115FDC44F200411A
:10799000C4F20001884200F0B58044F60001C4F250
:1079A0000001884240F04A81002643F630000196EB
:1079B000C4F20200016941F480210161016901F40E
:1079C0008021019101990196016841F00401016053
:1079D000006802A900F00400019001984FF4406093
:1079E00002900220CDE903060320059007200690AF
:1079F0000020C4F2020000F50060FEF707F84CF624
:107A00000C6546F22800C2F20105C4F202004FF0F4
:107A100000614FF480624FF4807385E8430028468C
:107A2000C5E90362C5E90566C5E907366E62FDF77B
:107A30001BFF002818BFFCF79BFC27200521002214
:107A4000E563AC63FEF778FA272056E041F2004187
:107A5000C4F20101884200F0828041F20001C4F2C8
:107A60000101884240F0EA80002643F6300001968A
:107A7000C4F202004169002441F0100141614169F2
:107A8000C4F2020401F0100101910199019601680C
:107A900002AD41F00201016001684FF0020801F0FF
:107AA000020101910199019601684FF0030941F02B
:107AB000010101600068072700F0010001900198B2
:107AC0008020029004F580602946CDE90386CDF838
:107AD00014900697FDF79AFF4FF40070CDE9020865
:107AE00020462946CDE904690697FDF78FFF25203A
:107AF00005210022FEF720FA2520FEF719FA07B02B
:107B0000BDE8F083002043F630010190C4F2020189
:107B10000A6942F400320A610A6902F400320192F1
:107B2000019A01900A6842F008020A60096801F0AF
:107B3000080101910199602102910221CDE9031010
:107B400003200590072006900020C4F2020000F5F3
:107B5000406002A9FDF75AFF07B0BDE8F083002698
:107B600043F630000196C4F20200416946F228084B
:107B700041F0200141614169C4F2020801F0200195
:107B8000019101990196016841F04001016000688E
:107B900002A900F04000019001984FF48440029047
:107BA0000220CDE90306032005900820069000205E
:107BB000C4F2020000F5C050FDF728FF40F67C0536
:107BC00008F58060C2F200054FF020674FF480692D
:107BD000C5E900072846C5E90266C5E90496C5E976
:107BE0000666C5E90866FDF73FFE002818BFFCF7EA
:107BF000BFFBE563AC634CF66C6508F58F60C2F2C1
:107C000001054021C5E9000705F1080080E84202AE
:107C10002846C5E90566C5E907666E62FDF724FEDC
:107C2000002818BFFCF7A4FB472005210022A5630C
:107C3000AC63FEF781F94720FEF77AF907B0BDE89B
:107C4000F083000080B590F84230202B1CBF02204A
:107C500080BD00294FF0010318BF002A01D118464A
:107C600080BD0023036302F0EBFE0346184680BD8F
:107C700080B502F0E9FD052808BF80BD40F2F8514B
:107C800000EBC000C2F2000101EB8000C0680028D8
:107C900018BF804780BD000080B502F0D5FD0528E3
:107CA00008BF80BD40F2F85100EBC000C2F20001F5
:107CB00001EB80008068002818BF804780BD00006D
:107CC000B0B5044690F8410020281CBF0220B0BD8A
:107CD0004FF00100C9B3002A134608BFB0BD4FF0F2
:107CE000000C21202162A384E384C4F844C084F8FA
:107CF0004100A06B4AF2797E4AF2B9752268C0F65B
:107D0000000EC0F60005C0E90FE54AF28965C0F62D
:107D100000050432C0E9135CFDF70EFE30B11020FF
:107D20006064202084F841000120B0BD20686FF01D
:107D300040010160206850E8050F216840F0800094
:107D400041E80502002AF5D10020B0BD034690F8B5
:107D5000410020281CBF0220704700294FF001007D
:107D600018BF002A00D170471962002021219A848F
:107D7000DA84586483F841101968CA6842F08002B6
:107D8000CA60704780B502F05FFD052808BF80BD5E
:107D900040F2F85100EBC000C2F2000101EB80009C
:107DA0004068002818BF804780BD000080B502F001
:107DB0004BFD052808BF80BD40F2F85100EBC00024
:107DC000C2F2000151F82000002818BF804780BD92
:107DD000FEE7000045F6DF1110EE100AC5F6377118
:107DE000B6EE001AA1EB600020EE011A00EE100AB8
:107DF00021EE002A22EE002AB7EE083A33EE422A9C
:107E000022EE000A21EE001A20EE011A33EE411A8A
:107E100020EE010A7047000040F26111884204BF61
:107E200001207047B0F5806F04BF03207047A0F2B7
:107E30009F60B0FA80F040094000704710B52DED0A
:107E4000088B88B3B0EE408A90ED010A90ED069A57
:107E500090ED021A90ED07AA29EE000A38EE400ACA
:107E60002AEE011A30EE41BA04461BEE100A02F067
:107E70007BFF002808BFB0EE4B8A94ED030A94ED17
:107E8000041A94ED052A20EE080A29EE011A30EEB4
:107E9000010A2AEE021A30EE010A84ED068A84ED08
:107EA000079ABDEC088B10BD9FED020ABDEC088B54
:107EB00010BD00BF00000000002808BF704710B5CB
:107EC000F5EE400A0446C0ED000A0020F1EE10FA7B
:107ED000A061E0612EDD80EE200A9FED1E1A81EE8A
:107EE000000A07F0BBFA9FED1C1AB7EE002A20EE3D
:107EF000011A31EE023A20EE000ABFEE005A30EECF
:107F0000033A30EE055A32EE411A80EE034A35EE5E
:107F1000055A30EE010A85EE035A80EE030A34EE6C
:107F2000041A84ED034A84ED041A84ED054A84EDB5
:107F3000015A07E04FF07E519FED050AC4E9031096
:107F40006061606084ED020ABDE81040704700BFC8
:107F500000000000DB0F4940F304B53F10B52DEDE4
:107F6000048B10B3B0EE408A90ED030A90ED041A32
:107F700090ED052A30EE010A30EE020A88EE009AF2
:107F8000044619EE100A02F0DFFE00282046B0EE8B
:107F9000480A08BFB0EE489A84ED069A84ED079A25
:107FA000FFF74CFFBDEC048B10BD9FED020ABDEC4A
:107FB000048B10BD00000000B0B5012802D9FF20DD
:107FC00040B2B0BD4CF22C15C2F20105044655F882
:107FD000200060B98820FAF713FC002845F8240037
:107FE000EDD08821F8F7DAFB55F824000470002062
:107FF00040B2B0BD80B584B0D8B100F029F80146D8
:1080000000284FF0FC0015D08A888DF80C000092F3
:1080100008228DF804204FF0FF32CDF8052002929F
:1080200008786946FAF780FA002818BF4FF0FF3049
:1080300000E0FE2040B204B080BD000001288FBFE8
:1080400000204CF22C11C2F2010151F820007047BF
:108050002DE9F04128B3057880462846FFF7EEFF6A
:10806000F8B1014690F88400D8B10A1D002309E058
:108070000126002E08BFBDE8F08191F8846001332D
:10808000B3420ED252F82340002CF1D02678AE42F3
:10809000EED16688B8F80270BE42E9D100262046CB
:1080A000E7E70020BDE8F08110B50C460146002846
:1080B0004FF0FE0018BF002C01D140B210BD0846A1
:1080C000FFF7C6FF20B1214600F0D4F840B210BD42
:1080D000FC2040B210BD0000B0B52DED028B002891
:1080E0006BD00D46002968D00446B5F801009FED1D
:1080F000340A0004DFED330A00BA102104F0B4F9A9
:1081000084ED070AE8782979000140EA1110BBEEF6
:108110000E0AF3EE0E0A0C2104F0A6F984ED080A0B
:108120002879697900F00F00B0EE408A41EA00201A
:10813000BAEE080AF2EE080A0C2104F095F984ED73
:10814000090AA87994ED071A02EE100AB5EE401A52
:10815000B8EE422AF1EE10FA84ED0A2A0BDA9FED0E
:108160001A2A00BF31EE021AB5EE401AF1EE10FAEB
:10817000F8DB84ED071A94ED071A9FED132AB4EE8D
:10818000421AF1EE10FA0ADB9FED103A31EE031AB3
:10819000B4EE421AF1EE10FAF8DA84ED071AE0793B
:1081A00058B132EE411AB1EE482AB1EE400A84EDE0
:1081B000071A84ED082A84ED090ABDEC028BB0BDD4
:1081C000DA0F49C1DA0F4941DB0FC940DB0FC9C0E3
:1081D00070B538B104460078FFF7EEFE28B1FF20F5
:1081E00040B270BDFE2040B270BD2078FFF726FF80
:1081F0000028F4D090F8842005469AB1281D00216B
:1082000005E000BF95F88420013191420AD250F870
:108210002120002AF6D0528863889A42F2D1FD20AC
:1082200040B270BD1F2ADAD83020FAF7E9FA0028E8
:10823000D5D030210646F8F7B1FA20686168C6E962
:1082400000010020E27930722078618832760322C2
:10825000FAF724F818B13046FAF746FABFE795F86E
:10826000840005EB8001013085F88400002040B2D5
:108270004E6070BD2DE9F04381B02DED048B84B0CC
:10828000044600284FF0FE0071D00D4600296ED044
:1082900095ED001A95ED012A95ED023AE079B1EEDF
:1082A000430AB1EE428AB1EE419A002802BFB0EE15
:1082B000430AB0EE428AB0EE419ADFED300A9FEDFC
:1082C000301A102002F032FF8046FBEE0E0AB3EEA9
:1082D0000E1AB0EE480A0C2002F028FF9FED298A02
:1082E00095ED030A9FED281A0746F0EE480A0C2088
:1082F00002F01CFF95ED040A8146B1EE041AF0EE7F
:10830000480A0C2002F012FF0646FAEE080AB2EE06
:10831000081AB0EE490A0C2002F008FF3A094FEAA9
:108320001923A5888DF8072022784FEA182143EAFF
:108330000713070A47EA06173609009508258DF83E
:1083400005108DF80C00694610468DF804508DF824
:1083500006808DF808308DF809908DF80A608DF848
:108360000B70FAF7E1F8002818BF4FF0FF3040B269
:1083700004B0BDEC048B01B0BDE8F083DA0F49C155
:10838000DA0F4941000000000000FA43F0B587B061
:10839000A0B3077805463846FFF750FEA8B390F81B
:1083A000841069B3011D002205E000BF90F88430FD
:1083B00001329A4224D251F82240002CF6D0638830
:1083C0006E88B342F2D1F4B169886D4638462A46C8
:1083D0000023F9F75DFED0B1FAF7D6FAD4E9042309
:1083E000801A48F2A162C0F201029941801A71F12B
:1083F000000024BF00202072FF2014E0FE2012E0C5
:108400000024002CE0D1FC200DE0FC200BE001203A
:108410002072FAF7B9FAC4E9040105F10D0120460A
:10842000FFF75AFE002040B207B0F0BDB0B50128FA
:1084300002D9FF2040B2B0BD40F28C65C2F2000507
:10844000044655F8200060B94820FAF7D9F9002809
:1084500045F82400EDD04821F8F7A0F955F824009C
:108460000470002040B2B0BDB0B584B048B3047809
:108470000546204600F064F828B36988A1F201217E
:108480000A295BD8012202FA01F10A071DD111F075
:10849000F00F30D040F2FF11009108218DF8041048
:1084A0000A3000216A4600BF00EB41035B7802EB13
:1084B00041056B7110F8113001310429AB71F3D112
:1084C00031E0FE2037E0FC2035E04FF400710091F0
:1084D00008218DF80410023000216A4600EB4103A8
:1084E0005B7802EB41056B7110F811300131042902
:1084F000AB71F3D117E040F2FF21009108218DF814
:108500000410123000216A4600EB41035B7802EB55
:1085100041056B7110F8113001310329AB71F3D1B2
:108520000020ADF80B0069462046F9F7FDFF002852
:1085300018BF4FF0FF3040B204B0B0BDFF20FAE7E3
:1085400001288FBF002040F28C61C2F2000151F877
:108550002000704748B102280BD0012814BF4FF605
:10856000FF704FF4804000B2704742F2107000B2CA
:10857000704747F2305000B270470000022905D220
:10858000A0F2012189B2072909D805E007D1A0F29C
:10859000052189B2062902D8013840B27047FF2070
:1085A00040B27047F0B581B008B307460078FFF7D6
:1085B000C7FFE0B1014690F84400C0B101F11802D4
:1085C000002306E0012585B191F844500133AB4208
:1085D0000DD252F82340002CF4D065887E88B54235
:1085E000F0D100252046002DEED101B0F0BD0020D5
:1085F00001B0F0BD022884BFB7EE000A704740B258
:1086000002A101EB800090ED000A704700001042CB
:108610002CA099410000803F70B538B10446007825
:10862000FFF704FF28B1FF2040B270BDFE2040B22A
:1086300070BD2078FFF784FF0028F4D090F8442024
:1086400005469AB105F11800002104E095F8442090
:10865000013191420AD250F82120002AF6D05288E6
:1086600063889A42F2D1FD2040B270BD0A2ADAD85E
:108670005020FAF7C5F80028D5D006462068616872
:10868000C6E9000106F118002821F8F787F8627999
:108690002078618886F828200322F9F7FFFD18B1B9
:1086A0003046FAF721F8BEE795F8440005EB800163
:1086B000013085F84400002040B28E6170BD00009A
:1086C00070B52DED048B00283ED005460078B0EE45
:1086D000408AFFF735FFC8B3B7EE000AB4EE408A10
:1086E000F1EE10FAC8BFB0EE408ABFEE000AB4EE59
:1086F000408A0446F1EE10FAB8BFB0EE408A6879BD
:10870000B1EE489A0028284608BFB0EE489AFFF715
:1087100049FFE8B12E7968883146FFF72FFF00281E
:1087200018D405463046FFF715FF00EE100AB8EEE4
:10873000C00A29EE000ABDEEC00A10EE100A04EBD2
:1087400045014880002006E0FE2004E0FC2002E015
:10875000FC2000E0FF2040B2BDEC048B70BD0000A7
:108760002DE9F04F87B0002852D004460078FFF77B
:10877000E7FE00284ED0054690F8440000284BD074
:1087800005F11806E8464FF0010A40F2E93B4FF0C8
:10879000000908E00121002941D095F8441009F1B1
:1087A000010989453AD256F82970002FF2D07A880B
:1087B00061888A42EED1207842460023F9F768FCAE
:1087C00070B1FAF7E1F8D7E90823801A9941B0EBC4
:1087D0000B0071F1000016D300203876FC2013E066
:1087E00087F818A0FAF7D0F8C7E9080138464146DB
:1087F00000F06EFB07F108030FCB07F12C0C8CE89F
:108800000F00002000E0FF2000210029C5D106E074
:10881000FE2004E0FC2002E0FC2000E0FC2040B24E
:1088200007B0BDE8F08F000010B54CF6845046F25A
:108830000041C2F20100C4F200010322002380E8DB
:108840000E0000F10C014FF4C02C4FF4A00E4FF0BD
:10885000807481E808504FF4807184618183FCF753
:10886000D1FC002818BFFBF783FD10BD10B540F206
:10887000F47046F60001C2F20000C4F200010322C7
:10888000002380E80E0000F10C014FF4C02C4FF4DF
:10889000A00E4FF0807481E808504FF4807184611D
:1088A0008183FCF7AFFC002818BFFBF761FD10BD0A
:1088B00080B582B0002043F630010190C4F202017D
:1088C0000A6842F400120A600A6802F40012019277
:1088D000019A00900868002240F48000086008684F
:1088E000052100F48000009000980C20FDF724FB87
:1088F0000C20FDF71DFB392005210022FDF71CFB94
:108900003920FDF715FB3A2005210022FDF714FB65
:108910003A20FDF70DFB3B2005210022FDF70CFB63
:108920003B20FDF705FB452005210022FDF704FB58
:108930004520FDF7FDFA02B080BD000080B549F684
:10894000053040F6BC32C0F60000C0F6010200213E
:1089500002F07CFF40F20871C2F20001086049F6A3
:10896000E97040F64032C0F60000C0F60102002176
:1089700002F06CFF80BD00002DE9F04F87B00026AB
:1089800043F630000696CDE90466CDE9026601960D
:10899000C4F202000168002441F002010160016894
:1089A000C4F2020401F002010191019901960168EB
:1089B00004F5C05741F0400101600168002201F058
:1089C0004001019101990196016841F001010160A6
:1089D000016801F00101019101990196016841F0DE
:1089E00008010160016801F00801019101990196F7
:1089F000016841F004010160016801F00401019186
:108A000001990196016841F020010160016801F0BF
:108A10002001019101990196016841F080010160F6
:108A2000016801F08001019101990196016841F00E
:108A3000100101600068402100F0100001900198D1
:108A40003846FDF7B7F804F5E05A50464FF4E051C8
:108A50000022FDF7AFF82046102101224FF0010857
:108A6000FDF7A8F804F5805948464FF4006101224B
:108A7000FDF7A0F804F58060012101220090FDF7C8
:108A800099F8802002900220CDE903080590032088
:108A900004F5006B02AD069058462946FCF7B6FF78
:108AA0004020CDE9020838462946CDE90488FCF784
:108AB000ADFF4FF4E050CDE9020850462946CDE91C
:108AC0000486FCF7A3FF082002904FF404163846F2
:108AD0002946CDE90368FCF799FF20462946CDE9F0
:108AE0000286CDF81080FCF791FF1020CDE9020836
:108AF00020462946CDE90488FCF788FF302002A9EA
:108B000081E8410158462946FCF780FF4FF4006098
:108B1000CDE902080220059048462946CDF810808C
:108B2000FCF774FF00982946CDE90288CDE9048856
:108B3000FCF76CFF062005210022FDF7FDF9062059
:108B4000FDF7F6F9092005210022FDF7F5F90920C6
:108B5000FDF7EEF90A2005210022FDF7EDF90A20C4
:108B6000FDF7E6F9172005210022FDF7E5F91720AA
:108B7000FDF7DEF907B0BDE8F08F000080B54CF6D8
:108B8000CC6045F20041C2F20100C4F2000148F29B
:108B9000A06200234FF4804CC0F2010280E80E0076
:108BA000C0E9033CC0E90533C0E90733FDF70EF81F
:108BB000002818BFFBF7DCFB80BD000080B540F645
:108BC000DC0045F60001C2F20000C4F2000148F2E8
:108BD000A06200234FF4804CC0F2010280E80E0036
:108BE000C0E9033CC0E90533C0E90733FCF7EEFFF9
:108BF000002818BFFBF7BCFB80BD0000B0B54CF6E9
:108C0000207043F20001C2F20100C4F201014FF4EE
:108C10008272002380E80E0000F10C014FF0020C7C
:108C20004FF0010E4FF40074182581E808500A2116
:108C3000C0E90645C0E90833C0E90A31FDF754FC34
:108C4000002818BFFBF794FBB0BD000080B588B0CA
:108C500040F6781044F200420021C2F20000C4F253
:108C6000010241F288330791CDE90511CDE90311E5
:108C7000CDE90111C0E90021C0E902130161816160
:108C8000FEF702FA002818BFFBF772FB40F67810D7
:108C9000C2F20000FEF72CFC002818BFFBF768FBAF
:108CA000602001900020CDE90200059040F6781088
:108CB000C2F2000001A90022FEF7CEFB002818BF77
:108CC000FBF756FB40F67810C2F20000FEF770FB8F
:108CD00008B080BD10B596B040F6301000220021DB
:108CE000C2F20000C4F20102A72344F61F641591EA
:108CF000CDE91311CDE91111CDE90F11CDE90D1118
:108D0000CDE90B11CDE90911CDE90711CDE9051127
:108D1000CDE90311CDE90111C0E90023C0E9021436
:108D2000C0E904118161FEF7AFF9002818BFFBF715
:108D30001FFB4FF48050129040F63010C2F200003A
:108D400012A9FEF729FA002818BFFBF711FB40F61D
:108D50003010C2F20000FEF7CBFB002818BFFBF773
:108D600007FB40F630100024C2F2000010A9CDE944
:108D70001044FEF72DF9002818BFFBF7F9FA602020
:108D8000CDE9090440F63010C2F2000009A9002222
:108D9000CDE90B44CDE90D440F94FEF75DFB0028AF
:108DA00018BFFBF7E5FA00200590CDE90300CDE9F7
:108DB00001004FF40051089040F630100691C2F2C5
:108DC000000001A9FEF7DEF8002818BFFBF7D0FA73
:108DD00040F63010C2F20000FEF7EAFA16B010BDFD
:108DE00080B54CF6787041F20001C2F20100C4F285
:108DF000010100234FF00C0C4FF4E13280E80E002B
:108E0000C0E90333C0E905C3C361FEF77DFD002857
:108E100018BFFBF7ADFA80BD80B540F6C01044F234
:108E20000041C2F20000C4F2000100234FF00C0C1C
:108E30004FF4E13280E80E00C0E90333C0E905C316
:108E4000C361FEF761FD002818BFFBF791FA80BDF2
:108E500010B54CF6C07044F6000C48F2A062C2F2A5
:108E60000100C4F2000CC0F201024FF48053002153
:108E70004FF4806E0424C0E900C2C0E90231C0E9A9
:108E800004E4C0E90611FEF73FFD002818BFFBF718
:108E90006FFA10BD80B540F6082041F20041C2F2E1
:108EA0000000C4F2010100234FF00C0C4FF4E1323A
:108EB00080E80E00C0E90333C0E905C3C361FEF7D3
:108EC00023FD002818BFFBF753FA80BDFEE7000022
:108ED0002DE9F0478846B1F80D10044608BA4FEA6C
:108EE0001049B8F811002679B8F80F1005BA3046C5
:108EF00091FAB1FAFFF72EFB07463046FFF77AFBEF
:108F000001EE109A9FED453AB8EE412A9FED441AC2
:108F100022EE032A22EE014A02EE10AA15FB27F0E8
:108F2000B8EEC23A02EE100AA0799FED3E5AB8EEB2
:108F3000C22A22EE052A48B1B4F84000A9EB00008D
:108F4000B0F5805F0CDD4FF0FF300DE00020A4F89D
:108F50004090C4E9110084ED024A84ED033A1CE01C
:108F600010F5805F03DA0120616C0844606494EDC1
:108F7000115A83EE003AB8EEC55A25EE015A34EE86
:108F8000054A84EE004AA4F8409020EE022A84EDBF
:108F9000033A84ED124A84ED024A94ED020A84ED0C
:108FA000042AB5EE400AF1EE10FA08DA30EE010AB2
:108FB000B5EE400AF1EE10FAF8DB84ED020A94ED0A
:108FC000020AB4EE410AF1EE10FA0ADB9FED162A0E
:108FD00030EE020AB4EE410AF1EE10FAF8DA84ED4E
:108FE000020A94F8280078B131EE400A84ED020AB2
:108FF00094ED030A94ED041AB1EE400A84ED030ADD
:10900000B1EE410A84ED040A98F8130000EE100A4C
:10901000B8EE400A84ED050ABDE8F087000000398B
:10902000DB0FC94000008038DB0FC9C0FEE700003D
:1090300000F0070080F00703042B28BF04234FF043
:10904000FF3C03380CFA03F338BF002099438140FA
:109050000CFA00F022EA000008437047B0B52DED8D
:109060000A8B044610EE100AB0EE618AB0EE419A07
:10907000B0EE60AAB0EE40BA01F06EFE002800F03B
:109080009C801AEE100A01F067FE002800F095801F
:1090900019EE100A01F060FE002800F08E8018EE34
:1090A000100A01F059FE002800F087806068B0EED9
:1090B0004B0A90ED071AF0EE4A0AFAF7B9FE60681B
:1090C000B0EE40BA90ED001A04F11C0020EE01CA87
:1090D00021EE0A0AFEF7B2FE207888B1012811D1EC
:1090E00094ED051A94ED022A30EE411AB4EE428A4C
:1090F000F1EE10FAC8BFB0EE482A81EE029A01E004
:109100009FED309A19EE100A84ED04BA84ED050A39
:1091100001F022FE65689FED2B0A002808BFB0EE23
:10912000409A95ED010A95ED032A2CEE000A29EEEE
:10913000022A95ED021A30EE42AA94ED030A9FED41
:10914000229A2CEE082A32EE008AB4EE491AF1EE89
:1091500010FA28EE01BA1ADD18EE100A01F0FCFD33
:10916000A8B13AEE0B0A95ED051AB0EEC00AB4EEBE
:10917000410AF1EE10FA0ADC95ED040AB0EEC81AC5
:10918000B4EE401AF1EE10FAD8BF84ED038A3AEE3D
:109190000B8A18EE100A01F0DFFD70B1D5ED050A5B
:1091A000F4EE490AF1EE10FA05DDB0EE480AF8F7E0
:1091B000BBFCB0EE408A84ED068A94ED060ABDEC55
:1091C0000A8BB0BD00000000BD37863570B52DEDAF
:1091D000048B90B3044650681646B0EE408A0D46A4
:1091E00001F0BAFD58B3B06801F0B6FD48B3F068BD
:1091F00001F0B2FD38B3306901F0AEFD28B37069FB
:1092000001F0AAFD18B3B7EE000A80EE089A666076
:1092100019EE100A01F0A0FDD8B1D6ED060A04F14E
:109220001C00B0EE480A84ED029AFEF745FE204687
:10923000257000F013F800200CE0FF200AE0FF206A
:1092400008E0FF2006E0FF2004E0FF2002E0FF200E
:1092500000E0FF2040B2BDEC048B70BD10B568B1DA
:1092600000F11C0100249FED070AC0E90344C0E996
:1092700005440846FEF772FE60B210BDFF2460B2DE
:1092800010BD00BF00000000000000000000000052
:10929000EFF30980BFF36F8F154B1A681EF0100FA4
:1092A00008BF20ED108A20E9F04F10602DE9090079
:1092B0004FF0500080F31188BFF34F8FBFF36F8FD3
:1092C00003F040FC4FF0000080F31188BDE8090076
:1092D00019680868B0E8F04F1EF0100F08BFB0EC36
:1092E000108A80F30988BFF36F8F704700BF00BFFB
:1092F000A4D0012080B502F0A5FA4DF29811C2F277
:1093000001010860A8B149F23932C0F6000202201A
:109310000321F9F78FFB4CF23411C2F20101002056
:10932000C1E90000C1E90200C1E90400087640B2C9
:1093300080BDFE2040B280BD80B54DF29810C2F2D3
:1093400001000068012102F0DFF980BD80B5022034
:10935000F9F742FB4CF23411C2F201011922FEF777
:1093600071FC002818BF4FF0FF3080BD80B5024669
:109370000120012102F008FA0138B0FA80F040091A
:1093800080BD000080B5806B01684A6822F003024E
:109390004A60416D41F010014165012180F8511092
:1093A000FDF790F880BD000080B5806BFDF7D0FA26
:1093B00080BD000080B5806BFDF7A6FD80BD00007C
:1093C00080B5806BFDF7C4FD80BD0000B0B5846B37
:1093D0000546FCF7F5FB29680968C90526D402464D
:1093E0002068A168436823F02003436031B96168B5
:1093F000B1F5827F02D16FF0030101E06FF001014E
:109400004368194041602046642100F079F8002843
:109410001CBF202060650020E087012084F85100F7
:10942000606D18B12046FDF74DF8B0BD2046FDF740
:109430007DFAB0BDB0B582B0846B0546FCF7C0FBC9
:1094400029680968C90528D402462068416821F0C6
:1094500020014160416821F0020141602046642101
:1094600000F096F818B1606D40F020006065A068CB
:1094700038B9002001902068C1680191806801908E
:1094800001980020E086012084F85100606D20B131
:109490002046FDF717F802B0B0BD2046FDF724FDC9
:1094A00002B0B0BDB0B5846B0546FCF789FB2968F6
:1094B0000968C9051FD402462068416821F02001CF
:1094C00041602046642100F063F818B1606D40F0FF
:1094D000200060652068416821F0030141600020A0
:1094E000E086E087012084F85100606D18B12046C5
:1094F000FCF7E8FFB0BD2046FDF718FDB0BD000049
:10950000B0B582B0044640680B46B0F5827F20D1EA
:10951000A168B1F5004F02D0B1F5806F04D1216888
:109520000D6825F040050D60B0F5827F11D1A0686F
:10953000B0F5806F1DD10092204601210022002548
:1095400000F076F890B1606D032540F02000606572
:109550000CE00092204601210022002500F068F86E
:1095600020B1606D032540F020006065284602B000
:10957000B0BD0092204680210022002500F058F85E
:109580000028F3D0606D032540F020006065EDE712
:1095900070B582B00D461646022101222B460446C4
:1095A000009600F045F838B1606D032540F02000CA
:1095B0006065284602B070BD40F20000C2F20000B3
:1095C000006849F68171C1F25E61A0FB0101480D9E
:1095D0004FF47A71484301906068B0F5827F0FD1F3
:1095E0002046802100222B460096002500F020F81E
:1095F0000028DED0606D032540F020006065D8E7CC
:10960000019840B1019801380190206880680006F7
:10961000F6D40025CDE70025CBE70000006843F233
:109620000001C4F20101401A18BF01204000704738
:109630002DE9F04782B00A9C984615460E468146B1
:10964000FCF7BEFA201A00EB0804FCF7B9FA40F266
:109650000001C2F200010968C1F3CB3161430191FD
:10966000D9F8001089683140891BB1FA81F14909A4
:10967000A94203D1002002B0BDE8F087824608F17C
:1096800001070CE0019801380190D9F800008068CA
:109690003040801BB0FA80F04009A842EAD0002F89
:1096A000F3D0FCF78DFAA0EB0A00A04204D2019897
:1096B0000028E7D10024E8E7D9E900014268B1F5C4
:1096C000827F22F0E00242600BD1D9F80810B1F598
:1096D000004F02D0B1F5806F03D1016821F0400145
:1096E0000160D9F82810B1F5005F07D1016821F4B5
:1096F00000510160016841F400510160012089F8C6
:109700005100002089F85000032002B0BDE8F08726
:10971000074B19680868B0E8F04F80F30988BFF379
:109720006F8F4FF0000080F31188704700BF00BFBB
:10973000A4D0012080B501F05DFB80BDB0B52DED5A
:10974000028B9FED1C8AD0ED011A90ED0B0AD0ED33
:10975000650A044600F5F76500F5F670B0EE481AA4
:10976000FFF77CFCD4ED011AD4ED690A04F51970F9
:10977000B0EE481AFFF772FC85ED000AD4ED011A2D
:1097800094ED0B0AD4ED660A04F50A70B0EE481A9F
:10979000FFF764FCD4ED011AD4ED6A0A04F52870D1
:1097A000B0EE481AFFF75AFC85ED010ABDEC028BBA
:1097B000B0BD00BF000000002DE9F04F81B02DEDDD
:1097C000028B834600284FF0FF0000F0928088460D
:1097D000002900F08E80B5EE400AB0EE408AF1EE2E
:1097E00010FA40F3868098F80440CBF81880F8F718
:1097F0008FFCB4B308F1700908F1900A08F12C0548
:109800000BF5D2760BF2EC472846FEF705FF304603
:109810000121B0EE480A4A46FFF7D8FC06F5B470BD
:109820000121B0EE480A5246FFF7D0FCDBF81800E1
:10983000B0EE480AD0ED4C0A3846FEF73DFBDBF8A7
:109840001800B0EE480AD0ED4D0A07F1C000FEF74F
:1098500033FB013C05F10A0506F13C0607F1200740
:10986000D2D108F16800FEF7D7FEDBF8180090F8B7
:109870006C0078B101283BD10BF2744008F1F00282
:109880000121B0EE480AFFF7A1FC0BF5966008F540
:1098900088720CE00BF2744008F1B0020121B0EEC6
:1098A000480AFFF793FC0BF5966008F1D0020121FE
:1098B000B0EE480AFFF78AFCDBF81800B0EE480A61
:1098C000D0ED4E0A0BF26C60FEF7F6FADBF81800EA
:1098D000B0EE480AD0ED4F0A0BF28C60FEF7ECFABE
:1098E0000020CBE94700CBE94900CBF82C0100E090
:1098F000FC2040B2BDEC028B01B0BDE8F08F00004F
:1099000000280EBFFF200177002040B27047000002
:10991000002800F0EB802DE9F0472DED068B824604
:10992000806990F80480B8F1000F57D09FED718ADC
:109930004FEA88093427002540F2EC462424B7EE8C
:10994000009ABFEE00AA2EE00AEB040090ED000A98
:109950000AEB0600FEF772FA80EE081A0AEB050021
:1099600080ED380A043520361034B4EE491AF1EE91
:1099700010FAC8BFB0EE491ADAF81810B4EE4A1A55
:10998000F1EE10FAB8BFB0EE4A1AC95D80ED3E1A8A
:109990000AEB810090ED430A0A3730EE010AA9452F
:1099A00080ED430A1AD0DAF8180038440838FEF778
:1099B000D7FEDAF8180038440838FEF7F3FD00281F
:1099C000C2D000F12C0C0AEB85019CE80C10806BD6
:1099D00001F1200E8EE80C10C862B5E79AED450A39
:1099E00001EE108AB8EEC11A80EE010ADAF818000A
:1099F000B6EE001A683020EE010A8AED450AFEF73D
:109A0000AFFEDAF818006830FEF7CCFD01460AF127
:109A100080005022F6F788FEDAF818009AED321A24
:109A200090ED040A20EE010AB5EE400AF1EE10FABC
:109A30008AED490A0BDA9FED301A00BF30EE010AB9
:109A4000B5EE400AF1EE10FAF8DB8AED490A9AED1C
:109A5000490A9FED291AB4EE410AF1EE10FA0ADB29
:109A60009FED262A30EE020AB4EE410AF1EE10FA1A
:109A7000F8DA8AED490A9AF8A80000281CBF31EEEE
:109A8000400A8AED490A9AED230A0AF26C60FEF751
:109A9000D5F99AED231A9FED1A2AB7EE003A81EE16
:109AA000021A8AED4A0A9AED090A9AED0D2A0AF27B
:109AB000AC6030EE420AB4EE431AF1EE10FAC8BFC1
:109AC000B0EE431ABFEE003AB4EE431AF1EE10FACC
:109AD000B8BFB0EE431A8AED4B1A80ED000A0020A1
:109AE000BDEC068BBDE8F04740B27047FF2040B2A6
:109AF000704700BF00C0DA45DB0FC940DB0FC9C0AB
:109B00000080BB4580B501F09DFE01F0F9FE80BDEF
:109B1000B0B501380024B4EB106F1CBF0120B0BDFC
:109B20004EF21005CEF2000568604FF0FF300F21B5
:109B300001F04EF90720AC6028602046B0BD00005F
:109B400080B5FCF77BF903F023FF012818BF03F071
:109B5000F5F880BD70B592B006AC20463021F6F71E
:109B60001DFE002543F640000595CDE90355CDE9DE
:109B700001550095C4F202000168022641F08051AF
:109B80000160006800F080500090009847F20000EB
:109B90000095C4F20000016841F480410160006852
:109BA00000F4804000900098012006904FF480302F
:109BB00007904FF480000D9006200E90A820CDE96C
:109BC0000F060420119020460C96FCF7D7FA88B9AE
:109BD0000F20CDE901064FF4A05004904FF48050BF
:109BE000059001A805210395FCF7BAF9002804BFE8
:109BF00012B070BDFAF7BCFB4EF68850CEF20000F2
:109C0000016841F4700101607047000080B540F6C2
:109C10003010C2F20000FDF731FB80BDB0B540F658
:109C2000FF3E0568C4F2000E40F2004C7045C4F2DD
:109C3000010C0FDCB0F1804F19D040F20043C4F2A8
:109C40000003984213D040F60003C4F20003984288
:109C50000DD011E040F60043C4F20003984206D054
:109C6000604504D00023C4F20103984204D14B683C
:109C700025F0700243EA020541F6FF73C4F20003C7
:109C800098420DDC70451FDCB0F1804F41D040F2AE
:109C90000043C4F2000398423BD040F6000321E0A9
:109CA00043F6FF73C4F20103984220DC42F2000342
:109CB000C4F2000398422CD00023C4F2010398425E
:109CC00027D0604525D029E040F60043C4F20003C8
:109CD00098421ED041F60003C4F20003984218D007
:109CE00041F60043C4F20003984212D016E044F259
:109CF0000003C4F2010398420BD044F60003C4F2FF
:109D00000103984205D044F20043C4F20103984293
:109D100004D1CB6825F4407243EA02050A688C68D6
:109D20004B69C46240F480648262644504BF09697F
:109D30000163026825F0800142F0040219430260C9
:109D4000012242610160B0BD80B501F01F014FF0FA
:109D5000010CD0F820E00CFA01F32EEA03030362B1
:109D6000036A02FA01F11943016280BDD0F808C00C
:109D700011432CF47F4C41EA032141EA0C0181603C
:109D800070470000826822F07002114341F0070121
:109D900081607047B0B5026A036A40F2004523F063
:109DA00001030362D0F804E0D0F818C08C6822F0F8
:109DB000020240F48063C4F20105AB4242EA0402AD
:109DC00005D1CC6822F00C0224F0040422430C6874
:109DD000AB4207D1D1E905532EF4407E45EA0E058A
:109DE00045EA030E2CF073032343C0F804E08361BB
:109DF000496841630262B0BD70B5026A036A40F20D
:109E0000004423F010030362D0F804E0D0F818C037
:109E10008D6822F0200240F48063C4F20104A34262
:109E200042EA051207D1CD686FF0400622F0C00269
:109E300006EA05152A430D68A34207D1D1E9056456
:109E40002EF4406343EA860343EA840E2CF4E6438F
:109E500043EA0523C0F804E0836149688163026234
:109E600070BD000070B5026A036A40F2004423F43A
:109E700080730362D0F804E0D0F81CC08D6822F42F
:109E8000007240F48063C4F20104A34242EA052256
:109E900007D1CD6840F2FF462D0222F44062B5435F
:109EA0002A430D68A34207D1D1E905642EF440533B
:109EB00043EA061343EA041E2CF073032B43C0F855
:109EC00004E0C3614968C163026270BD70B5D0F837
:109ED00020C0026A40F2004622F4805202624268C8
:109EE000C3690C68D1F808E040F48065C4F201064B
:109EF000B54204D14D6922F4804242EA851223F42E
:109F0000E64343EA04234260C3612CF400564968E7
:109F100046EA0E320164026270BD0000D0F820C033
:109F2000036A23F001030362836923F0F00343EA29
:109F300002122CF00A03194382610162704700008B
:109F4000D0F820C0036A23F010030362836923F46E
:109F5000704343EA02322CF0A00343EA011182610C
:109F6000016270470000000001F0E0F905F0A9FF70
:109F70009FED1B0B53EC102B05F0E0FD05F074FF7B
:109F80000446002001F08AF901F0C6F90546FFF702
:109F9000B1F94CF618264DF2B8072544C2F2010675
:109FA000C2F2010710E000BF3046FAF779F8B86D49
:109FB00001F002FBB86D31460022002301F0B4FA33
:109FC000284601F07BF92544FFF7C0F91420FFF77C
:109FD000CDF90028E8D03046FAF718F8E7E700BFD7
:109FE0000000000000407F4010B501F0B7F94AF2D0
:109FF000411040F66822C0F60000C0F601020021C0
:10A0000001F024FC4DF2B804C2F2010420604AF2CF
:10A01000E14040F61C32C0F60000C0F6010200210B
:10A0200001F014FC60604AF2F92040F6B022C0F65C
:10A030000000C0F60102002101F008FCA0604AF215
:10A04000915040F66432C0F60000C0F601020021D3
:10A0500001F0FCFBE0604AF2811040F68C22C0F671
:10A060000000C0F60102002101F0F0FB20614AF27D
:10A07000794040F6F822C0F60000C0F60102002147
:10A0800001F0E4FB60614AF2913040F6D422C0F660
:10A090000000C0F60102002101F0D8FBA06149F6E2
:10A0A000697040F64422C0F60000C0F601020021AB
:10A0B00001F0CCFB20624AF2196040F68832C0F60B
:10A0C0000000C0F60102002101F0C0FB6062022026
:10A0D0000A21002201F0D8F9A062022034210022D6
:10A0E00001F0D2F9606302201421002201F0CCF9C2
:10A0F000A06302202021002201F0C6F9A064022002
:10A100000321002201F0C0F9E06202205821002260
:10A1100001F0BAF9606502204D21002201F0B4F986
:10A12000A06502204D21002201F0AEF9A06501F0EA
:10A1300045F901F087FB01F0E3FB10BD00000000D2
:10A1400001F0F4F805F0BDFE9FED0B0B53EC102B66
:10A1500005F0F4FC05F088FE0446002001F09EF8AE
:10A1600001F0DAF8051900BF284601F0A7F82544E8
:10A17000FAE700BF00BF00BF0000000000407F40C2
:10A1800084B001F0D3F805F09CFE9FED570B53EC23
:10A19000102B05F0D3FC05F067FE0546002001F00A
:10A1A0007DF801F0B9F84CF2E80AC2F2010A4CF26B
:10A1B00004010446C2F201015046F7F70BFD504678
:10A1C000F7F7E2FC4CF6705040F65821C2F201005D
:10A1D000C2F20001F6F7A0FF5046F7F7D5FCB7EE44
:10A1E000001A81EE000A4DF2080040F69042C2F2D9
:10A1F0000100C0F601020021FEF7E8FF0120F8F798
:10A2000033FB0AF110004CF668289FED398A9FED68
:10A21000399A40F2C07904EB050B02900AF11C0058
:10A22000C2F20108C2F2000903950190F7F720FE7F
:10A23000F7F796FCF7F7A0FCF7F7B6FCF7F7C2FCC8
:10A2400001F08CF85046F7F767FD5046F7F7AEFD82
:10A250004CF67054C2F20104DDE9012140F65823A6
:10A260002046C2F20003F7F71FF840462146F6F7F2
:10A27000E5FE01F0A3F8DAED0A0A4DF20800C2F299
:10A280000100B0EE480AB0EE491AF0EE491AFEF7A6
:10A29000E5FE0120F8F7B8FA0AF1100C9CE8181056
:10A2A00098E80700DAF82460C9E90A344DF2B804E6
:10A2B000C2F20104DAE90775C9E90260606BC9E915
:10A2C0000075C9E90412C9F830C001F075F9606B76
:10A2D00049460022002301F027F9584600F0EEFF1E
:10A2E00003988344A2E700BF0000000000407F40C5
:10A2F000000020420000000001F018F805F0E1FD28
:10A300009FED1F0B53EC102B05F018FC05F0ACFD76
:10A310000446002000F0C2FF00F0FEFF0646F9F7F9
:10A32000B9FD4CF26015C2F201059FED170A00F568
:10A330003071284600F076FD4DF2B80840F294677F
:10A340002644C2F20108C2F2000700BFD8F8480054
:10A3500039460022002301F053F82846F9F74CFC57
:10A36000284639463246F8F7B9FF2846F9F714F976
:10A37000304600F0A3FF2644E8E700BF00BF00BF5F
:10A380000000000000407F400000FA430000000091
:10A3900082B000F0CBFF05F094FD9FED350B53EC40
:10A3A000102B05F0CBFB05F05FFD0446002000F00C
:10A3B00075FF00F0B1FF0646F9F76CFD4CF64C193D
:10A3C000C2F2010900F22C414846F8F7FDFD019464
:10A3D00026444DF2B8054CF6102440F204784CF6B1
:10A3E000142AC2F2010509F1880BC2F2010409F135
:10A3F000AC07C2F2000809F1C109C2F2010A00BFAC
:10A40000A86D40F2B461C2F200010022002300F006
:10A41000F7FF4CF64C10C2F20100F8F7E7FEA86B0C
:10A42000C4F800B0C8F80070CAF8009001F0C4F891
:10A43000A86BD8F800100022002301F075F8E86A34
:10A4400001F0BAF8E86ADAF800100022002301F0FF
:10A450006BF8A86C01F0B0F8A86C2168002200230A
:10A4600001F062F8304600F029FF01980644C7E782
:10A470000000000000407F4000F058FF05F021FD83
:10A480009FED150B53EC102B05F058FB05F0ECFC81
:10A490000446002000F002FF00F03EFF40F210757D
:10A4A000C2F2000506462846F9F780FD4DF2B807CE
:10A4B0002644C2F2010700BF786D01F07DF8786D87
:10A4C00029460022002301F02FF8304600F0F6FE66
:10A4D0002644F1E700BF00BF0000000000407F40BD
:10A4E00000F024FF05F0EDFC9FED250B53EC102B45
:10A4F00005F024FB05F0B8FC8146002000F0CEFEFC
:10A5000000F00AFF0646F9F7C5FC4CF67825C2F2C2
:10A5100001059FED1D0A01462846FAF78DF94DF217
:10A52000B80440F28C7840F278774E44C2F20104CD
:10A53000C2F20008C2F2000714E000BFA06B394667
:10A540000022002300F05CFF2846FAF7EFFA2846C5
:10A550003946F9F723FF2846FAF71AFA304600F091
:10A56000ADFE4E44606B41460022002300F048FFE0
:10A570000028E3D128464146FAF768FBDEE700BF32
:10A580000000000000407F400000FA43000000008F
:10A5900000F0CCFE05F095FC9FED1B0B53EC102B4F
:10A5A00005F0CCFA05F060FC0446002000F076FED1
:10A5B00000F0B2FE0646F9F76DFC40F67878C2F27C
:10A5C00000089FED130A00F5C0714046FFF7F4F84C
:10A5D00040460121FFF794F94DF2B80541F2286792
:10A5E0002644C2F20105C2F2000700BFE86A3946FC
:10A5F0000022002300F004FF4046FFF789F93046AF
:10A6000000F05CFE2644F1E70000000000407F40BF
:10A610000000FA430000000000F088FE05F051FC45
:10A620009FED130B53EC102B05F088FA05F01CFC82
:10A630000446002000F032FE00F06EFE05460220C7
:10A6400000F07AFB4CF250162544C2F201064FF09E
:10A65000804700BF304602210022776000F014FBE3
:10A66000284600F02BFE2544F4E700BF00BF00BFE2
:10A670000000000000407F4080B5806B0021C18554
:10A68000FDF700F880BD000010B5846B20684069BC
:10A6900094F84110212907D110F0800004D0002047
:10A6A000E084204600F0C2F82068406994F8421027
:10A6B000222907D110F0400004D00020E085204678
:10A6C00000F080F8606C40F0100060642046FCF7F9
:10A6D000D9FF10BD80B50168806B0968C9052FD40A
:10A6E0000021C185016851E8031F026821F48071CF
:10A6F00042E80313002BF5D1016851E8051F0268F9
:10A7000021F0010142E80513002BF5D1016851E861
:10A71000051F026821F0400142E80513002BF5D126
:10A72000202180F84210016B012909D1016851E80C
:10A73000031F026821F0100142E80313002BF5D13A
:10A7400000214163016B012903D1818DFCF798FF42
:10A7500080BDFDF78DFA80BD80B5806B012141631E
:10A76000016B012904D1818D4908FCF789FF80BD67
:10A77000FDF792FA80BD000080B50168806B096822
:10A78000C90516D40021C184016851E8051F02687B
:10A7900021F0800142E80513002BF5D1016851E852
:10A7A000031F026841F0400142E80313002BF5D17A
:10A7B00080BDFDF7E7FA80BD80B5806BFDF7F6FA46
:10A7C00080BD0000016851E8031F026821F4907108
:10A7D00042E80313002BF5D1016851E8051F026818
:10A7E00021F0010142E80513002BF5D1016B01298D
:10A7F0000AD100BF016851E8031F026821F010016F
:10A8000042E80313002BF5D1202180F842100021EB
:10A810000163704780B50168CA6822F04002CA60CF
:10A82000202180F84110FDF7ADFA80BD016851E8A4
:10A83000031F026821F0C00142E80313002BF5D189
:10A84000202180F841107047006840F6FF71C4F283
:10A850000101884210DC44F20041C4F20001884248
:10A8600004BF0120704744F60001C4F20001884291
:10A8700004BF022070470FE041F20001C4F2010161
:10A88000884204BF0020704741F20041C4F2010138
:10A89000884204BF032070470520704780B582B00E
:10A8A00090F8421022291ED18268B2F5805F02D151
:10A8B000016900294AD0816AB2F5805F07D00AB9E0
:10A8C000026922B10268526802F07F0201E0026868
:10A8D00052680A700121826A11448162C18D013976
:10A8E0000A04C18501D002B080BD0168CA6822F0A7
:10A8F0002002CA60CA6822F48072CA604A6922F0E3
:10A9000001024A61202180F8421000214163026B5C
:10A91000012A23D1016300BF016851E8031F0268C7
:10A9200021F0100142E80313002BF5D101680A68F9
:10A93000D20606D5002201920A6801924968019167
:10A940000199818DFCF79CFE02B080BD0168826A8E
:10A9500049686FF35F2111800221BCE7FDF788F998
:10A9600002B080BD10B504460068D4E902C2236974
:10A97000016921F4405111430161626943EA0C010C
:10A98000E3691143C268194349F20C639A431143C6
:10A99000C1604169A26921F4407141F20043114351
:10A9A00040F48062C4F201039A42416102D1FBF794
:10A9B0009FFB01E0FBF78AFBE16963681922B1F5AF
:10A9C000004FA0FB02011CD15A00DB0FF5F792FCEF
:10A9D00048F21F51C5F2EB11A0FB01235A096FF099
:10A9E000630302FB0300322303EBC000A0FB010161
:10A9F0004FF4F87000EA111000EB0210C1F342119D
:10AA00001AE09A009B0FF5F775FC48F21F51C5F24A
:10AA1000EB11A0FB01235A096FF0630302FB030053
:10AA2000322303EB0010A0FB0101F02000EA5110DB
:10AA300000EB0210C1F3431122680843906010BD7F
:10AA4000F0B581B0134600270446816283854764D0
:10AA5000222084F84200E06B4AF2D5654AF259762A
:10AA60000A462168C0F60005C0F60006C0E90F5688
:10AA70004AF28966C0F600060431C0E91367FAF7A6
:10AA80005BFF38B110206064202084F84200012070
:10AA900001B0F0BD00972068016800914068009007
:10AAA0000098206950B100BF206850E8030F21686A
:10AAB00040F4807041E80302002AF5D1206850E894
:10AAC000050F216840F0010041E80502002AF5D198
:10AAD000206850E8050F216840F0400041E8050279
:10AAE000002AF5D1002001B0F0BD000090F841101F
:10AAF000212923D18168B1F5805F01D1016931B18C
:10AB0000016A02684B1C03620978516007E0016A20
:10AB1000036831F8022B6FF35F225A600162C18C27
:10AB200001390A04C18418BF70470068C16821F068
:10AB30008001C160C16841F04001C1607047000000
:10AB400010B54CF67874C2F201042046FCF7AEFD55
:10AB50002046F7F751FF10BD10B54CF6C074C2F295
:10AB600001042046FCF7A2FD2046F7F745FF10BD83
:10AB700010B540F60824C2F200042046FCF796FD0A
:10AB80002046F7F739FF10BDFEE700002DE9F04F32
:10AB900083B08B4601393F2942D84DF61444BBF1AE
:10ABA000000FC2F20104029228D0061F4FF00008E5
:10ABB0004FF0000940F6BC4740F60C50C0F60107C4
:10ABC000C0F60100B8F1000F08BF074656F8040FA1
:10ABD00004EB090AC9F5827505F06AFD41EC100B1A
:10ABE0005046294610A23B468DED000BF5F710FCB0
:10ABF00008F10108C3458144DCD101E04FF00009B0
:10AC000004EB0900C9F5827109A2F5F701FC2046A1
:10AC1000F5F726FD029B82B200202146F7F724FFBC
:10AC200003B0BDE8F08F00BF2573252E326600000B
:10AC30000A00000070B50D4601393F2988BF70BD7C
:10AC40004DF61446C2F2010614460146AA003046EB
:10AC5000F5F76AFD4FF0FF4046F82500042000EBB1
:10AC60008502002031462346F7F7FEFE70BD000046
:10AC7000B0B50C460546F5F7F3FC82B20020294634
:10AC80002346F7F7F1FEB0BDF0B5C1B0144640F26F
:10AC90000402C2F2000212780F46022A054627D0AB
:10ACA000012A2CD092BB0FB3286805F001FD01AE3C
:10ACB00002460B4617A13046F5F794FB012F0CD046
:10ACC0003046F5F7CDFC3718686805F0F1FC024610
:10ACD0000B4614A13846F5F785FB3046F5F7C0FC66
:10ACE0000A21315230462146FFF7C2FF00200EE014
:10ACF000284639462246FFF79DFF002007E02846F8
:10AD000039462246FFF742FF002000E0FF2040B214
:10AD100041B0F0BD4368616E6E656C313A20252EFE
:10AD2000326600002C204368616E6E656C323A20FA
:10AD3000252E32660000000040F204020146C2F2F5
:10AD4000000200201170704700F0FF40B0F1FF409A
:10AD500018BF01207047000000F0FF40B0F1FF4035
:10AD600018BF01207047000020F00040A0F1FF4014
:10AD7000B0FA80F040097047002848BF704700F0E3
:10AD80001F01012202FA01F14EF280124009CEF2B7
:10AD9000000242F82010BFF34F8FBFF36F8F704750
:10ADA000002848BF704700F01F01012202FA01F19C
:10ADB0004EF200124009CEF2000242F82010704715
:10ADC0004EF60C50CEF200000068C0F3022070472F
:10ADD0004EF6145300F00F02CEF2000309011A449C
:10ADE00000F16043B0F1FF3FC8BF03F5644211704A
:10ADF000704700004EF61F50CEF200000021017097
:10AE0000704700004EF60C51CEF200010A684FF672
:10AE1000FF031A4060F30A2242F0806040F0FD70A8
:10AE20000860704770B52DED048B044600284FF084
:10AE3000FF0018BF002900F01481B5EE400AB0EE03
:10AE4000408AF1EE10FA40F30C810320C4F8041696
:10AE50002076D1F8600104F2FC55C5F8E801D1F87C
:10AE60006401C5F8EC01F7F753F94FF4847600BF9D
:10AE7000D4F804063044FDF7CFFB0836B6F5947FCE
:10AE8000F6D14FF4947600BFD4F804063044FDF7B1
:10AE9000C3FB0836B6F5A47FF6D14FF4A87600BF01
:10AEA000D4F804063044FDF7B7FB0836B6F5AC7F9E
:10AEB000F6D042F6CC7047F2AC21C4F2A600C3F63D
:10AEC000C171C5E9001040F6AC30C0F6010090E851
:10AED0000E00C06804F2BC450026C4F8EC15C4F8A6
:10AEE000F025C4F8F435C4F8F80500BFD4F804160A
:10AEF000A81901F1C8020021B0EE480AFEF766F970
:10AF00003C36F02EF2D10025D4F80416661906F569
:10AF1000737001F188020121B0EE480AFEF756F97C
:10AF2000D4F8041606F5377001F1A8020121B0EE3D
:10AF3000480AFEF74BF93C35F02DE5D1D4F804165C
:10AF400004F2AC5001F1E8020121B0EE480A04F528
:10AF5000F675FEF73BF94826D4F80406012182195C
:10AF60002846B0EE480AFEF731F9D4F8041605F188
:10AF700078003144A1F140020121B0EE480AFEF709
:10AF800025F92036682E05F13C05E5D0B3EE049A8C
:10AF900004F5C160B0EE480AF0EE490AFCF78CFFF8
:10AFA00004F5C560B0EE480AF0EE490AFCF784FFEC
:10AFB00004F5C960B0EE480AF0EE490AFCF77CFFE0
:10AFC00004F5CD60B0EE480AF0EE490AFCF774FFD4
:10AFD00004F5D160B0EE480AF0EE490AFCF76CFFC8
:10AFE00004F5D560B0EE480AF0EE490AFCF764FFBC
:10AFF00004F5D960B0EE480AF0EE490AFCF75CFFB0
:10B0000004F5DD60B0EE480AF0EE490AFCF754FFA3
:10B0100004F5E160B0EE480AF0EE490AFCF74CFF97
:10B0200004F5E560B0EE480AF0EE490AFCF744FF8B
:10B0300004F5E960B0EE480AF0EE490AFCF73CFF7F
:10B04000DFED0A0A04F5ED60B0EE480AFCF734FFC4
:10B05000DFED070A04F5F160B0EE480AFCF72CFFBB
:10B06000002040B2BDEC048B70BD00BF0000484220
:10B070000000C8427047000040F6DB7110EE100A75
:10B08000C3F6C97161F31E0000EE100A704700009C
:10B09000F0B581B0F0B104464DF2A400C2F2010057
:10B0A0000068A0421FD001F06BFA40F60C30C2F2EB
:10B0B0000000656907684DF2B000C2F20100066841
:10B0C00001F082FABD424FF0020018BFB5420DD127
:10B0D00001B0F0BD4FF0500080F31188BFF36F8FC7
:10B0E000BFF34F8FFEE7002001B0F0BD4DF6985042
:10B0F000C2F2010085420CD04BF29C210120C2F229
:10B100000101002D08BF04208D4208BF042001B0BA
:10B11000F0BDA06A10B1022001B0F0BD94F85C103F
:10B120000320012908BF022001B0F0BD4FF0FF311C
:10B1300001FA00F0C04302EE100A30EE600AB8EEE9
:10B14000C22A31EE601A20EE020A80EE010ABDEE3C
:10B15000C00A10EE100A704700207047FAF77CFE14
:10B16000FEF7F8FCFDF708FCFDF7A2FBFDF75CFB22
:10B17000FDF77CFBFDF702FDFDF720FDFDF73EFD31
:10B18000FDF72EFEFDF748FEFDF762FEFDF75EFDC2
:10B19000FDF780FEFDF79EFD00F0CCF8FDF7CEFB3D
:10B1A00000F0F2F8FEE700000146C068B6EE002AA3
:10B1B00090ED4C1A90ED4B0A21EE021A30EE010A86
:10B1C000002081ED130A704730EE600A32EE612AEA
:10B1D00020EE020A31EE601A80EE010A30EE210AFA
:10B1E000704700004DF24801C2F2010101EB8001FD
:10B1F00091ED001A9FED152A30EE411A81ED000AFB
:10B20000B4EE421A40F66421F1EE10FAC2F20001E7
:10B2100002DD4FF0FF3207E09FED0D2AB4EE421A37
:10B22000F1EE10FA05DA012251F820301A4441F803
:10B23000202001EB800090ED001A9FED062AB8EE69
:10B24000C11A21EE021A31EE000A7047DB0F4940A5
:10B25000DB0F49C0DB0FC940401A811000EE101A05
:10B260009FED0B1AB8EEC00A30EE011A9FED0A2AC4
:10B270000C28C8BFB0EE410A9FED061AB4EE420A90
:10B2800030EE011AF1EE10FAB8BFB0EE410A704785
:10B29000DB0FC9C0DB0FC940DB0F49C0EFF30581ED
:10B2A00000291CBF6FF005007047002804BF002074
:10B2B000704780B501F068FA002080BD10B582B0FB
:10B2C000EFF3058119B16FF0050002B010BD04461F
:10B2D00002F072FB211A0129019005DB01A801F09F
:10B2E0007DFA002002B010BD6FF0030002B010BD67
:10B2F00080B502F04DFB022808BF80BD08B90320CD
:10B3000080BD40F2F450C2F2000000680138B0FA8B
:10B3100080F0400980BD000080B5EFF3058010B1DA
:10B3200002F050FB80BD02F047FB80BD4FF47A7005
:10B3300070470000EFF3058000281CBF6FF0050088
:10B34000704740F2F450C2F200000168002911BFBA
:10B350004FF0FF30012101600020704780B5EFF30E
:10B36000058000281CBF6FF0050080BD02F010FBB7
:10B3700028B1022805D101F0DDFB002080BD0120AD
:10B3800080BD4FF0FF3080BD10B5EFF30580002881
:10B390001CBF6FF0050010BD40F2F454C2F200046F
:10B3A000206801281CBF4FF0FF3010BDFEF7C2F926
:10B3B0000220206001F06AFB002010BD10B5EFF301
:10B3C000058018B16FF00504204610BD02F0E0FAC8
:10B3D00002280ED080B902F0CDFC01284FF0010404
:10B3E0000CD002F0D5FA002808BF4FF0FF342046F9
:10B3F00010BD0024204610BD4FF0FF34204610BD84
:10B4000010B582B01C46B0FA80F3B1FA81F25B0944
:10B410005209EFF3058CBCF1000F42EA030219D088
:10B42000002C18BF0124224315D10022019201AA49
:10B4300001F088FF01281AD10198A8B14EF60450F6
:10B44000CEF200004FF080510160BFF34F8FBFF389
:10B450006F8F09E01AB16FF0030002B010BD2246F1
:10B4600001F0AEFE012806D1002002B010BD6FF041
:10B47000020002B010BD6FF00100002C08BF6FF099
:10B48000020002B010BD0000B0B582B01446002921
:10B490004FF00005EFF3058218BF002802D12846BF
:10B4A00002B0B0BD002AFAD19CB1A568D5B1E2685E
:10B4B000502A16D32269A2B1D4F814C001FB00F2BD
:10B4C000002394454FF0000228BF012210D24DB155
:10B4D0000EE0012300226AB9E3B1002201F064FC0E
:10B4E0000EE01DB9E2680AB92269C2B10022002348
:10B4F000002AF1D0A36822690025009501F078FCAC
:10B50000054655B1002C14BF21680021284601F0E2
:10B5100005F9C4E70025002DF4D10025BFE76269D5
:10B52000B2FA82F25309D5E7B0B582B01C46B0FA40
:10B5300080F3B1FA81F5EFF305825B096D09002A0A
:10B5400043EA050207D0002C18BF0124224306D08D
:10B550006FF003052CE0CAB16FF0030528E000226C
:10B56000019201AA002301F0A1FD01281CD101983C
:10B57000E8B14EF60450CEF200004FF08051016069
:10B58000BFF34F8FBFF36F8F002511E022460023DA
:10B59000002501F0B9FC01280AD06FF00105002C4C
:10B5A00008BF6FF0020503E06FF0020500E0002520
:10B5B000284602B0B0BD000010B5EFF3058119B107
:10B5C0006FF00504204610BD00280FBF6FF0030484
:10B5D0000021002401F058FC204610BD10B50C4697
:10B5E000EFF3058100291CBF6FF0050010BD014677
:10B5F00020F0010050B111F001010AD1214601F003
:10B60000F7FE012804BF002010BD09E06FF0030021
:10B6100010BD214601F0D0FF012804BF002010BD5D
:10B620006FF00100002C08BF6FF0020010BD000099
:10B6300070B5EFF30581B9B90028044614BF6068FE
:10B640000020010710D494B1A36843B1E26800213F
:10B650004F2A4FF0000288BF01220AD84BB9E16897
:10B66000B1FA81F1490903E00025284670BD0121A6
:10B67000002200F001063AB1A168002E0CBF0120A3
:10B68000042001F07FFB06E0C9B1002E0CBF0120B1
:10B69000042001F06BFB054635B1002C14BF216876
:10B6A0000021284601F03AF8B5FA85F0400986F005
:10B6B0000101084308BF45F00105284670BD00257B
:10B6C000002DEAD1F0E7000080B5EFF305810029F5
:10B6D0001CBF6FF0050080BD014620F0010040B1A5
:10B6E00011F0010108D100210022002301F00CFC1F
:10B6F00004E06FF0030080BD01F040FD013818BF89
:10B700006FF0020080BD0000B0B584B048B3B1F165
:10B71000FF3F26DD04464FF0FF300390EFF3058036
:10B7200018B300250DF1080C2046012200230295D4
:10B73000CDF800C002F090F803AB204600210022B3
:10B74000009502F089F80298D0B14EF60450CEF27E
:10B7500000004FF080510160BFF34F8FBFF36F8F38
:10B760000EE06FF0030003900AE020460122002360
:10B7700001F0F4FF03AB20460021002201F0EEFFB0
:10B78000039804B0B0BD00002DE9F04F83B00C4623
:10B79000EFF3058129B16FF00507384603B0BDE826
:10B7A000F08F0546002849D44FF0000B9246A007C1
:10B7B00058BFAB4602F000F900906FF0010804F0AA
:10B7C000010054460027BAF1000F08BF6FF00208CD
:10B7D000019002E04746002EDFD00020594602AA21
:10B7E000234602F0A3F906460128F3D1029807EA9E
:10B7F000050140EA01090198002809EA050007D17E
:10B8000000286FF0020718BF4F4607D0C5E700BFFA
:10B81000A8426FF0020708BF4F46BED0BAF1000F32
:10B82000BBD002F0C9F800994F46401A241A4FF0D5
:10B83000000038BF0446002ECFD1AEE76FF00307FB
:10B84000ABE7000080B502F09DF880BD70B584B014
:10B850008E46002100280391EFF3058146D0002990
:10B8600044D1FAB19369002B08BF1823382B16D89E
:10B870001179C90713D15569946811684FEA950C7D
:10B88000002D08BF4FF0800CFCB1D668602E1BD392
:10B89000D5B11569C5B10024012555B91BE00020BB
:10B8A00004B070BD0124002118234FF0800C002546
:10B8B0008DB1946812690294CDE9003262467346F4
:10B8C00001F010FF039011E00CB9D4689CB1002581
:10B8D0000024002DEDD14CB103AC00931FFA8CF283
:10B8E0007346019401F0CAFE012802D1039804B006
:10B8F00070BD0020E6E71469B4FA84F46409D6E761
:10B9000010B5EFF3058100291CBF6FF0050010BDD5
:10B91000044660B12046FFF7BBFB042804BF6FF06C
:10B92000020010BD204600F0ADFF002010BD6FF0FA
:10B93000030010BDF0B581B00D464DF6AC514DF28F
:10B94000A406C2F20101C2F201060F683168044682
:10B95000081D00F09FFD601C0AD14DB13068011D2B
:10B960004DF69850C2F2010000F0F2FD01B0F0BDBA
:10B970003068E41944600AD34DF2B000C2F201000D
:10B9800000683168043100F0C5FD01B0F0BD40F63B
:10B990000C30C2F2000000683168043100F0BAFDDA
:10B9A0004BF27420C2F2010001688C4238BF04607F
:10B9B00001B0F0BD70B5044600F0E2FD4AF6D87063
:10B9C000C2F2010001684DF2A40501310160C2F22A
:10B9D000010529684DF69456C2F2010641B130685E
:10B9E00060B92868E16AC06A884298BF2C6005E0A7
:10B9F0002C600068012801D100F0E0F94AF6E070FF
:10BA0000C2F2010001680131016061644AF6E4712B
:10BA1000C2F20101E06A0A68904288BF086040F6FD
:10BA2000143100EB8000C2F2000101EB8000211D07
:10BA300000F08EFD00F0C8FD306880B12868E16A32
:10BA4000C06A884228BF70BD4EF60450CEF2000096
:10BA50004FF080510160BFF34F8FBFF36F8F70BD08
:10BA600070B582B000F08CFD4DF6B056C2F2010602
:10BA7000306850BB4DF61854C2F20104204600F065
:10BA800039FD4BF24825C2F20105284600F032FD8F
:10BA90004DF2A800C2F20100046040F61030C2F27C
:10BAA000000040F66C224DF2500305600025C2F202
:10BAB0000002C2F201030A201021009501F098F95A
:10BAC000306010B103A100F029FE00F07DFD02B04E
:10BAD00070BD00BF546D725100000000F0B581B020
:10BAE0004DF6B015C2F201052868E0B14BF29C2674
:10BAF0004AF6D877C2F20106C2F2010700F040FD13
:10BB0000F068C468201D00F0C5FC38680138386052
:10BB100028680138286000F057FD204600F058F8EA
:10BB200028680028EAD101B0F0BD000080B5026CA1
:10BB3000002A08BF80BDD0E902C31344C360634537
:10BB400024BF0368C360C36808461946F4F7A7FD1D
:10BB500080BD000070B5866B036C0446E3B11546EA
:10BB60001AB3E0681A46F4F79AFDE168206C22687F
:10BB7000091A9142E16003D2A16840420844E060A2
:10BB8000A81EB0FA80F040093146002E18BF0121EE
:10BB90000840361A002516E02068002598B9A068EC
:10BBA00002F00CF8A56005460DE060681A46F4F74F
:10BBB00076FD216CD4E901020025084460609042C2
:10BBC00024BF20686060711C2846A16370BD00001E
:10BBD00010B5044690F85D00022808BF10BD01288A
:10BBE00003D030B9206B00F007FD204600F004FDC3
:10BBF00010BD4FF0500080F31188BFF36F8FBFF37B
:10BC00004F8F00BFFEE70000416A00290FBF0020F0
:10BC1000006B0068C0F13800704700004DF2A801C9
:10BC2000C2F2010109680A68B2FA82F35B09036093
:10BC3000002A0EBF0020C8680068704741F23460D7
:10BC4000C2F20000C21D22F0070210F0070CA0EBA8
:10BC5000020318BF10464BF29422C2F201020021E7
:10BC6000C2E9000149F69912C0F20102BCF1000FCD
:10BC700018BF1A440244083A4DF2AC0322F00702FE
:10BC8000C2F201031A60C2E90011111A1A68C0E970
:10BC900000214DF64850C2F2010001604BF27020C5
:10BCA000C2F2010001604DF62C50C2F201000121E8
:10BCB0000170704740F614344EF60455C2F2000489
:10BCC000CEF200054FF08056FFF708FF20680228EB
:10BCD000FAD32E60BFF34F8FBFF36F8FF4E70000EE
:10BCE000002808BF704780B500210160C0E902113B
:10BCF00000210022002301F007F9BDE880407047D1
:10BD0000B0B5049D002914BF2A602D60C5E90F015C
:10BD1000284601211C4601F0B7F885F84C40B0BD1B
:10BD20002DE9F0470A9C8246206B16460F46DDE956
:10BD300008599100A5229846F4F728FD206B00EBE6
:10BD40008600A0F1040020F007067FB104F1340062
:10BD5000002100BF7A5C42547A5C1AB10F2901F1CC
:10BD60000101F7D3002084F8430002E0002084F8AA
:10BD700034000027201D372D28BF3725E562C4E990
:10BD8000135700F0C3FB04F1180000F0BFFBC5F12E
:10BD90003800A061304651464246246164626765BE
:10BDA000A76584F85C7000F04BFBB9F1000F2060D0
:10BDB00018BFC9F80040BDE8F0870000B0B540F6F4
:10BDC00014350024C2F20005281900F093FB143446
:10BDD000B4F58C6FF8D14DF63054C2F20104204610
:10BDE00000F088FB4BF25C25C2F20105284600F00A
:10BDF00081FB4BF28020C2F2010000F07BFB4BF292
:10BE00009C20C2F2010000F075FB4DF69850C2F282
:10BE1000010000F06FFB40F60C30C2F2000004603D
:10BE20004DF2B000C2F201000560B0BD80B54BF22A
:10BE30009422C2F2010200BF114612688242FBD373
:10BE4000D1F804C001EB0C03834203D14068604485
:10BE500048600846D0F804C000EB0C03934201D0C0
:10BE600013460BE04DF2AC03C2F201031B689A4289
:10BE700004D0D2E9003E0EEB0C0242608142036026
:10BE800018BF086080BD000080B58C46014641F8AF
:10BE900004CF9445006108D99A4201D29C4511D241
:10BEA0004DF2A800C2F2010007E08069D21A824276
:10BEB00008D240F61030C2F20000006800F02AFB01
:10BEC000002080BD012080BD10B5044600F058FB65
:10BED000A06BB0FA80F0440900F076FB204610BD5C
:10BEE00010B5044600F04CFBA06BE16B401AB0FAB1
:10BEF00080F0440900F068FB204610BD0848006847
:10BF0000006880F308884FF0000080F3148862B660
:10BF100061B6BFF34F8FBFF36F8F00DF00BF00BF6D
:10BF200008ED00E070B582B04DF2A802C2F2010245
:10BF300012680546D2680E46D468201D00F0AAFAA1
:10BF400094F82800410704D400F0FE0084F828008B
:10BF500010E0A0693246411920462B46FFF794FFB6
:10BF600040B10026204600212A460023009601F019
:10BF7000C5FF20B1216A2046884702B070BD4FF04E
:10BF8000500080F31188BFF36F8FBFF34F8F00BF56
:10BF9000FEE700002DE9F04186B04DF6B057C2F241
:10BFA0000107386802A900224FF0000801F008F9E3
:10BFB00000286AD001AC02AD0BE000F0FE0086F86C
:10BFC000280000BF38682946002201F0F9F800284F
:10BFD0005BD00298B0F1FF3F03DCDDE90320059957
:10BFE000904702980028EDD4049E706910B1301D6E
:10BFF00000F050FA204600F0B3F802990929E1D880
:10C000000246DFE801F0080808052A390808052A71
:10C0100096F82800D1E796F82800039BB16940F014
:10C02000010086F8280019443046FFF72DFF00284C
:10C03000C8D0316A3046884796F828004007C1D5F5
:10C040000398B16900230A1830460021CDF800801A
:10C0500001F054FF0028B5D123E096F8280040F005
:10C060000101039886F82810B06188B18118304624
:10C070001346FFF709FFA5E796F8280081073FF56B
:10C080009CAF304600F0B8FA9CE706B0BDE8F081FE
:10C090004FF0500080F31188BFF36F8FBFF34F8FC5
:10C0A000FEE74FF0500080F31188BFF36F8FBFF3AE
:10C0B0004F8F00BFFEE7000070B582B00E46044609
:10C0C00000F038FD01A800F04BF8019919B101F01A
:10C0D00051FE02B070BD05464EB9A54207D301F02E
:10C0E00049FE20462946FFF71DFF02B070BD4EB144
:10C0F00040F61030C2F2000000680068B0FA80F02C
:10C10000420900E000224DF6B050C2F20100006882
:10C11000611B00F017FB01F02DFE0028D9D14EF66F
:10C120000450CEF200004FF080510160BFF34F8FFA
:10C13000BFF36F8F02B070BD40F60C30C2F200004A
:10C140000168096821B10068C068C068406801E002
:10C150004FF0FF304BF27421C2F2010108607047CA
:10C1600070B5044601F028FC4DF2A006C2F20106AB
:10C1700031680546884203D200F008F8012000E04B
:10C18000002020602846356070BD00002DE9F04198
:10C1900082B04DF2A807C2F201073868016891B376
:10C1A0004FF0000809E000BF60603868294624614C
:10C1B00000F0B0F93868016829B3C068C46806683F
:10C1C000251D284600F066F9216A2046884794F824
:10C1D00028004007EED5A0693044B042E4D820469C
:10C1E000002132460023CDF8008001F087FE0028B0
:10C1F000E0D14FF0500080F31188BFF36F8FBFF391
:10C200004F8F00BFFEE740F61031C2F200010A680E
:10C2100008603A6002B0BDE8F081000081B0002003
:10C2200000904CF21400C2F2010000684FF050017F
:10C2300081F31188BFF36F8FBFF34F8F013001D0AF
:10C24000FEE700BF00980028FCD001B07047000056
:10C2500082B001AC2046FFF7E1FC0199FFF72CFF0B
:10C26000FFF798FEF6E70000F0B581B0044600F055
:10C2700087F994F94560012E0FDB04F1240500BF16
:10C28000286850B1284601F02DFD002818BF00F0A5
:10C2900069FB70B2013E0128F2DCFF2684F845609C
:10C2A00000F092F900F06CF994F94470012F0EDB64
:10C2B00004F11005286850B1284601F013FD00284C
:10C2C00018BF00F04FFB78B2013F0128F2DC84F880
:10C2D000446000F079F901B0F0BD00002DE9F043B1
:10C2E00081B0044600F026FC4DF2AC06C2F2010615
:10C2F0003068002808BFFFF7A1FC4DF62C58C2F2A9
:10C30000010898F80000002818BF4FF000402042B4
:10C310000DD0002401F02EFD60071ED04FF050001C
:10C3200080F31188BFF36F8FBFF34F8FFEE7C4B167
:10C3300014F0070004F108011EBF081A00F10801FB
:10C340005FEA41700ED04FF0500080F31188BFF3C8
:10C350006F8FBFF34F8F00BFFEE7204601B0BDE8EF
:10C36000F08300214BF27029C2F20109D9F80000D4
:10C370004A1E8242CDD24BF29420C2F201000568DF
:10C380002F4657F8042F8A4211D22B685BB100BFA9
:10C390001F4657F8042F28461D468A4207D22B68AD
:10C3A000002BF5D103E04BF29420C2F20100336878
:10C3B0009D42AED004682B68521A112A036010D334
:10C3C0006818430709D04FF0500080F31188BFF37D
:10C3D0006F8FBFF34F8F00BFFEE742603960FFF7FA
:10C3E00025FD4DF648503968D9F80020C2F2010009
:10C3F0000368511A9942C9F8001038BF016098F8D3
:10C400000000396800284FF0000018BF41F00041DB
:10C4100028604BF27820C2F20100026808343960CB
:10C42000511C016076E700004DF2A400C2F2010049
:10C43000016819B101680A6D01320A650068704728
:10C4400003464CF21D20C0F600004FF0807C21F026
:10C45000010103E903106FF0020043F8240CA3F17B
:10C46000440043F8202C704702EE100A4FF0FF30D2
:10C47000884030EEC01AB8EEC22AC04321EE021A3C
:10C4800002EE100AB8EEC22A81EE021A31EE000A5C
:10C4900070470000D0E9013201699A60D1F804C008
:10C4A00082688445536008BF4A60002202610868C0
:10C4B00001380860086870474AF6E873C2F2010361
:10C4C00003604DF6B410C2F20100086080201060D5
:10C4D000704700004DF6B433C2F2010303604BF223
:10C4E0004800C2F201000860802010607047000020
:10C4F000704700004FF0FF31024642F8081F00214C
:10C500004260C0E903220160704700000021016120
:10C510007047000080B5D1F800C01CF1010207D0BF
:10C5200000F108039E465B681A686245FAD901E08B
:10C53000D0F810E0DEF8042008614A609160C1F88C
:10C5400008E0CEF8041001680131016080BD0000F0
:10C55000D0F800C0436808619A684B608A609A68A6
:10C56000996051600CF1010101607047DFF80C0027
:10C57000016841F470010160704700BF88ED00E080
:10C580004FF0500080F31188BFF36F8FBFF34F8FD0
:10C590004CF21400C2F2010001684A1C026001B1B1
:10C5A00070474EF60450CEF200000068000608BF47
:10C5B00070474FF0500080F31188BFF36F8FBFF3C7
:10C5C0004F8F00BFFEE700004CF21400C2F20100E2
:10C5D000016839B10139016018BF7047002080F34C
:10C5E000118870474FF0500080F31188BFF36F8FB0
:10C5F000BFF34F8FFEE70000B0B5002808BFB0BD05
:10C6000004464DF62C50C2F20100007854F8041C88
:10C61000002818BF4FF0004008420CD0A4F10805D4
:10C620002A6892B14FF0500080F31188BFF36F8FEA
:10C63000BFF34F8FFEE74FF0500080F31188BFF338
:10C640006F8FBFF34F8F00BFFEE721EA000044F871
:10C65000040C00F06FFA4BF27021C2F2010154F8A1
:10C66000040C0A68104408602846FFF7DFFB4DF60B
:10C670005050C2F2010001680131016001F07AFB03
:10C68000B0BD00004EF21000CEF2000000210160AB
:10C69000816040F20001C2F20001096844F6D35201
:10C6A000C1F26202A1FB02124FF0FF3101EB9211C5
:10C6B0004160072101607047EFF30580102814D313
:10C6C0004EF2F031CEF20001405C4AF6CD71C2F27A
:10C6D00001010978884208D24FF0500080F3118898
:10C6E000BFF36F8FBFF34F8FFEE74EF60C50CEF2C5
:10C6F00000004AF6D0710068C2F20101096800F436
:10C70000E060884298BF70474FF0500080F3118876
:10C71000BFF36F8FBFF34F8FFEE700004DF6545C01
:10C720000022C2F2010C00BF5CF8323023B10132AA
:10C73000082A08BF7047F7E70CEBC2034CF8321029
:10C740005860704770B515460E460446FFF718FF4F
:10C7500094F84400FF2804BF002084F8440094F8B3
:10C760004500FF2804BF002084F84500FFF72CFF98
:10C77000A06B28B904F1240031462A4600F014F9D0
:10C780002046FFF771FD70BD10B5D8B104464AF6DA
:10C79000DC70C2F20100006848B14FF0500080F335
:10C7A0001188BFF36F8FBFF34F8F00BFFEE700F01C
:10C7B000C1F920460021FFF7BDF801F0DBFA00289F
:10C7C00018BF10BD4EF60450CEF200004FF080515D
:10C7D0000160BFF34F8FBFF36F8F10BDB0B590B145
:10C7E0000D46D1B104464AF6DC70C2F20100006881
:10C7F000E8B14FF0500080F31188BFF36F8FBFF3A3
:10C800004F8F00BFFEE74FF0500080F31188BFF359
:10C810006F8FBFF34F8F00BFFEE74FF0500080F3E4
:10C820001188BFF36F8FBFF34F8F00BFFEE700F09B
:10C8300081F94DF6AC50C2F20100006822689042C6
:10C8400002EB050102D2914202D309E0914201D3E9
:10C85000814205D92160081A0021FFF76BF800E03A
:10C86000216001F087FA002818BFB0BD4EF60450D1
:10C87000CEF200004FF080510160BFF34F8FBFF345
:10C880006F8FB0BD70B50446FFF77AFE4DF2A40677
:10C89000002CC2F2010608BF3468251D2846FFF7A8
:10C8A000F9FDA06A18B104F11800FFF7F3FD4AF68C
:10C8B000E070C2F201000168013101603068844219
:10C8C0000CD04AF6D870C2F201000168013901604B
:10C8D0002046FFF77DF9FFF72FFC0DE04BF29C207F
:10C8E000C2F201002946FFF733FE4DF6B010C2F246
:10C8F0000100016801310160FFF766FE4DF69450BA
:10C90000C2F201000068E8B13068844218BF70BD0F
:10C910004AF6DC70C2F20100006840B14FF05000EE
:10C9200080F31188BFF36F8FBFF34F8FFEE74EF692
:10C930000450CEF200004FF080510160BFF34F8FE2
:10C94000BFF36F8F70BD00004DF64C51C2F2010174
:10C95000096801604DF6AC51C2F2010109684160FD
:10C96000704700004DF6B450C2F201000121016091
:10C970007047000010B568B10C464DF2A401C2F238
:10C98000010109681831FFF7C5FD20460121FEF7B6
:10C99000D1FF10BD4FF0500080F31188BFF36F8FAF
:10C9A000BFF34F8FFEE70000B0B590B10D464DF2DA
:10C9B000A401C2F20101096814461831FFF7C8FD4D
:10C9C000002C18BF4FF0FF3528462146FEF7B2FF76
:10C9D000B0BD4FF0500080F31188BFF36F8FBFF3ED
:10C9E0004F8F00BFFEE7000070B528B3026D04460C
:10C9F0001AB3E06C884238BF0846012A1CD1E16AAC
:10CA0000814208BF70BD4DF2A402C2F20102126859
:10CA1000A2421CD0A269E062002A5CBFC0F13800CB
:10CA2000A06140F61436606901EB8101C2F2000694
:10CA300006EB8101884214D070BD4FF0500080F3A6
:10CA40001188BFF36F8FBFF34F8F00BFFEE74FF02A
:10CA5000500080F31188BFF36F8FBFF34F8F00BF7B
:10CA6000FEE7251D2846FFF715FD4AF6E471C2F2E0
:10CA70000101E06A0A68904288BF086000EB80000C
:10CA800006EB80002946FFF763FD70BD10B586B048
:10CA9000002405A804A903AACDE90444FFF70CFD6E
:10CAA000DDE9032005990023CDE901014BF6B540EE
:10CAB000C0F600001DA1009400F014FE4DF6445194
:10CAC000C2F20101086010B101F0DEF90446601CF9
:10CAD00022D0012C1ED14FF0500080F31188BFF3FB
:10CAE0006F8FBFF34F8F4BF27420C2F201004FF0F3
:10CAF000FF3101604DF69450C2F201000121016046
:10CB00004DF6AC50C2F2010000210160FEF7B2FA0E
:10CB100000F08AF806B010BD4FF0500080F3118885
:10CB2000BFF36F8FBFF34F8FFEE700BF49444C4503
:10CB3000000000004AF6DC70C2F201000168013119
:10CB400001607047B0B54AF6DC70C2F201000068BF
:10CB500030B14DF6B450C2F2010001210160B0BD08
:10CB60004DF6B450C2F2010000210160FEF7F4FA64
:10CB70004AF6D471C2F201010A684DF2A40590424E
:10CB8000C2F2010504D92B68821A5C6D22445A65F1
:10CB900008602868006B0168B1F1A53F0BD14168BE
:10CBA000B1F1A53F07D18168B1F1A53F03D1C068BC
:10CBB000B0F1A53F04D0286829683431FFF798FC0C
:10CBC0004AF6E470C2F20100016840F6143201EB4B
:10CBD0008103C2F2000252F823404CB902EB8303F6
:10CBE000143B00BFB1B153F814490139002CF9D0FE
:10CBF00001EB810302EB830252F8043F5B68141DD2
:10CC0000A342136001D15B6813601268D2682A6086
:10CC10000160B0BD4FF0500080F31188BFF36F8FFB
:10CC2000BFF34F8FFEE7000080B582B04EF20040A8
:10CC3000CEF200004CF27021C4F20F11D0F800299E
:10CC40004B1C9A4209D14FF0500080F31188BFF37A
:10CC50006F8FBFF34F8F00BFFEE7D0F800298A42E5
:10CC600009D14FF0500080F31188BFF36F8FBFF3ED
:10CC70004F8F00BFFEE701784AF6CD720191FF2188
:10CC800001700178C2F201028DF803109DF80310C3
:10CC900001F0500111704AF6D071C2F20101072271
:10CCA0000A609DF90320B2F1FF3F0CDC0A6800BF67
:10CCB0009DF80330013A5B008DF803309DF9033095
:10CCC000002BF5D40A600A68032A2DD14FF4E063E3
:10CCD00003EA02220A6001990170D0F8201941F498
:10CCE0007001C0F82019D0F8201941F07041C0F847
:10CCF0002019FFF7C7FC4CF21400C2F2010000211A
:10CD00000160FFF733FC4EF63470CEF2000001688C
:10CD100041F040410160FFF7F1F8FFF713FFFFF723
:10CD20007DFA002002B080BD4FF0500080F31188E2
:10CD3000BFF36F8FBFF34F8FFEE7000080B54FF05A
:10CD4000500080F31188BFF36F8FBFF34F8F00F057
:10CD500043FE30B14EF60450CEF200004FF0805149
:10CD60000160002080F3118880BD000010B50246EC
:10CD70000120002100F018F80446FEF7B1FF20461C
:10CD800010BD000010B582B00B4684460120002182
:10CD90000022CDF800C000F02BF80446FEF7A0FFFB
:10CDA000204602B010BD0000F0B581B0B0B105461C
:10CDB0004843503014460E46FFF790FA074650B1EC
:10CDC000002007F1500287F84600284631462346E6
:10CDD0000097FEF795FF384601B0F0BD4FF05000C8
:10CDE00080F31188BFF36F8FBFF34F8FFEE7000012
:10CDF000B0B582B068B11D46ABB1F1B9EAB14FF040
:10CE0000500080F31188BFF36F8FBFF34F8F00BFC7
:10CE1000FEE74FF0500080F31188BFF36F8FBFF330
:10CE20004F8F00BFFEE74FF0500080F31188BFF333
:10CE30006F8FBFF34F8F00BFFEE751B14AB94FF07C
:10CE4000500080F31188BFF36F8FBFF34F8F00BF87
:10CE5000FEE750230193019B502B0AD1069B019CB6
:10CE6000012485F846400095FEF74AFF284602B0A7
:10CE7000B0BD4FF0500080F31188BFF36F8FBFF348
:10CE80004F8F00BFFEE7000070B5F8B104460E46B4
:10CE9000FFF776FB2068D4E90F12002502FB01039F
:10CEA000013901FB0201A563C4E90103FF20E16030
:10CEB00084F8440084F8450004F110007EB1FFF7C7
:10CEC00019FB04F12400FFF715FB18E04FF05000A8
:10CED00080F31188BFF36F8FBFF34F8FFEE70168B8
:10CEE00069B100F0FFFE50B14EF60450CEF20000E2
:10CEF0004FF080510160BFF34F8FBFF36F8FFFF78B
:10CF000063FB012070BD00002DE9F04F83B0029259
:10CF1000B8B11D460E460446E9B1022D03D1E06BBF
:10CF2000012840F09A8000F033FD00BB0298F0B178
:10CF30004FF0500080F31188BFF36F8FBFF34F8F16
:10CF4000FEE74FF0500080F31188BFF36F8FBFF3FF
:10CF50004F8F00BFFEE7206C0028DED04FF050005E
:10CF600080F31188BFF36F8FBFF34F8FFEE7FFF79A
:10CF700007FBA06B022D58D0E16B884255D304F11A
:10CF8000100801206F464FF0000B0DF108094FF01B
:10CF9000805A00BF0299002900F07B80C00702D0B0
:10CFA0003846FFF7D1FCFFF70FFBFFF7C3FDFFF794
:10CFB000E7FA94F84400FF2808BF84F844B094F8D6
:10CFC0004500FF2808BF84F845B0FFF7FDFA384652
:10CFD000494600F00FFB00285ED12046FEF780FF97
:10CFE000A0B102994046FFF7C5FC2046FFF73CF987
:10CFF00000F0C0FE78B94EF60450CEF20000C0F842
:10D0000000A0BFF34F8FBFF36F8F04E02046FFF700
:10D010002BF900F0AFFEFFF7B3FAA06B022D04D09E
:10D02000E16B88424FF00000B4D2204631462A46D8
:10D03000FEF790FD54F8241FC9B1204600F052FEBF
:10D0400008B34EF60450CEF200004FF0805101605C
:10D05000BFF34F8FBFF36F8F15E04FF0500080F399
:10D060001188BFF36F8FBFF34F8F00BFFEE750B142
:10D070004EF60450CEF200004FF080510160BFF335
:10D080004F8FBFF36F8FFFF79FFA012003B0BDE80A
:10D09000F08FFFF799FA04E02046FFF7E5F800F07B
:10D0A00069FE002003B0BDE8F08F00002DE9F043D9
:10D0B00081B0E8B11E46914605460F4609B3022EDF
:10D0C00002D1E86B012837D1FFF7F6FAEFF31188A8
:10D0D0004FF0500080F31188BFF36F8FBFF34F8F75
:10D0E000A86B022E19D0E96B884216D300203FE0CE
:10D0F0004FF0500080F31188BFF36F8FBFF34F8F55
:10D10000FEE7286C0028DAD04FF0500080F3118839
:10D11000BFF36F8FBFF34F8FFEE795F84540A86BC5
:10D12000284639463246FEF715FDFF2C0DD0601C0F
:10D1300085F8450001201BE04FF0500080F3118876
:10D14000BFF36F8FBFF34F8FFEE755F8240F70B119
:10D15000284600F0C7FD0146B9F1000F4FF001006D
:10D1600006D000291CBF0120C9F8000000E0012002
:10D1700088F3118801B0BDE8F0830000B0B5A8B114
:10D180008568044600F0FEFB85421CBF0020B0BD50
:10D19000E0680138E0601CBF0120B0BD20460021DE
:10D1A00000220023FFF7B0FE0120B0BD4FF0500079
:10D1B00080F31188BFF36F8FBFF34F8FFEE700003E
:10D1C0002DE9F04F85B0049298B10C460546002930
:10D1D00000F0A58000F0DCFBA8B9049898B14FF0EE
:10D1E000500080F31188BFF36F8FBFF34F8F00BFE4
:10D1F000FEE74FF0500080F31188BFF36F8FBFF34D
:10D200004F8F00BFFEE705F1240005F110090190E2
:10D2100002AF0DF1100A4FF000080AE02846FFF7B0
:10D2200023F800F0A7FD2846FEF74EFE002840F048
:10D230008480FFF7A5F9D5F838B0BBF1000F1DD0F9
:10D2400028462146FEF772FCABF10100A86328696D
:10D2500070B1484600F046FD50B14EF60450CEF293
:10D2600000004FF080510160BFF34F8FBFF36F8F0D
:10D27000FFF7AAF900200126A0B95FE0049850B199
:10D28000B8F1000F02D13846FFF75EFB4FF00108FE
:10D29000012038B952E0FFF797F900260020002856
:10D2A0004CD000BFFFF790F9FFF744FCFFF768F997
:10D2B00095F84400FF2804BF002085F8440095F845
:10D2C0004500FF2804BF002085F84500FFF77CF9E2
:10D2D0003846514600F08EF900289FD12846FEF7C7
:10D2E000F3FDB0B104990198FFF744FB2846FEF71F
:10D2F000BBFF00F03FFD00289BD14EF60450CEF25C
:10D3000000004FF080510160BFF34F8FBFF36F8F6C
:10D310008FE72846FEF7A8FF00F02CFD89E7286C70
:10D3200000283FF457AF4FF0500080F31188BFF34F
:10D330006F8FBFF34F8F00BFFEE70026304605B06A
:10D34000BDE8F08F2DE9F04381B000B3914605466A
:10D350000E4631B3FFF7B0F9EFF311884FF05000EC
:10D3600080F31188BFF36F8FBFF34F8FAC6B24B383
:10D3700095F8447028463146FEF7D8FB601EFF2F13
:10D38000A8631CD0781C85F8440001202AE04FF0E7
:10D39000500080F31188BFF36F8FBFF34F8F00BF32
:10D3A000FEE7286C0028D5D04FF0500080F311889C
:10D3B000BFF36F8FBFF34F8FFEE7002012E055F8E9
:10D3C000100F70B1284600F08DFC0146B9F1000F36
:10D3D0004FF0010006D000291CBF0120C9F8000051
:10D3E00000E0012088F3118801B0BDE8F08300005F
:10D3F0002DE9F04F85B0049158B10446006C90B10E
:10D400004FF0500080F31188BFF36F8FBFF34F8F41
:10D41000FEE74FF0500080F31188BFF36F8FBFF32A
:10D420004F8F00BFFEE700F0B3FA50B9049840B147
:10D430004FF0500080F31188BFF36F8FBFF34F8F11
:10D44000FEE704F1240004F1100501904FF00008FC
:10D4500002AF0DF1100A4FF000094FF0000B0AE087
:10D460002046FEF701FF00F085FC2046FEF72CFD6C
:10D47000002840F07F80FFF783F8A06BF0B10138FF
:10D48000A063206810B9FEF7CFFFA060286870B1D4
:10D49000284600F027FC50B14EF60450CEF20000B2
:10D4A0004FF080510160BFF34F8FBFF36F8FFFF7D5
:10D4B0008BF801260020B8B96FE000BF049850B186
:10D4C000BBF1000F02D13846FFF73EFA4FF0010BD7
:10D4D000012048B961E0B9F1000F62D1FFF774F89B
:10D4E00000200026002858D0FFF76EF8FFF722FB37
:10D4F000FFF746F894F84400FF2808BF84F84480FA
:10D5000094F84500FF2808BF84F84580FFF75CF8D1
:10D510003846514600F06EF80028A1D12046FEF7AB
:10D52000D3FC28B92046FEF79FFE00F023FCA2E7BB
:10D53000206838B9FFF724F8A06800F089FB81461D
:10D54000FFF742F804990198FFF714FA2046FEF716
:10D550008BFE00F00FFC00287FF48DAF4EF60450D8
:10D56000CEF200004FF080510160BFF34F8FBFF348
:10D570006F8F80E7B9F1000F0ED0FFF701F820465A
:10D58000FEF742FBA168024608461146FFF72CFA57
:10D59000FFF71AF8002600E00026304605B0BDE887
:10D5A000F08F4FF0500080F31188BFF36F8FBFF3FF
:10D5B0004F8F00BFFEE7000070B568B18668044673
:10D5C0000D4600F0DFF986420FD020462946FFF7CE
:10D5D0000FFF58B9002070BD4FF0500080F3118844
:10D5E000BFF36F8FBFF34F8FFEE70120E16801317A
:10D5F000E16070BDB0B5D0B10D4611B30446FEF781
:10D60000BFFF4DF6AC50C2F2010001682868421C11
:10D6100021D04DF64C536268C2F20103D3F800C02A
:10D6200091421AD323689C4517D0012422E04FF081
:10D63000500080F31188BFF36F8FBFF34F8F00BF8F
:10D64000FEE74FF0500080F31188BFF36F8FBFF3F8
:10D650004F8F00BFFEE700240CE0891A884206D9EC
:10D66000401A28602046FFF76FF9002402E00020EE
:10D6700001242860FEF7A8FF2046B0BD2DE9F04345
:10D6800083B007469000984615468946FEF726FE69
:10D6900078B106466020FEF721FE38B104460663E5
:10D6A00054B94FF0FF3003B0BDE8F0833046FEF7C9
:10D6B000A3FF0024002CF4D0DDE90A10002284F836
:10D6C0005D20CDE90010384649462A46434602947B
:10D6D000FEF726FB2046FEF76DF9012003B0BDE8FA
:10D6E000F083000070B586B00B9CCCB10C9E06B3E5
:10D6F00060250495049D602D25D1049DDDF828C08A
:10D70000022586F85D5005AD3463CDE900C502966B
:10D71000FEF706FB3046FEF74DF9059806B070BDE2
:10D720004FF0500080F31188BFF36F8FBFF34F8F1E
:10D73000FEE74FF0500080F31188BFF36F8FBFF307
:10D740004F8F00BFFEE74FF0500080F31188BFF30A
:10D750006F8FBFF34F8F00BFFEE70000F0B581B0C1
:10D76000D0B11D46174604460E46FEF709FF002DB0
:10D770001CBFA06D286094F85C000221042F84F87F
:10D780005C1012D80125DFE807F023031C262000D7
:10D79000A16D3143A1651FE04FF0500080F3118867
:10D7A000BFF36F8FBFF34F8FFEE7A16D013113D031
:10D7B0004FF0500080F31188BFF36F8FBFF34F8F8E
:10D7C000FEE7A16D0131A16506E0022803D1002525
:10D7D00001283CD103E0A6650125012837D1261D8B
:10D7E0003046FEF757FE4AF6E471C2F20101E06AE4
:10D7F0000A68904288BF086040F6143100EB800050
:10D80000C2F2000101EB80003146FEF7A1FEA06AE2
:10D8100048B14FF0500080F31188BFF36F8FBFF312
:10D820004F8F00BFFEE74DF2A401C2F20101E06A92
:10D830000968C96A88420AD94EF60450CEF200003F
:10D840004FF080510160BFF34F8FBFF36F8FFEF732
:10D85000BBFE284601B0F0BD2DE9F04120B31D46C6
:10D86000174604460E46FEF727FFEFF311884FF0E8
:10D87000500080F31188BFF36F8FBFF34F8F002DDF
:10D880001CBFA06D286094F85C000221042F84F86E
:10D890005C1012D80125DFE807F023031C262000C6
:10D8A000A16D3143A1651FE04FF0500080F3118856
:10D8B000BFF36F8FBFF34F8FFEE7A16D013113D020
:10D8C0004FF0500080F31188BFF36F8FBFF34F8F7D
:10D8D000FEE7A16D0131A16506E0022803D1002514
:10D8E000012849D103E0A6650125012844D1A06A99
:10D8F00048B14FF0500080F31188BFF36F8FBFF332
:10D900004F8F00BFFEE74AF6DC70C2F201000068EC
:10D9100030B14BF2802004F11801C2F2010015E091
:10D92000261D3046FEF7B6FD4AF6E471C2F201014B
:10D93000E06A0A68904288BF086040F6143100EB44
:10D940008000C2F2000101EB80003146FEF700FECC
:10D950004DF2A401C2F20101E06A0968C96A884275
:10D960000AD9069800281CBF012101604DF6B45069
:10D97000C2F201000121016088F311882846BDE848
:10D98000F08100004DF2A400C2F20100006870476F
:10D990004DF69450C2F201000068002804BF012037
:10D9A00070474AF6DC70C2F201000068B0FA80F0FD
:10D9B00040094000704700004DF6AC50C2F2010033
:10D9C0000068704780B5FEF777FE4DF6AC50C2F2A6
:10D9D0000100006880BD00002DE9F04F81B04AF6DB
:10D9E000DC70C2F20100006840B14BF27C20C2F250
:10D9F0000100016800240131016092E04DF6AC5055
:10DA0000C2F2010001684E1C066021D340F60C30C2
:10DA1000C2F200000168096849B14FF0500080F37C
:10DA20001188BFF36F8FBFF34F8F00BFFEE74DF23A
:10DA3000B002C2F201020168136803604DF64C5057
:10DA40001160C2F20100016801310160FEF774FB50
:10DA50004BF27421C2F2010108684DF2A40A40F6AB
:10DA600014388642C2F2010AC2F2000801D2002430
:10DA700045E040F60C37C2F2000738680024006821
:10DA800098B34AF6E47BC2F2010B19E0D9F82C00F6
:10DA9000DBF80010884288BFCBF8000000EB800064
:10DAA00008EB80002946FEF753FDD9F82C00DAF880
:10DAB0000010C96A3A68884228BF01241068B8B1CA
:10DAC0003868C068D0F80C904D4655F8040F86426F
:10DAD00010D32846FEF7DEFCD9F828000028D5D060
:10DAE00009F11800FEF7D6FCD0E74FF0FF3005E053
:10DAF0004FF0FF304BF27421C2F201010860DAF8F6
:10DB00000000C06A00EB800058F8200001284DF6A4
:10DB1000B450C2F2010088BF01240068002818BF79
:10DB20000124204601B0BDE8F08F00002DE9F0414E
:10DB30001E46154688460746FEF722FD4DF2A40410
:10DB4000C2F20104206890F85C00022819D0206815
:10DB5000816D21EA0701816520684FF0010180F89D
:10DB60005C1076B130460121FDF7E4FE4EF604501C
:10DB7000CEF200004FF080510160BFF34F8FBFF332
:10DB80006F8FFEF721FDFEF7FBFC15B12068806D5D
:10DB900028602068002590F85C100020022905D13B
:10DBA000216801258A6D22EA08028A65216881F8C8
:10DBB0005C00FEF709FD2846BDE8F081B0B580B1F4
:10DBC00004464DF2A400C2F201000068A0420AD04F
:10DBD0004FF0500080F31188BFF36F8FBFF34F8F6A
:10DBE000FEE70020B0BD206D38B3013820654FF04E
:10DBF000000018BFB0BDE16AE26C91421CD0251D47
:10DC00002846FEF747FCE06CC0F13801A1614AF6F6
:10DC1000E471E062C2F201010A68904288BF0860C4
:10DC200040F6143100EB8000C2F2000101EB8000ED
:10DC30002946FEF78DFC0120B0BD4FF0500080F367
:10DC40001188BFF36F8FBFF34F8F00BFFEE7000057
:10DC5000F0B581B000B34DF2A406C2F2010604464D
:10DC6000C06A3168C96A884219D2A169002904D4FE
:10DC70003168C96AC1F13801A16140F614376169A0
:10DC800000EB8000C2F2000707EB800081420FD05A
:10DC90003068C06AE06221E0002001B0F0BDE16CB4
:10DCA0003068C26A0020914238BF012001B0F0BD47
:10DCB000251D2846FEF7EEFB30684AF6E471C06A7F
:10DCC000C2F20101E0620A68904288BF086000EB7E
:10DCD000800007EB80002946FEF73AFC012001B0E6
:10DCE000F0BD0000B0B5C068C5687DB105F118048D
:10DCF0002046FEF7CFFB4AF6DC70C2F20100006856
:10DD000068B14BF28020C2F201001DE04FF05000DC
:10DD100080F31188BFF36F8FBFF34F8FFEE72C1D89
:10DD20002046FEF7B7FB4AF6E471C2F20101E86A49
:10DD30000A68904288BF086040F6143100EB80000A
:10DD4000C2F2000101EB80002146FEF701FC4DF21A
:10DD5000A401C2F20101E86A0968C96A884291BF58
:10DD600000204DF6B451C2F20101012088BF0860C5
:10DD7000B0BD00002DE9F04F81B04AF6DC74C2F26C
:10DD80000104206868B1FEF7FBFB206801382060C1
:10DD9000206880B10024FEF717FC204601B0BDE8E2
:10DDA000F08F4FF0500080F31188BFF36F8FBFF3F7
:10DDB0004F8F00BFFEE74AF6D870C2F2010000683C
:10DDC00000285DD04BF28026C2F2010630684DF685
:10DDD000B458C2F2010890B34AF6E47740F6143919
:10DDE0004DF2A40BC2F20107C2F20009C2F2010B0C
:10DDF0004FF0010AF068C56805F11800FEF74AFB0C
:10DE00002C1D2046FEF746FBE86A3968884288BF29
:10DE1000386000EB800009EB80002146FEF798FB9C
:10DE2000E86ADBF80010C96A884228BFC8F800A079
:10DE300030680028DED1002D18BFFEF77DF94BF2C7
:10DE40007C24C2F20104256855B10126FFF7C4FD08
:10DE5000002818BFC8F80060013DF7D100202060FD
:10DE6000D8F8000070B14EF60450CEF200004FF02A
:10DE700080510160BFF34F8F0124BFF36F8F8AE79A
:10DE8000002488E7002486E780B586B0FDF7E8FD2A
:10DE90004DF6B050C2F20100006808B30020CDE991
:10DEA000040005A804A903AAFEF714FBDDE903207A
:10DEB0000221DDF814C0CDE900104CF25120C0F66B
:10DEC00000000CA10023CDF808C0FFF70BFC4BF2BB
:10DED000B021C2F20101086010B1012006B080BD7E
:10DEE0004FF0500080F31188BFF36F8FBFF34F8F57
:10DEF000FEE700BF546D72205376630010B584B006
:10DF0000A8B14DF6B054C2F2010484462068C0B1F5
:10DF10000529CDE90012CDF808C015DCFFF738FD62
:10DF200001462068022916D1069A694615E04FF08D
:10DF3000500080F31188BFF36F8FBFF34F8F00BF86
:10DF4000FEE7002004B010BD69461A460023FFF723
:10DF5000ADF804B010BD694600220023FEF7D4FFDF
:10DF600004B010BD5FEA400C08BF91F0000F4FEA0B
:10DF70008C234FEAC12243EA51514FEA1C5018BF8B
:10DF800000F5F0404FEA300018BF41F000415FEA71
:10DF90006C5C00F02980BCF1FF3F08BF40F080407E
:10DFA0007047130C06BF12044FF0100C4FF0000C1A
:10DFB000130E04BF12020CF1080C130F04BF120160
:10DFC0000CF1040C930F04BF92000CF1020CD30F60
:10DFD00004BF52000CF1010C11464FF00002A0F1F9
:10DFE0001F00A0EB0C00704711F0004F08BF7047F6
:10DFF00031F000413FF4D5AF0B0C06BF09044FF0E0
:10E00000100C4FF0000C0B0E04BF09020CF1080CB1
:10E010000B0F04BF09010CF1040C8B0F04BF890026
:10E020000CF1020CCB0F04BF49000CF1010CCCF138
:10E03000200322FA03F341EA030102FA0CF2A0EBF7
:10E040000C0000F10100704723F07F4720F07F4C67
:10E0500080EA030000F00040ACEB070303F57C53BB
:10E0600003F1FF032DE9804909B44FEA144324EA80
:10E0700003484FEA154B25EA0B4E0FF2042606EB38
:10E0800013273E7803FB0667C7F5000707FB06F674
:10E090004FEAD64606F102064FEA543707FB066CF4
:10E0A000CCF1005C4FEA1C472CEA074C0CFB06F550
:10E0B00007FB06F404EB15464FEA961649085FEA9B
:10E0C000320234BF00204FF000404FEAD13706FB48
:10E0D00007FC4FEA1C4C0CFB0BF7D21B03FB0CF7A5
:10E0E00061EB07010CFB0EF7B0EB074072EB174238
:10E0F0000CFB08F734BFA2EB0742B2EB074261EB1F
:10E1000017414FEA0C444FEA910706FB07FC4FEA20
:10E110001C4C0CFB0BF7B0EBC74072EB573203FB08
:10E120000CF734BFA2EBC742B2EBC74261EB5731E9
:10E130000CFB0EF7B0EBC70072EB57720CFB08F745
:10E1400034BFA2EBC702B2EBC70261EB57714FEAD3
:10E15000816141EA92114FEA826242EA90124FEAEB
:10E16000806004EBCC04039F4FEAD13706FB07FC29
:10E170004FEA1C4C0CFB0BF7D21B03FB0CF761EBBB
:10E1800007010CFB0EF7B0EB074072EB17420CFBDC
:10E1900008F734BFA2EB0742B2EB074261EB17412D
:10E1A0004FEA8C5504EB9C244FEA910706FB07FCD1
:10E1B0004FEA1C4C0CFB0BF7B0EBC74072EB57322D
:10E1C00003FB0CF734BFA2EBC742B2EBC74261EBD3
:10E1D00057310CFB0EF7B0EBC70072EB57720CFB1C
:10E1E00008F734BFA2EBC702B2EBC70261EB57716D
:10E1F0004FEA816141EA92114FEA826242EA90124B
:10E200004FEA806015EB4C2544F100044FEAD1370A
:10E2100006FB07FC4FEA1C4C0CFB0BF7D21B03FB65
:10E220000CF761EB07010CFB0EF7B0EB074072EB4C
:10E2300017420CFB08F734BFA2EB0742B2EB0742D0
:10E2400061EB17414FEA813141EA92414FEA823254
:10E2500042EA90424FEA80304FEA0C7615EB1C15EB
:10E2600044F1000448EA03434EEA0B484FF0000E25
:10E27000B2EB080C71EB030724BF624639464EEB44
:10E280000E0E4FF0000B0018524149414BEB0B0BA7
:10E29000B2EB080C71EB03077BF1000B24BF624665
:10E2A00039464EEB0E0E4FF0000B0018524149411B
:10E2B0004BEB0B0BB2EB080C71EB03077BF1000B84
:10E2C00024BF624639464EEB0E0E51EA020718BFD4
:10E2D00046F0010616EB0E7655F1000254F10001EE
:10E2E00003D5BDE88901BDE80088BDE88901BDE826
:10E2F0000048B619524141EB0101A3F101037047F7
:10E3000080807F7E7D7C7B7A797877767675747372
:10E31000727171706F6E6E6D6C6C6B6A6A69686831
:10E32000676666656464636362616160605F5F5EC7
:10E330005E5D5D5C5C5B5B5A5A595958585757563D
:10E3400056555555545453535252525151505050A2
:10E350004F4F4F4E4E4D4D4D4C4C4C4B4B4B4A4AF4
:10E360004A49494948484847474747464646454538
:10E370004544444444434343434242424241414171
:10E380009C46002B30D477002BD04FEA37071CB5C2
:10E3900003B44FF010004FF01001BAF1000F06D097
:10E3A000BCF1000FDCBF40F0080040F008014FF066
:10E3B00000000FBCBDE810400BF1010BBBF1010FD9
:10E3C00008BF5FEA170722BF12F1010211F1010134
:10E3D0004FF0004143F1000300F0004043EA000029
:10E3E0007047F9D35708D0E746EA06464FEA164683
:10E3F00013F1400F1FDD13F1200FDFBF16430A4654
:10E40000002120335B42BED0C3F1200746EA064616
:10E410004FEA164602FA07F746EA070622FA03F21F
:10E42000C3F1200701FA07F742EA070221FA03F1D4
:10E430004FF00003A7E746EA020646EA06464FEA1F
:10E44000164646EA0106BCBF46EA0646360C4FF0C1
:10E4500000034FF000024FF0000194E72DE9804CDB
:10E4600070B49A46934691E8380007C831EA400CE8
:10E4700048BF34EA430C03D5FFF7E6FDFFF780FF02
:10E48000F0BCBDE8008C2DE9804C70B49A469346F0
:10E4900091E8380007C810F0804F08BF13F0804F94
:10E4A00003D100F005F8FFF76BFFF0BCBDE8008C6E
:10E4B00020F07F4723F07F4C80EA030000F000400B
:10E4C00007EB0C03A3F57C53A3F1FE0392F0000FBE
:10E4D00000F0B38095F0000F00F077802DE901493E
:10E4E0004FEA114021EA00484FEA144624EA064761
:10E4F00000FB06FC08FB06F607FB08F818EB0648CD
:10E500004CEB164C00FB07F718EB07484CEB174099
:10E510004FEA124B22EA0B4E4FEA154625EA064710
:10E520000BFB06FC0EFB06F607FB0EFE1EEB064E73
:10E530004CEB164C0BFB07F71EEB074E4CEB174B47
:10E5400018EB0B0840F1000018EB0E0B58EB00081D
:10E5500040F100008F1A4FF000014FF000063CBF61
:10E56000C943661B14BFB5EB040C00213CBFC94373
:10E57000F61B4FEA174427EA04454FEA1C472CEAEA
:10E58000074C04FB076205FB07F70CFB05F616EBCF
:10E59000074642EB174204FB0CFC16EB0C4642EB21
:10E5A0001C421BEB060658EB020241414EEA8E0E5E
:10E5B00046EA9E0601D5BDE80189B619524141EBF4
:10E5C0000101A3F10103BDE801894FEA144524EAE2
:10E5D00005464FEA114721EA074C05FB07F406FB05
:10E5E00007F70CFB06F111EB074144EB174405FB61
:10E5F0000CFC11EB0C4144EB1C444FEA124722EA9D
:10E60000074C05FB07F206FB07F70CFB06F616EBBB
:10E61000074642EB174205FB0CFC16EB0C4642EB9F
:10E620001C456A1854F1000148BF7047B6195241A1
:10E6300041EB0101A3F10103704795F0000F37D0C2
:10E640004FEA114221EA02464FEA144724EA074CF6
:10E6500002FB07F106FB07F70CFB06F414EB07447B
:10E6600041EB174102FB0CFC14EB0C4441EB1C4149
:10E670004FEA154725EA074C02FB07F506FB07F7AB
:10E680000CFB06F616EB074645EB174502FB0CFCA8
:10E6900016EB0C4645EB1C42121951F1000148BF24
:10E6A0007047B619524141EB0101A3F101037047D4
:10E6B0004FEA144524EA05464FEA114721EA074C80
:10E6C00005FB07F106FB07F70CFB06F212EB07420E
:10E6D00041EB174105FB0CFC12EB0C4251EB1C41CA
:10E6E0004FF0000648BF7047921841EB0101A3F1BB
:10E6F0000103704703B401984100009850EAC1201B
:10E7000018BF04204A0D18BF40F0010040F2FF720C
:10E71000B2EB515F08BF40F00200012808BF05209E
:10E7200002B070474100080218BF04200A0E18BF4B
:10E7300040F001004FF07F4232EA010108BF40F093
:10E740000200012808BF05207047000010B54FF0F7
:10E750000E402DED028BB0EE408A18EE104A00EB11
:10E760004400B0F1506F4AD84FF0FC40B0EB440F7A
:10E7700022D2B0EEC80AF7EE000A30EEC00AF6EE7A
:10E78000000A60EE208A18EE900A01F0B0F801EE5F
:10E79000100A14F0004F1DBFDFED2D0A9FED2D0A6A
:10E7A000B1EE411ADFED2C0A08BF9FED2C0AF8EEFE
:10E7B000001A21EE218A05E0DFED290A68EE088AB9
:10E7C000B0EE600A9FED271ADFED271A30EE080A37
:10E7D00048EE811A9FED251A08EEA11ADFED241AE2
:10E7E00048EE811A9FED231A08EEA11A68EE281A46
:10E7F000BDEC028B01EE810A30EE200A10BD4FF015
:10E80000E440B0EB440F0CD918EE100AFFF78AFF72
:10E81000042808BF00F09EFFB0EE480ABDEC028B52
:10E8200010BD4FF07F40B0EB440F07D2B0EE480A66
:10E83000BDEC028BBDE8104000F07EBF0120F1F777
:10E84000DCFFBDEC028BBDE8104000F07BBF000098
:10E850000000C9BF22AAFDB90000C93F22AAFD39A4
:10E860000000000024FE1C3DC78AD83C1E67383DCE
:10E870001B93993DAFAA2A3E70B59B482DED020B24
:10E880002DED068B079D25F00044A04218DC97482B
:10E89000844202DC0AD1069840B19DED060BBDEC26
:10E8A000068B02B0BDE8704000F012BF002DCCBF57
:10E8B0009FED8F0B9FED900BBDEC068B02B070BDF2
:10E8C0008F48A04215DD8F48A042D8BF4FF0FF34DB
:10E8D00058DD9DED060B51EC100BFFF70BFF0428E4
:10E8E00008BF00F019FF9DED060BBDEC068B02B0D2
:10E8F00070BD9DED060B51EC100B00F0ECFFCDE967
:10E90000060181489FED828BA0423CDD8248A042F7
:10E910001FDD00249FED82AB9DED060B53EC1A2BFF
:10E9200051EC100B01F056F89DED060B41EC190B64
:10E9300053EC1A2B51EC100B01F04EFB53EC182B3F
:10E9400001F0C8FD53EC192B01F0F8F8CDE90601F0
:10E9500049E09DED060B012453EC182B51EC100BF4
:10E9600001F038F89DED060B41EC190B53EC182B18
:10E9700051EC100B01F0AEFD53EC192B01F0DEF859
:10E98000CDE906012FE06848A0421FDD02249FED7B
:10E99000689B9DED060B53EC192B51EC100B01F00D
:10E9A0001BFB53EC182B01F015F89DED060B41EC09
:10E9B000180B53EC192B51EC100B01F08BFD53ECA1
:10E9C000182B01F0BBF8CDE906010CE09DED060B1C
:10E9D000032453EC102B9FED580B51EC100B01F05E
:10E9E000ADF8CDE906019DED060B53EC102B51EC73
:10E9F000100B01F0F1FA41EC180B53EC182B01F05D
:10EA0000EBFA41EC190B4E480621B0EE490AF0EE44
:10EA1000690A784400F0E0FD53EC182B51EC100B20
:10EA200001F0DAFA41EC180B4648B0EE490AF0EE74
:10EA3000690A0521784400F0CFFD53EC192B51EC05
:10EA4000100B01F0C9FA41EC100B51EC180B53EC10
:10EA5000102B002C0EDA00F0BDFF9DED061B53ECD1
:10EA6000112B01F0B9FA9DED061B53EC112B01F0AF
:10EA700059FC35E000F0AEFF9DED061B53EC112B69
:10EA800001F0AAFA41EC100B2F48784400EBC400C7
:10EA900090ED001B51EC100B53EC112B01F01AFD03
:10EAA0009DED061B53EC112B01F014FD41EC100BF6
:10EAB0002648784400EBC40090ED001B51EC100B8D
:10EAC00053EC112B01F02EFC41EC100B002DA2BFDA
:10EAD000BDEC068B02B070BD51EC100B00F03CFF9A
:10EAE00041EC100B01E70000000010440000F07F33
:10EAF000182D4454FB21F93F182D4454FB21F9BF34
:10EB00000000DC3F0000203E0000F33F000000005A
:10EB1000000000000000F03F0000E63F00000000A1
:10EB200000000000000000400080034000000000E2
:10EB3000000000000000F83F000000000000F0BFEF
:10EB4000C21E0000781E0000021E0000BA1D000058
:10EB500070B56F4E2DED040B2DED048B82B0DDF8FA
:10EB600024C0DDE907235C422CF000411C4341EA4C
:10EB7000D474069D22F00040B44205D86C422C4368
:10EB800040EAD474B4420BD99DED081B9DED060BF1
:10EB900002B0BDEC048B04B0BDE8704000F0A2BD33
:10EBA000ACF14054A4F17F641C430BD0022404EA6E
:10EBB000AC7444EAD27405439FED578B9FED582BFC
:10EBC00007D015E09DED060B51EC100B00F07BFE1D
:10EBD00042E0002C11BF012C9DED060B02B0BDECF4
:10EBE000048B04BF04B070BD022C38D0032C3BD082
:10EBF0000B439FED4D1B9FED4E0B0AD0B14218D138
:10EC0000B04209D121F0804120F080400991079065
:10EC10000FE0002A15DA10E0474B7B44002C08BFB8
:10EC200093ED000B0DD0012C10D0022C17D0032C2B
:10EC30001AD0B0421DD1002A03DAB0EE410AF0EE3C
:10EC4000610A02B0BDEC048B04B070BD93ED000B03
:10EC500051EC100B00F080FE41EC100BF1E7B0EE30
:10EC6000480AF0EE680AECE7B0EE420AF0EE620AFB
:10EC7000E7E7401A00159FED329B3C28C8BF8DED99
:10EC8000000B17DCBCF1000FBCBF10F13C0F8DED89
:10EC9000009B0FDB9DED080B53EC102B9DED060B3D
:10ECA00051EC100B00F04AFF00F015FE00F00BFED7
:10ECB000CDE90001B4B1012C10D0022C9FED220B44
:10ECC00053EC102B9DED000B51EC100B19D001F003
:10ECD00001FC53EC182B01F0FDFBBDE7019880F01F
:10ECE000004001909DED000B53EC192B51EC100BE3
:10ECF00001F07EF804BF0220F1F77FFD9DED000BCF
:10ED00009FE701F0E7FB53EC182B01F00BFBA3E7A7
:10ED10000000F07F00000000182D4454FB21094042
:10ED2000182D4454FB2109C0182D4454FB21F9BF70
:10ED3000182D4454FB21F93FEA1C0000000000009C
:10ED40000000000000000000075C143326A6A13C70
:10ED500070B54FF068422DED048BF0EE408A18EE4E
:10ED6000900AB0EE608A18EE101A02EB4003B3F17D
:10ED7000654F3CBF02EB4102B2F1654F7DD200BF4F
:10ED8000C0F3C753C1F3C7529A1A1B2A09DD10F00A
:10ED9000004F14BF9FED830A9FED830ABDEC048BE7
:10EDA00070BD12F11A0F36DA11F0004F09D010F0D1
:10EDB000004F0CBF9FED7D0A9FED7D0ABDEC048BDB
:10EDC00070BD88EE889A19EE100AFFF7ABFC042894
:10EDD00008BF00F0BFFC18EE900AFFF7A3FC054641
:10EDE00018EE100AFFF79EFC044619EE100AFFF712
:10EDF00099FC042D18BF052D08D1042C18BF052C33
:10EE000004D1002804BF0220F1F7F7FCB0EE490A54
:10EE1000BDEC048B70BD4200B2EB410F3AD910F04B
:10EE2000004F19BFDFED630A9FED630ADFED630A50
:10EE30009FED630AB0EE481A0A46B1EE688A80F088
:10EE40000041F0EE418A10460A1A5200B2F1807F6A
:10EE500034D2484010F0004FDFED5A1A9FED5A2A85
:10EE60001DBFBEEE001A70EEE10A30EE420AB6EEA9
:10EE7000001A08BF70EEA10A00E040E008BF30EEC3
:10EE8000020AB0EE682A01EE482A08EE818AC2EE34
:10EE9000081A15E011F0004F04BF9FED4C0AF0EE88
:10EEA000400AD1D010F0004F19BFDFED490A9FEDA5
:10EEB000490ADFED490A9FED490AC5E7C8EE881AFD
:10EEC00021EEA11A9FED462ADFED462A41EE022AE5
:10EED0009FED452A01EE222ADFED442A41EE022A67
:10EEE0009FED432ABDEC048B01EE222A21EE811A0C
:10EEF00001EE020A30EE210A30EE200A70BD4FF01A
:10EF00007F42B2EB400F28BFB2EB410F09D2F0EEC7
:10EF1000480AB0EE680ABDEC048BBDE8704000F012
:10EF20000EBC40EA01035B0008BF41F0FF410BD07B
:10EF3000B2EB400F08BFB2EB410F08D120F0804088
:10EF400008EE900A21F0804108EE101A18E7B2EBA3
:10EF5000400F12BF5FEA410340F0FF4001F0004163
:10EF60003FF40EAFB2EB410F12BF5FEA400200F078
:10EF7000004041F0FF413FF403AF4A0092EA4003F2
:10EF80003FF5FEAE002AACBF9FED1A0A9FED1A0AAC
:10EF900068EE808A28EE008A18EE900A18EE101AA1
:10EFA000EEE60000DB0FC9BFDB0FC93FDB0F4940B6
:10EFB000DB0F49C00000C9BF22AAFDB90000C93F4C
:10EFC00022AAFD390060ED3EC30ACE3700000000E2
:10EFD000000049C022AA7DBA0000494022AA7D3A19
:10EFE0002DAD65BD8FB8D53D0FB511BE61C84C3E86
:10EFF000A8AAAABE0000804F0000802F10EE101AB1
:10F0000008B5444A6846B2EB410F28D94FF0E640B4
:10F01000B0EB410F94BF00204FF0FF3000900098FC
:10F02000002861DB60EE000A10F0010F45D010F0FF
:10F03000020FDFED391A9FED391A00EEA11ADFED4C
:10F04000381A40EE811A21EEA01AF0EE400A40EE86
:10F05000010A08BFF1EE600AB0EE600A08BD314B4C
:10F0600021F0004293423CD911F0004FDFED2E0A0F
:10F0700020EE201ADFED2D0A19BF31EE601A71EE75
:10F08000200A31EE201A71EE600ABDEEE01A11EE90
:10F09000100A9FED271A00F0030000EEC10A9FED51
:10F0A000251A009000EEC10A9FED231A00EEC10A56
:10F0B0009FED221A00EEC10AB1E79FED211A9FEDE4
:10F0C000210A10F0020F00EE810A9FED1F1A00EED8
:10F0D000801AB7EE000A00EE810A18BFB1EE400AAE
:10F0E00008BD00F03FFB9AE710EE100A4000B0F1B7
:10F0F0007F4F3CBFB7EE000A08BD07D14FF00100BB
:10F10000F1F77BFBBDE8084000F01CBBBDE8084000
:10F1100000F012BBB61F927E336D4CB9DA82083C08
:10F12000A0AA2ABE490E494683F9223F0000004B9F
:10F130000000C93F00A0FD390020A2331A61342C21
:10F14000B93AB2BACA9F2A3DDDFFFFBE10B52DED18
:10F15000040B86B09DED060B10EE100A10EE901A0F
:10F160008DED000B002818BF0120084320F000405F
:10F17000C0F17F6000F1E040C00F21D19DED080B90
:10F1800010EE101A10EE900A8DED000B002918BF3A
:10F190000121084320F00040C0F17F6000F1E04011
:10F1A000C00F0DD129490798B1EB400F04BF069855
:10F1B000002842D00998400004BF089800283CD09D
:10F1C0009DED080B53EC102B9DED060B51EC100B35
:10F1D00000F0FAFFCDE902019DED020B40F2FF7154
:10F1E00010EE900A8DED000B31EA105021D00798F7
:10F1F000039900F0004001F00041884219D09DEDD4
:10F20000080B8DED040B9DED020B8DED000B10EE48
:10F21000900A059961F31E0005909DED041B9DED7C
:10F22000020B51EC110B53EC102B01F07BF8CDE9E4
:10F2300002019DED020B0AB010BD0120F1F7DDFACD
:10F240000AB0BDE8104000F057BA00000000E0FF2F
:10F2500000B510EE101A2DED028B81B0524A6846AF
:10F26000B2EB410F2ED94FF0E640B0EB410F94BF07
:10F2700000204FF0FF3000900098B0EE408A002848
:10F280006ADB10F0010F4BD068EE080A9FED471AB9
:10F290009FED470A00EE810A9FED461A10F0020F1B
:10F2A00000EE801AB7EE000A00EE810A02BF01B03C
:10F2B000BDEC028B00BD00BF01B0B1EE400ABDEC59
:10F2C000028B00BD3C4B21F00042934241D911F02A
:10F2D000004FDFED3A0A20EE201ADFED390A19BFA0
:10F2E00031EE601A71EE200A31EE201A71EE600ADA
:10F2F000BDEEE01A11EE100A9FED321A00F0030085
:10F3000000EEC10A9FED301A009000EEC10A9FED99
:10F310002F1A00EEC10A9FED2E1A00EEC10AABE7CC
:10F3200028EE080A9FED2B1ADFED2B0A10F0020FD2
:10F3300040EE010A9FED291A00EE201A61EE000A44
:10F34000B0EE480A08EE200AB6D101B0BDEC028B3F
:10F3500000BD00F007FA8FE718EE100A4000B0F188
:10F360007F4F0DD218EE100AFFF7DCF9042808BF12
:10F3700000F0F0F9B0EE480A01B0BDEC028B00BD20
:10F3800009D10120F1F739FA01B0BDEC028B5DF82B
:10F3900004EB00F0D7B901B0B0EE480ABDEC028B27
:10F3A0005DF804EB00F0C8B9B61F927EB93AB2BA64
:10F3B000CA9F2A3DDDFFFFBE490E494683F9223F21
:10F3C0000000004B0000C93F00A0FD390020A2331F
:10F3D0001A61342C336D4CB9DA82083CA0AA2ABEDB
:10F3E00000B52DED048BB0EE409AF0EE609A83B03C
:10F3F00051EC190B00F0A2FF41EC180B18EE100AAB
:10F4000018EE901A8DED008B002818BF01200843DC
:10F4100020F00040C0F17F6000F1E040C00F14D048
:10F4200019EE101A19EE900A8DED009B002918BFF5
:10F430000121084320F00040C0F17F6000F1E0406E
:10F44000C00F04BF0120F1F7D8F9B0EE480A03B0AD
:10F45000F0EE680ABDEC048B00BD000000B510EEB4
:10F46000101A2DED028B81B04D4A6846B2EB410F68
:10F470003CD94FF0E640B0EB410F94BF00204FF075
:10F48000FF3000900098B0EE408A00285FDB28EE45
:10F49000080ADFED440A9FED441A00EE201ADFED62
:10F4A000430A40EE010A9FED421A00EE201ADFEDFA
:10F4B000410A10F0010F40EE010A9FED3F1A00EEE5
:10F4C000201A61EE000AB0EE480A08EE200A02BFD8
:10F4D00001B0BDEC028B00BDBFEE001A01B0C1EE61
:10F4E000000ABDEC028BB0EE600A00BD334B21F088
:10F4F0000042934228D911F0004FDFED310A20EE8F
:10F50000201ADFED300A19BF31EE601A71EE200AC1
:10F5100031EE201A71EE600ABDEEE01A11EE100A0B
:10F520009FED291A00F0030000EEC10A9FED271A93
:10F53000009000EEC10A9FED261A00EEC10A9FED71
:10F54000251A00EEC10A9DE700F00CF99AE718EEC3
:10F55000100A4000B0F17F4F0DD218EE100AFFF7ED
:10F56000E1F8042808BF00F0F5F8B0EE480A01B051
:10F57000BDEC028B00BD09D10120F1F73EF901B0CD
:10F58000BDEC028B5DF804EB00F0DCB801B0B0EE2E
:10F59000480ABDEC028B5DF804EB00F0CDB800002A
:10F5A000B61F927EBCE9223C0B6D063B8A76CE3CB0
:10F5B000ACB5593D35A1083E29AAAA3E490E494697
:10F5C00083F9223F0000004B0000C93F00A0FD3935
:10F5D0000020A2331A61342C70B504462DED028B45
:10F5E0004D1E00EBC500B0EE408AF0EE608A90ED53
:10F5F000000B35F0060017D053EC182B51EC100B14
:10F6000000F0EAFC41EC100B6D1E04EBC50090ED20
:10F61000001B51EC100B53EC112B00F0DBF941EC0B
:10F62000100B35F00600E7D1022D36D0042D1CD08A
:10F63000062D1CBFBDEC028B70BD53EC182B51EC9A
:10F64000100B00F0C9FC94ED0A1B53EC112B00F0D9
:10F65000C1F953EC182B00F0BFFC94ED081B53ECE0
:10F66000112B00F0B7F941EC100B53EC182B51ECB7
:10F67000100B00F0B1FC94ED061B53EC112B00F0C5
:10F68000A9F953EC182B00F0A7FC94ED040B53ECF4
:10F69000102B00F09FF941EC100B53EC182B51ECA0
:10F6A000100B00F099FC94ED021B53EC112B00F0B1
:10F6B00091F953EC182B00F08FFC94ED001B53ECE8
:10F6C000112B00F087F9BDEC028B41EC100B70BDE3
:10F6D00010B553EC102B51EC100B00F07BF941EC02
:10F6E000100B10BD10B553EC112B51EC100B00F0AA
:10F6F00071F941EC100B10BD9FED050B10B553ECEB
:10F70000102B51EC100B00F019FA41EC100B10BD4E
:10F7100000000000000000009FED050B10B553EC49
:10F72000102B51EC100B00F057FC41EC100B10BDEE
:10F73000000000000000001030EE000A704730EEBC
:10F74000200A7047DFED020A80EEA00A7047000031
:10F75000000000009FED020A20EE000A7047000042
:10F76000000000102DE9F0014FF07F42B2EB410F95
:10F770009FBF4FF0FF310160BDE8F00170474FF0CF
:10F78000004242EA0123C1F3C752783A551112F000
:10F790001F0C434CCCF120067C44C1F3C752A2F1AC
:10F7A00078024FEA621204EB820254F8254008BF47
:10F7B000D2E9015612D0556804FA0CF425FA06F77E
:10F7C0003C43976805FA0CF527FA06F8D26807FA61
:10F7D0000CFCF24045EA08054CEA0206A4FB034C87
:10F7E000A5FB0352A6FB03631D449D4234BF0126C3
:10F7F00000261319334416B1934202D903E0934211
:10F8000001D2012200E00022624402F1200C9206A3
:10F81000DC0C42EA443200EE102A5B03DFED210AE1
:10F82000F8EEC01A00EE103A4FEA9C1C11F0004F9F
:10F83000B8EE400AC0F800C020EE201A00EE105AC0
:10F84000DFED190AB8EE400A20EE200A71EE810AB7
:10F8500070EE800A10EE902A02F500626FF30B0240
:10F8600000EE902A70EEE11A31EEC11ADFED101AA7
:10F8700030EE411A9FED0D0A20EE800A01EE210ABA
:10F880009FED0C1A00EE810A04BFBDE8F00170473D
:10F89000CCF180510160BDE8F001B1EE400A704743
:10F8A00074110000000000360000802C22AAFD29FF
:10F8B000DB0FC92F0000C92F30380A2801D20120E0
:10F8C00070470020704710B541EC100BFEF7D4FFD5
:10F8D00051EC100B10BD82B0CDE9000121F00040C9
:10F8E00001909DED000B02B051EC100B704710B56C
:10F8F00000EE100A2DED028BB1EEC08A18EE100A50
:10F9000020F00040C0F1FF40C00F0AD010EE100AF6
:10F9100020F00040C0F1FF40C00F04BF0120F0F70D
:10F920006CFF18EE100ABDEC028B10BD10B500295B
:10F930000AD00878002807D005487844F1F738FB4A
:10F94000002801D0002010BD0248784410BD0000FE
:10F95000161400000E14000081F00041704780F082
:10F960000040704721F00041704720F00040704790
:10F9700021F0004201F00043A2F16052B2F5801F75
:10F9800028BFD2F17F6C0BD95FEA001C43EAC202A8
:10F9900042EB507018BF704728BF20F0010070473D
:10F9A000B2F5801FBCBF184670474FEA410C1CF5EA
:10F9B000001F02D2084600F053BF70B500F0B6FB3E
:10F9C00000000089FFF7F6BF4FF00040A0F580006F
:10F9D0007047000010B591EA030F48BF83F0004361
:10F9E00000F18085841A71EB030C05D2121943EBE8
:10F9F0000C03001B61EB0C014FEA1154A4EB135CE8
:10FA0000DFF81CE11EEA430F18BF9EEA445F00F0D6
:10FA1000748021EA045123EA0E0343F48013DCF1DD
:10FA2000200E32D322FA0CFE10EB0E0023FA0CFE4D
:10FA300041EB0E01CCF1200E03FA0EFE10EB0E008E
:10FA4000CCF1200E51F10001B1F5801F32D201EB53
:10FA5000045112FA0EF2BDE8104058BF7047401C26
:10FA600038BF5FEA420218BF7047002814BF20F079
:10FA7000010041F100014FEA410313F5001F38BFB7
:10FA80007047A1F1C04100F047BC012A43EB0302DB
:10FA9000ACF1200CDCF11F0E32BF4FF0000E23FA48
:10FAA0000CF310EB030041EB0451B4EB115FD0D029
:10FAB000A1EB045101F58011490801EB04515FEA03
:10FAC00030000ED350F1000038BF12FA0EFE08D1FC
:10FAD000BDE81040C9E7401C38BF5FEA4202CAD106
:10FAE000C3E7BDE810404FEA410313F5001F38BFDC
:10FAF0007047A1F1C04100F00FBC9EEA445F08D0FE
:10FB000011EA5E0FBDE8104004BF01F00041002083
:10FB10007047BDE8104070B500F008FB64FBBE3EC6
:10FB20000000E0FF491058BFC1F140415B1058BFD1
:10FB3000C3F140438B42EFF3008070472DE9C04191
:10FB400030B4DFF8A4C23CEA111418BF3CEA131425
:10FB500000F0ED801CEA111481EA030544EAD57433
:10FB600018BF1CEA131500F0C880A4EB050404F1CB
:10FB70007F7404F500344FF0004545EAC12145EAA1
:10FB8000C32341EA505143EA52534FEAC0204FEA9F
:10FB9000C222994208BF904200F09D804FEA13654F
:10FBA0000FF24416765D4FEA134506FB05F7C7F1E1
:10FBB000807706FB07F74FEAD737A7FB0368764243
:10FBC000A7FB06CEC8F5803838BFA8F1010807FBAF
:10FBD00008E6A6FB028C4FF0000EE6FB03CEDCF13C
:10FBE000000CCEF1004E38BFAEF1010EA6FB0C5852
:10FBF0004FF00007E6FB0E87A1FB08C6A0FB07CE6F
:10FC000016EB0E064FF0000545F10005E1FB076518
:10FC100015F1E04E7EBFA4F580345FEA46066D41E3
:10FC200016F1800745F100054FEA172747EA0567F7
:10FC30004FEA15254FEA0666A6F1DE46B6F1805F6B
:10FC400020D9384605EBC47124F0010C01EB0C11EE
:10FC5000BCF1FE6F02D8F0BCBDE8008124425CBF5D
:10FC600001F5801E9EEAC47F02D4F0BCBDE800818D
:10FC7000244200F13980A1F1C041F0BCBDE800414F
:10FC800000F04ABB4FEAD02040EA41504FEAD12170
:10FC90004FEAD22242EA43524FEAD323A7FB02861D
:10FCA00007FB036605FB02661EEA0E0F58BFA6EBB4
:10FCB0000056B6EB00564FEA520E4EEAC37E18EBE2
:10FCC0000E0E56EB530EBCD518EB02085E417F1C9E
:10FCD00055F10005B5E74FF480154FF000074FF0E0
:10FCE00000064FF00008ACE701F1C04101F000410F
:10FCF0004FF00000F0BCBDE800810CEA131511EADA
:10FD00000C1F00D00CE013EA0C1F00F026804FF00F
:10FD1000000081EA030101F00041F0BCBDE8008170
:10FD2000F0BCBDE8004181EA030100F0F5BAF0BC87
:10FD3000BDE8004170B500F0F9F900BF097EFC3E56
:10FD400000F007B84FF0000081EA030101F0004124
:10FD5000704781EA030100F0DFBAF0BCBDE8004162
:10FD600022494FF000007047FFFDFBF9F7F5F4F270
:10FD7000F0EEEDEBE9E8E6E4E3E1E0DEDDDBDAD846
:10FD8000D7D5D4D3D1D0CFCDCCCBCAC8C7C6C5C4A4
:10FD9000C2C1C0BFBEBDBCBBBAB9B8B7B6B5B4B3BB
:10FDA000B2B1B0AFAEADACABAAA9A8A8A7A6A5A4A6
:10FDB000A3A3A2A1A09F9F9E9D9C9C9B9A9999986A
:10FDC0009797969595949393929191908F8F8E8E0D
:10FDD0008D8C8C8B8B8A898988888787868585849A
:10FDE00084838382828181800000FF070000F87F86
:10FDF00051EA030C17D41CF5801F58BFBCF5801FB7
:10FE000000F10680994218BF704708BF90427047C2
:10FE100007D711F5801F58BF13F5801F19D49942D9
:10FE20007047894270471CF5801F08D5BCF5801FBC
:10FE3000F7D58B4218BF704708BF824270474FF416
:10FE4000001C1CEB410F38BF1CEB430F01D28B424F
:10FE5000704770B500F06AF9922449004FF00051E4
:10FE60004FF08053FFF75EBE4FEA1153A3F5806356
:10FE7000D3F11E03A8BFD3F1200C08DB4FF00042E2
:10FE800042EAC12252EA505232FA03F07047094264
:10FE90000BD4102BC4BF0020704703F5787CBCF155
:10FEA000FF3F05D04FF0FF3070474FF00000704724
:10FEB00070B500F03BF900BF4992248000207047E4
:10FEC000F0E7B0FA80F310FA03F10AD0C3F11D0392
:10FED00003F580634FEA03524FEA415002EBD12110
:10FEE00070474FF00000704751EA030C17D41CF51F
:10FEF000801F58BFBCF5801F00F10680994218BFD3
:10FF0000704708BF9042704707D711F5801F58BF50
:10FF100013F5801F19D499427047894270471CF528
:10FF2000801F08D5BCF5801FF7D58B4218BF7047DE
:10FF300008BF824270474FF4001C1CEB410F38BFD2
:10FF40001CEB430F01D28B42704770B500F0EEF806
:10FF5000922449004FF080514FF00053FFF7E2BD6B
:10FF600051EA030C17D41CF5801F58BFBCF5801F45
:10FF700000F10680994218BF704708BF9042704751
:10FF800007D711F5801F58BF13F5801F19D4994268
:10FF90007047894270471CF5801F08D5BCF5801F4B
:10FFA000F7D58B4218BF704708BF824270474FF4A5
:10FFB000001C1CEB410F38BF1CEB430F01D28B42DE
:10FFC000704770B500F0B2F8922449004FF000512C
:10FFD0004FF08053FFF7A6BD70B5DFF848C11CEAAB
:10FFE000111E1EBF1CEA13159EEA0C0F95EA0C0F9A
:10FFF00000F06F8081EA03044EEAD47EAE4421EA29
:020000040801F1
:100000004C1123EA4C1341F4801143F48013AEF1F8
:100010007F7EA1FB024CA0FB0365361955EB0C0556
:10002000A1FB034C4CF10003A0FB021C16EB0C06D9
:10003000654153F10003094218BF46F0010613F46D
:10004000007F0BD14FEA03314FEA053041EA1551E9
:1000500040EA165034036FF003020AE04FEAC3216E
:100060004FEAC52041EA555140EA5650F4026FF07C
:10007000020202EB2E4201EB025585EACE710AD054
:100080005FEA440C18BF24F0004450F1000041F135
:10009000000120EAD47040F2FE7C624500D270BDBF
:1000A000A84214BF4FF080444FF04044002E08BFD8
:1000B0000024BEF1806FA8BFA1F1C041BDE870402F
:1000C00080F22A8101F1C04101F000414FF00000AF
:1000D00070470CEA13159EEA0C0F18BF95EA0C0F37
:1000E00006D081EA030E4FF000000EF0004170BD13
:1000F00000F01CF88900013E00F007B800F009B8D4
:100100004FEA430C5FEA5C5C08D081EA030100F02F
:1001100003B94FEA410C5FEA5C5CF6D102494FF04B
:10012000000070470000FF070000F87F0EF1020E8C
:100130002EF0030E5EF8046B364205D4012A43EB21
:10014000030515F5001F12D8012841EB010C1CF521
:10015000001F0CD80ED14FEAD17C0CEB4C0C0CF1EB
:10016000020C15F5001F08BF4CEBD37C04E04FF0E8
:10017000080C01E04FEAD37C0CEB4C0526FA05F69F
:1001800006F00706B6F1040C06D20EEB860CBDE8AD
:1001900070404CF0010C6047DFE80CF0090B0202E4
:1001A0004FF00041A1F500214FF0000070BD19464D
:1001B0001046012851EB010418BFD4F5001484BF88
:1001C000002001F0004170BD70B5DFF844C13CEA89
:1001D000111418BF3CEA131500F08F8011F1004F85
:1001E0000CEA11141CEA131568BF45F0050518BF89
:1001F00011EA0C1F00F0798021EA4C1123EA4C131C
:1002000041F4801143F480132E46A5F58035AC42AD
:100210003DDDA4F58036801A994109D54042C1F1EF
:10022000000134BFB1F10101B1F1000185F0010518
:1002300011F4F01F08D011F4801FE8D1400041EB09
:100240000101A4F58034F6E721F00041B1FA81F60E
:10025000202E04BFB0FA80FE0EF12006A6F10B0698
:10026000A4EB0644B6F1200E0CD2C6F1200E01FA22
:1002700006F120FA0EF641EA0601CEF1200600FA58
:1002800006F003E000FA0EF14FF00000BFE750EA7D
:10029000410E23D04FEA244EBEEB254F0FDB99428F
:1002A00008BF904204D00AD3520043EB0303B0E7E7
:1002B0004FEA1646B6EB144F08BF85F00105B4F5BA
:1002C000803401EB041181EAC57100DB70BD01F1DE
:1002D000C04101F000414FF0000070BD4FEA457190
:1002E0004FF0000001F0004170BD1CEA131F09D05F
:1002F0004FF0000001F0004170BDFFF717FF00BF95
:10030000EDFFFF3EBDE8704002494FF0000070472E
:100310000000FF070000F87F0808A0F500114FEA71
:100320003101704710B591EA030F81F000413FF5AC
:1003300059AB83F0004300F0D5B800002DE9F0413F
:1003400001F5801CBCF5001FC0F2A9804FEA115CCA
:1003500021EA0C5141F480110CF1FD0C5FEA5C0CB8
:100360000CF5C07C01D340004941890241EA90511B
:1003700087022EA48E0EA45D0A0C04FB04F602FB79
:1003800006F6C6F14046A4FB0662F60D46EA422692
:1003900006FB06F4A4FB01235242C3F1404338BFDD
:1003A0005B1EA6FB02420024E6FB0324D20B42EABA
:1003B0004446A6FB0623A1FB02E2A3FB07E4E3FB02
:1003C00061426442C2F1404E38BFAEF1010EA6FB5D
:1003D00004234FF00002E6FB0E32A2FB034634007A
:1003E000E2FB6264A1FB06E6A4FB07E8E4FB6168AC
:1003F0007642C8F1405838BFA8F10108A2FB06E4D4
:10040000A3FB08E5E2FB6854A1FB05E6A7FB04E8B3
:10041000E1FB648618F1200556F10006A80940EAC0
:100420008660B109A8F11B0808F03F08B8F10A0F6F
:100430001CD901EB0C51BDE8F08100BFFCF5EEE8E2
:10044000E2DDD8D3CFCBC7C3C0BDB9B6B4B1AEAC73
:10045000A9A7A5A3A19F9D9B9A9896959392908FEB
:100460008D8C8B898887868584838281A0FB006838
:1004700000FB01F208EB4208B8EB872807D53418D7
:1004800058EB0104D5D5401C51F10001D1E7341AD5
:1004900078EB0104CDD4401E71F10001C9E75FEA99
:1004A0004C0C5FEA9C5C0DD105D301F000414FF08C
:1004B0000000BDE8F081BDE8F04170B5FFF736FE01
:1004C0006DDBFFBEBDE8F04101494FF00000704711
:1004D0000000F87F10B591EA030F48BF83F0004396
:1004E0003FF580AA841A71EB030C07D28CF0004C04
:1004F000121943EB0C03001B61EB0C014FEA115482
:10050000A4EB135CDFF8A4E11EEA430F18BF9EEAD8
:10051000445F00F0B48021EA045123EA6E035242A2
:10052000C3EB6E0338BF5B1EDCF1200E25D322FA2D
:100530000CFE10EB0E0043FA0CFE41EB0E01CCF169
:10054000200E03FA0EFE10EB0E00CCF1200E51F13E
:10055000000129D401EB045112FA0EF2BDE810405B
:1005600058BF7047401C1CBFB2F1004F70470028B5
:100570000CBF491C20F00100704712EB020E43EB48
:10058000030218BF4FF0010E4EEA4202ACF1200CFC
:10059000DCF11E0E56D943FA0CFE10EB0E00CCF126
:1005A0001E0E51F1FF31D5D50EF1010E12FA0EFEDD
:1005B000404141EB010101EB445C5FEA5C5C10D916
:1005C00001EB045110EBDE7038BFBEF1004FBDE807
:1005D000104018BF704700280CBF491C20F00100D4
:1005E000704734D24FEAD42C24F4006411F5001182
:1005F0001BD0B1FA81F20B3AA41AA41ED2F1200347
:10060000914030FA03F31943904001EBCC7101EBB8
:100610000451002CBDE81040A8BF704701F1C04153
:1006200001F000414FF000007047B0FA80F310FA7B
:1006300003F102D1BDE810407047E41A173C4805A9
:10064000C90AE2E701EB0451BDE8104070474910C8
:100650004FEA300001EB0451BDE8104002E04FF0DA
:10066000000170474A0008BF0042F8D0B2F5001FF1
:1006700028BF704701F000414FF0000070479EEA2C
:10068000445F07D011EA5E0FBDE8104004BF0021AF
:1006900000207047BDE8104070B5FFF747FD00BF70
:1006A00040DFF63E104683F0004170470000E0FF57
:1006B00043004FEAD30C4FEA3C0C43401FBF4007B6
:1006C0000CF1605113F0FE4F70471CF0006F03D126
:1006D0000CF00041002070470CF0004343EA5070DA
:1006E00040EACC0010B500F068F800BF00000092AE
:1006F0004FEA0001FFF710BE4FF00041A1F50021C5
:100700004FF00000704710B5FFF772FB0CBF0120DF
:10071000002010BD10B5FFF76BFB14BF01200020B7
:1007200010BD10B5FFF7E0FB8CBF0120002010BD0D
:1007300010B5FFF7D9FB2CBF0120002010BD10B56C
:10074000FFF70EFC94BF0120002010BD10B5FFF78D
:1007500007FC34BF0120002010BD4FF07E5209E09D
:1007600011F0004204D54042C1F1000138BF491EDA
:1007700042F07E5202F170620B0012BF20235FEA4A
:1007800000017047B1FA81FC01FA0CF1A3EB0C03F4
:1007900020FA03FC41EA0C0102EBC352C3F120032F
:1007A00010FA03FC5CEA416C42EB112018BF5FF0C9
:1007B000806C28BF20F0010070470EF1020E2EF071
:1007C000030E5EF8044B244204D44FEA4102B2F116
:1007D0007F4F11D84FEA4003B3F17F4F0CD80ED1B1
:1007E0004FEAD07C0CEB4C0C0CF1020CB2F17F4FB9
:1007F00008BF4CEBD17C04E04FF0080C01E04FEA5D
:10080000D17C0CEB4C0324FA03F404F00704B4F19C
:10081000040C06D20EEB840CBDE810404CF0010C29
:100820006047DFE80CF0070802024FF00040A0F537
:10083000800010BD0846420018BFD2F1807288BF08
:1008400000F0004010BDF1EE100A4FF6FF71C0F24B
:10085000C03120EA010040F04070E1EE100A70471C
:10086000FF2141EAD050C0057047F0F7FDB8000005
:100870004FBB610567ACDD3F182D4454FB21E93FB8
:100880009BF681D20B73EF3F182D4454FB21F93FA7
:10089000E2652F227F2B7A3C075C143326A6813C2D
:1008A000BDCBF07A8807703C075C143326A6913CD8
:1008B000C4EB98999999C9BF711623FEC671BCBF44
:1008C0006D9A74AFF2B0B3BF9AFDDE522DDEADBFAC
:1008D0002F6C6A2C44B4A2BF0D5555555555D53FC4
:1008E000FF8300922449C23F6E204CC5CD45B73FDF
:1008F000513DD0A0660DB13FEB0D76244B7BA93F57
:1009000011DA22E33AAD903F000000000000000041
:10091000000000006E83F9A22915444ED15727FC30
:10092000C0DD34F5999562DB4190433CAB6351FEE9
:1009300002400000000000A0000000000540000090
:10094000000000C8000000000C4000000000409CB7
:1009500000000000194000000020BCBE00000000A4
:1009600034400000BFC91B8E00000004B5400000E9
:10097000504BCFD06607E2CF010000006C41000071
:100980003E8251AADFEEA73401000000D9420000E8
:10099000DCB5A0E23A301F97FFFFFFFFB44500002F
:1009A000FD25A0C8E9A3C14FFFFFFFFFFF3F0000E7
:1009B0000000008000000000FF3F000000000080F9
:1009C000000000000000000000000000010203041D
:1009D00006070809000000000102030401000000EE
:1009E0000000024010000000000002400100000072
:1009F0000004024010000000000802402000000037
:100A0000000802400008000000100240080000003A
:100A100000180240400000000018024000040000DE
:100A2000001C024000080000001C024000100000F2
:100A3000001C02403009002000000000780900205E
:100A400000000000FD0C0108000000000000000094
:100A5000000000000000000000040000180000007A
:100A60000000000000000000CC0C010800000000A5
:100A70000000000000000000000000000004000072
:100A8000180000000000000000000000CF0C01086A
:100A90000000000000000000000000000000000056
:100AA000000400001800000000000000000000002A
:100AB000E50C01080000000000000000000000003C
:100AC000000000000004000018000000000000000A
:100AD00000000000C80C0108000000000000000039
:100AE00000000000000000000004000018000000EA
:100AF0000000000000000000BE0C01080000000023
:100B000000000000000000000000000000040000E1
:100B1000180000000000000000000000D90C0108CF
:100B200000000000000000000000000000000000C5
:100B30000004000018000000000000000000000099
:100B4000030D01080000000000000000000000008C
:100B50000000000000040000300000000000000061
:100B600000000000F20C010800000000000000007E
:100B70000000000000000000000400001800000059
:100B80000000000000000000C30C0108000000008D
:100B90000000000000000000000000000004000051
:100BA000180000000000000000000000006E5C4221
:100BB000E06C944300109543A0D88643B00C010824
:100BC0000000000000000000000000000000000025
:100BD00000020000180000000000000000000000FB
:100BE000000000000100000000020000AD2C000821
:100BF0000100000002000000000200002D2C00088F
:100C0000020000000400000000020000C52C0008E3
:100C1000030000000800000000020000DD2C0008B6
:100C2000040000001000000000020000052C000875
:100C3000050000002000000000020000692C0008F0
:100C40000600000000000080000800008D2C000855
:100C5000070000000080000001080000992C000837
:100C6000080000008000000000020000F52C0008D1
:100C70000900000000010000010C0000292C000800
:100C80000A0000003040000001010000452C00086F
:100C90009A99193E0000803F00000000000000000B
:100CA0000000803F0000803F0000000000000000C6
:100CB00064656661756C745461736B002C006472BA
:100CC000313600766F666100636D640061690061B2
:100CD0007474695F657374690067696D62616C5FE4
:100CE0006374726C00636861737369735F637472B9
:100CF0006C0073686F6F745F6374726C004554317D
:100D00003673005461736B5F496E697400000000B4
:100D1000700D010800000020B0040000C4010008AC
:100D2000180F010800C00120180000002002000870
:100D3000180F0108B004002004AE01003C020008B6
:100D4000300F010818C00120A03200003C0200084A
:100D50001C00000043000000F8FFFFFF0C00000033
:100D60000E0000000F0000002E0000000000000038
:100D7000111324F4320145FD0C010813B4061420AC
:100D8000212F14082D2E1B082908191D2A012001C6
:100D9000101212220219193A113E01566009CDCCE7
:100DA000CC3E0AD7233C5B803F044ABF041122405B
:100DB0001A2004C14320413CDB0FC918A59A999918
:100DC0003EF94022C01A10301B8040684A3D1C2961
:100DD000402B80BF401301020A1402DA293CC00BE9
:100DE0007A449A99193E1F856BBE1CAE47A1441ADE
:100DF000C0040913CC19640922145A4CB469B021F7
:100E00004A061869C05B3F08EC920333DC42191CA8
:100E10001C010201B529B83A02BE0914C201164BE1
:100E200003023029643EC03F9A99998829902C6624
:100E300066667819F82904399C1A40BC69A8190813
:100E4000390459202B20404429DC4D0AD7233D2862
:100E500039B83DBFDB0FC91C9960192829F049201A
:100E60008960013CCBF041042B20416459B059709A
:100E700039B829747978091E20490C3AA04C49BC2C
:100E80001A40CC5B0C42D80A26C0200C139A991940
:100E900060291859A84E3D6F12833A1C29C0292099
:100EA0002BB4439C312A40206C3333333C99A0014E
:100EB0001E12013C010201081C0202010912015A22
:100EC00003085A04183C060202085A07083A0808A0
:100ED000215A0908811A040F29325A0508A9652BDD
:100EE0000203A449982AC0B01D3F03010417112A28
:100EF00001194113B130140805311B084D04293E76
:100F000013F12F1B081D141A8504C9682169348147
:100F10003210000000000000022B073DFEF7BBB8B6
:100F2000DD098A3BDE7772BC01000000AAAAAAAAEA
:040000050800018965
:00000001FF
